:04000000ABEF00F072
:100008005682D9CF08F0DACF09F0899289940F0186
:1000180012A918D08EA802D083A20ED0899425EEFA
:1000280004F0010EDBBE07D0DB5003E1020EDE5CFC
:1000380002E3899201D089828EB883B201D0898483
:1000480012997DD012A17BD08EB883B28992901C70
:100058000A6E8E1C0B6E04C50CF005C50DF00DBEA6
:1000680003D0020E0D5C2FE28EA802D083A22BD003
:100078000C4A0D2A0CC004F50DC005F502C50CF09C
:1000880003C50DF0060E0C24D96E050E0D20DA6E90
:100098000AC0DFFF060E0C24D96E070E0D20DA6E9B
:1000A8000BC0DFFF0C4A0D2A0468010E056E0CC058
:1000B80006F00DC007F0045006160550071606C0D6
:1000C80002F507C003F58EB883B2898489848EA0AF
:1000D800FED78EA802D083A202D0899401D0898449
:1000E8000BA81FD00BD0838202D0838405D08394C1
:1000F80018D083A216D08394839213D00A507F0B12
:10010800046E056A05500DE10450040AF2E0100A75
:10011800F0E0340AE8E01F0AEFE07F0AE6E01F0A91
:10012800E6E025EE04F0010EDBBE06D0DB5002E16E
:10013800DE0402E3899201D089820F0112910E0137
:10014800CA9909C0DAFF08C0D9FF5692110065EFB5
:1001580053F07DC0D9FF7EC0DAFFDE6ADD6A7CC05D
:100168000EF01BEC4BF00EC098F00FC099F0000198
:1001780099BF0B0CD8909835D96E9935DA6E4E0E1A
:10018800D926010EDA22DECFAFF0DDCFB0F0AF51C5
:10019800B01101E10C0C7DC0D9FF7EC0DAFFAFC001
:1001A800DEFFB0C0DDFF7F91AFC0D9FFB0C0DAFF7E
:1001B800DF5012E020EE01F0AF51D926B051DA221B
:1001C800DF5013EC68F00001A46FA4B105D07F5193
:1001D800D8A4A4A5000C0A0CAFC0D9FFB0C0DAFFA0
:1001E800DF6A20EE01F0AF51D926B051DA2298C06B
:1001F800DFFF20EE01F0AF51D926B051DA22DF50EF
:10020800BCEC47F00001A46FA4B1030C7F5102E0DD
:10021800A4B50A0CAFC060F0B0C061F0636B626B4C
:10022800B6EC4BF060C0ADF061C0AEF0040EAD1995
:10023800AE1101E1010CAE5103E1020EAD5D01E327
:100248000D0C20EE2BF0AF51D926B051DA22DECFBB
:10025800A0F0DECFA1F0DECFA2F0DECFA3F03A0E01
:10026800AF250E6E000EB0210F6E0EEC66F0020E7A
:100278000F180E1001E00D0C450E0001AF250E6E93
:10028800000EB0210F6E0EEC66F00EC0A9F00FC084
:10029800AAF00001AB6BAC6BA951AA11AB11AC1160
:1002A80010E1530EAF250E6E000EB0210F6ED8EC84
:1002B80059F00EC0A9F00FC0AAF010C0ABF011C0E1
:1002C800ACF0000120EE17F0AF51D926B051DA2278
:1002D800A9C0DEFFAAC0DEFFABC0DEFFACC0DEFFF8
:1002E80020EE3FF0AF51D926B051DA2210EE02F0DD
:1002F800AF51E126B051E222DFCFE7FF20EE02F056
:10030800AF51D926B051DA22DE040AE020EE02F01D
:10031800AF51D926B051DA22020EDE1801E00D0CD9
:10032800A9C00EF0AAC00FF0ABC010F0ACC011F01D
:1003380020EE02F0AF51D926B051DA22DF50126E0A
:10034800136A146A156A81EC5EF00EC0A9F00FC03A
:10035800AAF010C0ABF011C0ACF020EE3CF0AF51E9
:10036800D926B051DA22DF50806F816B20EE09F078
:10037800AF51D926B051DA2280C0DEFF81C0DDFF3F
:1003880020EE09F0AF51D926B051DA22DE50DE1046
:10039800D8B40D0C20EE09F0AF51D926B051DA22AD
:1003A800DECF80F0DDCF81F08269836920EE09F02D
:1003B800AF51D926B051DA22DECF84F0DDCF85F0F7
:1003C8008251842783518523805184178151851751
:1003D8008451851101E00D0C400EAF250E6E000E04
:1003E800B0210F6E0EEC66F0000120EE07F0AF5161
:1003F800D926B051DA220EC0DEFF0FC0DDFF20EE95
:1004080007F0AF51D926B051DA22DF50806F0F0EB6
:10041800801701E00D0C420EAF250E6E000EB021C4
:100428000F6E0EEC66F00EC09CF00FC09DF0000140
:100438009E6B9F6B9C519D119E119F1110E14F0E59
:10044800AF250E6E000EB0210F6ED8EC59F00EC01D
:100458009CF00FC09DF010C09EF011C09FF03D0EA3
:100468000001AF250E6E000EB0210F6E0EEC66F087
:100478000EC09AF00FC09BF000019A519B1101E148
:100488000D0C20EE07F0AF51D926B051DA22DECF9D
:1004980080F0DDCF81F0040E826FD89081338033F5
:1004A800822FFBD79A518025836F9B518121846FBE
:1004B800856BD8B0852B866BA9518325946FAA517B
:1004C8008421956FAB518521966FAC518621976F2A
:1004D80094519C5D95519D5996519E5997519F599C
:1004E80001E20D0C94519C5D0E6E95519D590F6E55
:1004F80096519E59106E97519F59116E20EE09F032
:10050800AF51D926B051DA22DECF80F0DDCF81F0AD
:1005180080C012F081C013F0146A156A3EEC5FF0D7
:100528000EC0A5F00FC0A6F010C0A7F011C0A8F02B
:100538000001A551A611A711A81101E10D0CAD6B81
:10054800AE6BF60EA55DFF0EA659FF0EA7590F0E4E
:10055800A85903E2AE6B030EAD6FA851A71108E1CD
:10056800F60EA55DFF0EA65903E2AE6B020EAD6F47
:10057800A851A71108E1F60EA55D0F0EA65903E2D2
:10058800AE6B010EAD6FAD51AE1101E10D0C020E57
:10059800A525806F000EA621816F000EA721826F0E
:1005A800000EA821836F20EE13F0AF51D926B05169
:1005B800DA2280C0DEFF81C0DEFF82C0DEFF83C09A
:1005C800DEFF20EE1BF0AF51D926B051DA22A0C0D1
:1005D800DEFFA1C0DEFFA2C0DEFFA3C0DEFF9A518E
:1005E800A025806F9B51A121816F000EA221826FEF
:1005F800000EA321836F20EE1FF0AF51D926B05112
:10060800DA2280C0DEFF81C0DEFF82C0DEFF83C049
:10061800DEFF9451A025806F9551A121816F9651DD
:10062800A221826F9751A321836F20EE27F0AF514B
:10063800D926B051DA2280C0DEFF81C0DEFF82C039
:10064800DEFF83C0DEFF030EAD19AE114DE1590E7A
:10065800AF250E6E000EB0210F6E0EEC66F00E5038
:100668000F1001E00D0C000120EE07F0AF51D92664
:10067800B051DA22DE50DE1001E00D0C5B0EAF2522
:100688000E6E000EB0210F6ED8EC59F0000120EE6E
:1006980023F0AF51D926B051DA220EC0DEFF0FC0C9
:1006A800DEFF10C0DEFF11C0DEFF20EE13F0AF51F9
:1006B800D926B051DA22DECF80F0DECF81F0DECF4E
:1006C80082F0DECF83F0020ED890803781378237F0
:1006D8008337E82EF9D780C090F081C091F082C0AE
:1006E80092F083C093F0B8D020EE07F0AF51D9262E
:1006F800B051DA22DE50DE1001E10D0C20EE1FF0C1
:10070800AF51D926B051DA22DECF80F0DECF81F0AA
:10071800DECF82F0DECF83F0A9518025846FAA5105
:100728008121856FAB518221866FAC518321876F00
:1007380020EE23F0AF51D926B051DA2284C0DEFF73
:1007480085C0DEFF86C0DEFF87C0DEFF020EAD1962
:10075800AE116BE020EE13F0AF51D926B051DA227A
:10076800DECF80F0DECF81F0DECF82F0DECF83F007
:10077800010E8015846F856B866B876B20EE13F0F6
:10078800AF51D926B051DA22DECF88F0DECF89F01A
:10079800DECF8AF0DECF8BF0030E8803F3CF8CF028
:1007A800F4CF8DF08E6B8F6B8903F3508D27F45047
:1007B8008E23000E8F238803F3508D27F4508E2349
:1007C800000E8F23030E8A03F3508E27F4508F23D5
:1007D800000E8903F3508E27F4508F23000E8803F0
:1007E800F3508E27F4508F23030E8B03F3508F277B
:1007F800000E8A03F3508F27000E8903F3508F27CA
:10080800000E8803F3508F27D8908F338E338D33A3
:100818008C3384518C25906F85518D21916F865131
:100828008E21926F87518F2116D020EE13F0AF5191
:10083800D926B051DA22DECF80F0DECF81F0DECFCC
:1008480082F0DECF83F0D8908035906F8135916F3C
:100858008235926F8335936FFF0E9025806F010E5E
:100868009121816F000E9221826F000E9321836F78
:100878000A0E05D0D8908333823381338033E82E33
:10088800F9D720EE17F0AF51D926B051DA228051AE
:10089800DE5C8151DE588251DE588351DE5801E218
:1008A8000D0C20EE0FF0AF51D926B051DA22DE68D8
:1008B800DE68DE68DD68DD52DD5210EE0BF0AF5108
:1008C800E126B051E222DECFE6FFDECFE6FFDECF43
:1008D800E6FFDECFE6FF20EE04F0AF51D926B05197
:1008E800DA22800EDF6E030EAD19AE1101E090D052
:1008F8005F0EAF250E6E000EB0210F6E0EEC66F087
:100908000E040F1001E084D0AFC03AF0B0C03BF045
:10091800010E0001A0253C6E000EA1213D6E000EC7
:10092800A2213E6E000EA3213F6E1BEC5BF0000976
:100938006FE1000120EE04F0AF51D926B051DA2260
:10094800DF6A2D0EAF250E6E020EB0210F6E0EEC73
:1009580066F0550E0E185CE1AA0E0F1859E12F0E1D
:100968000001AF250E6E000EB0210F6ED8EC59F0C5
:10097800520E0E184DE1520E0F184AE1610E101872
:1009880047E1410E111844E1130E0001AF250E6E28
:10099800020EB0210F6ED8EC59F0720E0E1838E125
:1009A800720E0F1835E1410E101832E1610E111860
:1009B8002FE1170E0001AF250E6E020EB0210F6E4B
:1009C800D8EC59F0000120EE0FF0AF51D926B05104
:1009D800DA220EC0DEFF0FC0DEFF10C0DEFF11C03E
:1009E800DEFF1B0EAF250E6E020EB0210F6ED8EC87
:1009F80059F0000120EE0BF0AF51D926B051DA22A0
:100A08000EC0DEFF0FC0DEFF10C0DEFF11C0DEFF2C
:100A1800AFC0D9FFB0C0DAFFADC0DFFF01014C4B5A
:100A28004D2B000120EE05F0AF51D926B051DA2246
:100A38004CC1DEFF4DC1DDFF000C87C042F088C00D
:100A480043F00101426B436BAFD385C03CF086C0D5
:100A58003DF0420E3E6E89C03FF03E50D96EDA6AD4
:100A6800DECFF6FFDDCFF7FFF86A000EF86E08005C
:100A7800F550250AD8A478D33E50D96EDA6ADE2A12
:100A8800000EDD220101446B456B4C6A4D6A4669D4
:100A980047693E50D96EDA6ADECFF6FFDDCFF7FF41
:100AA800F86A000EF86E0800F550640AD8B40FD042
:100AB8003E50D96EDA6ADECFF6FFDDCFF7FFF86A6F
:100AC800000EF86E0800F550690AD8A48AD13E5085
:100AD800D96EDA6ADE2A000EDD223F50D96EDA6A54
:100AE800DF50DF2ADF2AD96EDA6ADECF74F0DDCF75
:100AF80075F00001000E75BFFF0E766F776F786F87
:100B0800796F7A6F7B6F3CC02AF03DC02BF074C0C0
:100B18002CF075C02DF076C02EF077C02FF078C07D
:100B280030F079C031F07AC032F07BC033F02CC09D
:100B380068F02DC069F02EC06AF02FC06BF030C08D
:100B48006CF031C06DF032C06EF033C06FF06FAF33
:100B580002D0010E01D0000E666F676B66516711F7
:100B6800D8B410D06F1F6E1F6D1F6C1F6B1F6A1FCC
:100B7800691F686D000E69236A236B236C236D233C
:100B88006E236F23010147BF01D04C9247BF05D0A8
:100B9800475108E14605D8B005D00001636B010E46
:100BA800626F04D046C162F047C163F044C164F08B
:100BB80045C165F0000166516711D8A402D04CA464
:100BC80003D06407D8A06507716B1F0E706F020110
:100BD800976B6ED07007D8A07107780E7025D96E04
:100BE800020E7121DA6E68C00EF069C00FF06AC09B
:100BF80010F06BC011F06CC012F06DC013F06EC035
:100C080014F06FC015F00A0E166E176A186A196A82
:100C18001A6A1B6A1C6A1D6A26EC4FF00EC034F073
:100C28000FC035F010C036F011C037F012C038F0E0
:100C380013C039F014C03AF015C03BF034C020F0AE
:100C480036C021F072EC66F02050300FDF6E62077C
:100C5800D8A063076407D8A0650768C00EF069C00C
:100C68000FF06AC010F06BC011F06CC012F06DC0CC
:100C780013F06EC014F06FC015F00A0E166E176AE6
:100C8800186A196A1A6A1B6A1C6A1D6A79EC4AF0A2
:100C98000EC068F00FC069F010C06AF011C06BF0A8
:100CA80012C06CF013C06DF014C06EF015C06FF078
:100CB800000171BF1FD0715103E17005D8A01AD08F
:100CC800685169116A116B116C116D116E116F11F8
:100CD800D8A480D763BF05D0635102E16205D8B0BC
:100CE80079D765BF07D0655103E16405D8A002D064
:100CF8004CB270D766516711D8A402D04CA415D055
:100D08007007D8A0710766516711D8A403D0616B2A
:100D18002B0E02D0616B2D0E606F780E7025D96E88
:100D2800020E7121DA6E60C0DFFF2AC01FF02BC0EF
:100D380020F0780E7025216E020E7121226E64C09B
:100D480023F065C024F04CA00AD021C018F022C0BE
:100D580019F01FC01AF020C01BF028EC66F024BE62
:100D680005D023C028F024C029F002D0286A296AB7
:100D7800266A276A0BD0106A200E0F6E1FC011F06A
:100D880020C012F069EC5BF0264A272A2850265C1E
:100D98002750800A256E2950800A2558D8A0EBD7FD
:100DA8004CB00AD021C018F022C019F01FC01AF0A8
:100DB80020C01BF028EC66F021C00EF022C00FF016
:100DC800F9EC63F028500E241F6E29500F20206E76
:100DD8001FC02AF020C02BF02AC03CF02BC03DF0E9
:100DE800DED13E50D96EDA6ADECFF6FFDDCFF7FFEF
:100DF800F86A000EF86E0800F550780AD8B40FD0DB
:100E08003E50D96EDA6ADECFF6FFDDCFF7FFF86A1B
:100E1800000EF86E0800F550580AD8A47AD13E5052
:100E2800D96EDA6ADECFF6FFDDCFF7FFF86A000E7B
:100E3800F86E0800F5CF84F03E50D96EDA6ADE2AE3
:100E4800000EDD223F50D96EDA6ADF50DF2ADF2A32
:100E5800D96EDA6ADECF40F0DDCF41F040C07CF0D9
:100E680041C07DF000017E6B7F6B806B816B826B74
:100E7800836B3CC02AF03DC02BF07CC02CF07DC0B9
:100E88002DF07EC02EF07FC02FF080C030F081C0E2
:100E980031F082C032F083C033F084C034F00101F5
:100EA80047BF01D04C9247BF05D0475108E14605DE
:100EB800D8B005D00001656B010E646F04D046C13F
:100EC80064F047C165F044C16EF045C16FF04CA8AD
:100ED80005D00001FE0E6E27FF0E6F232CC066F0B2
:100EE8002DC067F02EC068F02FC069F030C06AF0DE
:100EF80031C06BF032C06CF033C06DF00001736B21
:100F08001F0E726F0201976B6DD07207D8A073071E
:100F18000F0E6615706F716B71BF08D0715104E1C7
:100F28000A0E705DD8A002D0570E01D0300E70277F
:100F3800000E7123BF0E356E36683450376E386A2E
:100F48003550372636503822385005E11A0E375CAE
:100F580002E2010E01D0000E606F616B60516111F9
:100F6800D8B425D09F0E356E3668200E7011376EB6
:100F7800000E7111386E35503726365038223850E9
:100F880005E11A0E375C02E2010E01D0000E626F15
:100F9800636B62516311D8B40AD070C014F071C089
:100FA80015F0B6EC63F014C070F015C071F0780E4F
:100FB8007225D96E020E7321DA6E70C0DFFF6407E6
:100FC800D8A065076E07D8A06F07040E356ED890B5
:100FD8006D336C336B336A33693368336733663325
:100FE800352EF5D7000173BF20D0735104E1020EEE
:100FF800725DD8A01AD066516711681169116A111B
:101008006B116C116D11D8A480D765BF05D06551DF
:1010180002E16405D8B079D76FBF07D06F5103E1FB
:101028006E05D8A002D04CB270D74CA816D0720763
:10103800D8A07307780E7225D96E020E7321DA6E66
:1010480034C0DFFF7207D8A07307780E7225D96EF7
:10105800020E7321DA6E300EDF6E2AC01FF02BC02D
:1010680020F0780E7225216E020E7321226E6EC05A
:1010780023F06FC024F04CA00AD021C018F022C081
:1010880019F01FC01AF020C01BF028EC66F024BE2F
:1010980005D023C028F024C029F002D0286A296A84
:1010A800266A276A0BD0106A200E0F6E1FC011F037
:1010B80020C012F069EC5BF0264A272A2850265CEB
:1010C8002750800A256E2950800A2558D8A0EBD7CA
:1010D8004CB00AD021C018F022C019F01FC01AF075
:1010E80020C01BF028EC66F021C00EF022C00FF0E3
:1010F800F9EC63F028500E241F6E29500F20206E43
:101108001FC02AF020C02BF02AC03CF02BC03DF0B5
:1011180046D03E50D96EDA6ADECFF6FFDDCFF7FF54
:10112800F86A000EF86E0800F550250AD8A413D006
:101138003E50D96EDA6ADE2A000EDD22106A250ECC
:101148000F6E3CC011F03DC012F069EC5BF03D6AD7
:10115800010E3C6E24D03E50D96EDA6ADE2A000EAB
:10116800DD223C6A3D6A1BD03E50D96EDA6ADECF7A
:10117800F6FFDDCFF7FFF86A000EF86E0800F550AD
:101188000F6E106A3CC011F03DC012F069EC5BF0C4
:101198003E50D96EDA6ADE2A000EDD22D8D73C50DE
:1011A800010142273D50432342C0F6FF43C0F7FFE9
:1011B8000800F55001E049D442C185F043C186F0EA
:1011C80012004A6E496AD1D2090E4A1817E15250E4
:1011D80015E0496A8390496A010E516E53501E0DFD
:1011E8001B0EF324D96E020EF420DA6E200EDF6E89
:1011F800030E01015F6F4E6A4F6A83904A5008E1FF
:10120800525006E0496A4F6A0A0EAAD0839025D345
:10121800020E4A1806E1525004E0496A4F6A140E59
:101228009FD01F0E4A6438D0300E4A6035D05250D5
:1012380033E04A50E00F536E496A0F0E531805E128
:101248005EC151F001015E6B8DD25350220D0A0E22
:10125800F324D96E030EF420DA6EDE50DE10DE10B1
:10126800DE1003E0030E53647DD2536A010E516E03
:1012780053501E0D1B0EF324D96E020EF420DA6EA5
:1012880053501E0D1B0EF324E16E020EF420E26E85
:10129800E7501009DF6E66D23F0E4A6428D0480E28
:1012A8004A6025D0525023E053501E0D000EF324FF
:1012B800D96E020EF420DA6E4A50C00FDF6E53501A
:1012C8001E0D000EF324D96E020EF420DA6EDF50E4
:1012D8000CE053501E0D1B0EF324D96E020EF420A1
:1012E800DA6E100EDF6E010E516E496A3BD2480E5F
:1012F8004A1807E1525005E0496A120E4F6EC00EB7
:101308002FD0310E4A1806E1525004E00C0E4F6EF1
:101318001D0E12D2340E4A1806E1525004E04E6AED
:101328004F6A496A73D7350E4A1807E1525005E0EB
:10133800496A0D0E4F6EAC0E13D0370E4A1807E1EE
:10134800525005E083800E0E4F6E750EF5D10D0ECE
:101358004A1808E1525006E0496A020E4F6EBC0E68
:101368004E6E54D7100E4A1806E1525004E0030E90
:101378004F6EE90EE1D1180E4A1806E1525004E00A
:10138800070E4F6E090ED8D13B0E4A1806E152508F
:1013980004E00E0E4F6E7E0ECFD13E0E4A1801E0CD
:1013A8005CD2525001E159D20F0E4F6E3D0EC4D19E
:1013B80053501E0D010EF324D96E020EF420DA6E7E
:1013C8004AC0DFFF030E4F6EEA0EB6D153501E0D12
:1013D800020EF324D96E020EF420DA6E4AC0DFFF43
:1013E800030E4F6EEB0EA8D153501E0D030EF324BF
:1013F800D96E020EF420DA6E4AC0DFFF030E4F6E7C
:10140800EC0E9AD153501E0D040EF324D96E020E21
:10141800F420DA6E4AC0DFFF030E4F6EED0E8CD15A
:1014280053501E0D050EF324D96E020EF420DA6E09
:101438004AC0DFFF030E4F6EEE0E7ED153501E0DD5
:10144800060EF324D96E020EF420DA6E4AC0DFFFCE
:1014580053501E0D050EF324D96E020EF420DA6ED9
:10146800DF50266E26C027F0286A296A2A6A29C012
:101478002AF028C029F027C028F0276A53501E0DEB
:10148800040EF324D96E020EF420DA6EDF502B6EB0
:101498002BC02CF02D6A2E6A2F6A2DC02FF02CC07D
:1014A8002EF02D6A2C6A53501E0D030EF324D96EAC
:1014B800020EF420DA6EDF50306E30C031F0326A3E
:1014C800336A346A31C034F0336A326A316A2C5074
:1014D8003124356E2D503220366E2E503320376E23
:1014E8002F503420386E27503524396E2850362036
:1014F8003A6E295037203B6E2A5038203C6E5350A4
:101508001E0D060EF324D96E020EF420DA6EDF509B
:1015180039243D6E000E3A203E6E000E3B203F6E91
:10152800000E3C20406E3DC041F03EC042F03FC03E
:1015380043F040C044F0456A44BE456845C046F0A3
:1015480045C047F045C048F053501E0D070EF32420
:10155800D96E020EF420DA6E41C0DEFF42C0DEFF13
:1015680043C0DEFF44C0DEFF45C0DEFF46C0DEFFED
:1015780047C0DEFF48C0DEFF53501E0D1C0EF3248B
:10158800D96E020EF420DA6EDECF26F0DDCF27F01A
:1015980026C00EF027C00FF0106A116A126A136A8B
:1015A800146A156A53501E0D070EF324D96E020EE5
:1015B800F420DA6EDECF28F0DECF29F0DECF2AF075
:1015C800DECF2BF0DECF2CF0DECF2DF0DECF2EF0ED
:1015D800DECF2FF028C016F029C017F02AC018F067
:1015E8002BC019F02CC01AF02DC01BF02EC01CF017
:1015F8002FC01DF0B5EC5DF00EC030F00FC031F01B
:1016080010C032F011C033F012C034F013C035F0FE
:1016180014C036F015C037F053501E0D070EF324D2
:10162800D96E020EF420DA6E30C0DEFF31C0DEFF64
:1016380032C0DEFF33C0DEFF34C0DEFF35C0DEFF60
:1016480036C0DEFF37C0DEFF83904E6A4F6A05D191
:1016580053501E0D1A0EF324D96E020EF420DA6EC2
:101668004AC0DFFF070E4F6E0A0E66D053501E0D9C
:10167800190EF324D96E020EF420DA6E4AC0DFFF89
:10168800070E4F6E0B0E58D053501E0D180EF32434
:10169800D96E020EF420DA6E4AC0DFFF070E4F6ED5
:1016A8000C0E4AD053501E0D170EF324D96E020E9D
:1016B800F420DA6E4AC0DFFF55D04E6A4F6A516A8D
:1016C800A5D54AC030F10F0E4F6E3E0E35D04AC038
:1016D80031F10F0E4F6E3F0E2FD04AC032F10F0E70
:1016E8004F6E400E29D04AC033F10F0E4F6E410E97
:1016F80023D04AC034F10F0E4F6E420E1DD04AC09F
:1017080035F10F0E4F6E430E17D04AC036F10F0E4B
:101718004F6E440E11D04AC037F124D00C0E4F6ED4
:101728001E0E0AD00C0E4F6E1C0E4E6E0A0E496E1F
:101738006DD50E0E4F6E760E4E6E8FD04E6A4F6A76
:10174800090E496E838089D04A500CE053501E0D13
:101758001B0EF324D96E020EF420DA6E080EDF6E2B
:10176800010E516E4E6A4F6A51D54EC026F04FC0D9
:1017780027F0275013E0030A15E0040A27E00B0AB4
:1017880033E0010A37E0030A3BE0010A42E01D0AA0
:101798005AE00E0A5DE03B0A5EE05FD0265001E1A8
:1017A80013D55BD02650E90A01E102D6030A01E10C
:1017B8000DD6010A01E118D6070A01E123D6010A6C
:1017C80001E12ED6030A01E139D647D02650090A8D
:1017D80001E13ED7030A01E149D7010A01E154D7E3
:1017E800070A01E15FD739D026501D0A97E0030A9E
:1017F80099E033D02650480A01E127D7E40A2DD0D2
:101808002650750A96E0030A99E0080A01E155D7BF
:1018180024D026503D0A01E154D7030A01E157D7E5
:10182800010A01E15AD77F0A01E15DD7010A01E106
:1018380060D7030A01E163D7010A01E166D7070A05
:1018480001E169D70AD02650C00A01E17DD705D049
:1018580026502A0A02D026500F0A49501200A0C06A
:10186800B6F0A1C0B7F0A451D96EDA6ADE6ADD6AB3
:101878009EC00FF09FC010F0C60E116E82EC59F09A
:101888000001B56FB5510AE120EE0FF09E51D9263F
:101898009F51DA22DF50B56FB55102E0B551120001
:1018A80020EE0EF09E51D9269F51DA22DFA2070CB6
:1018B80020EE10F09E51D9269F51DA2210EE10F03A
:1018C8009E51E1269F51E222E6CFA9F0E6CFAAF089
:1018D800E6CFABF0E6CFACF0A251A925AD6FA3518E
:1018E800AA21AE6F000EAB21AF6F000EAC21B06F16
:1018F800DE50AD5DDE50AE59DE50AF59DE50B05906
:1019080001E3DFD220EE10F09E51D9269F51DA2252
:10191800DECFA5F0DDCFA6F0A51DA26FA61DA36F93
:10192800D0D220EE10F09E51D9269F51DA22FF0E18
:10193800DE14A56F010EDE14A66F000EDE14A76F6D
:10194800000EDE14A86FA551A611A711A81101E079
:10195800FDD120EE10F09E51D9269F51DA22DECF1C
:10196800A5F0DECFA6F0DECFA7F0DECFA8F00A0EF6
:1019780005D0D890A833A733A633A533E82EF9D7D6
:10198800A969AA6920EE09F0C651D926C751DA22F9
:10199800DECFABF0DDCFACF0A951AB27AA51AC2319
:1019A800A551AB15B86FA651AC15B96FB81101E0C8
:1019B80091D020EE10F09E51D9269F51DA22DE50A8
:1019C800DE10DE10DE101EE120EE06F09E51D92654
:1019D8009F51DA22DECFC0F0DECFC1F0DECFC2F0F9
:1019E800DECFC3F0C051C111C211C31127E19EC09F
:1019F80081F09FC082F0836B846B856B866B8EEC65
:101A08002AF014D09EC081F09FC082F020EE14F01E
:101A18009E51D9269F51DA22DECF83F0DECF84F0A3
:101A2800DECF85F0DECF86F08EEC2AF081C0C0F0E4
:101A380082C0C1F083C0C2F084C0C3F0C051C111DC
:101A4800C211C31101E141D2C005C111C211C311B4
:101A580009E120EE0FF09E51D9269F51DA22020E9D
:101A6800DF6E020CC0290FE1C1290DE1C2290BE18B
:101A7800C32909E120EE0FF09E51D9269F51DA22A1
:101A8800010EDF6E010C20EE14F09E51D9269F51F5
:101A9800DA22C0C0DEFFC1C0DEFFC2C0DEFFC3C0A5
:101AA800DEFF20EE06F09E51D9269F51DA22DE5045
:101AB800DE10DE10DE100EE120EE06F09E51D92673
:101AC8009F51DA22C0C0DEFFC1C0DEFFC2C0DEFF08
:101AD800C3C0DEFF20EE18F09E51D9269F51DA22AE
:101AE80010EE2BF0C651E126C751E222DE50E6186F
:101AF80012E1DE50E6180FE1DE50E6180CE1DE5088
:101B0800E61809E1C6C027F0C7C028F07AEC48F00B
:101B1800000901E053D1C6C00EF0C7C00FF00001A4
:101B280020EE14F09E51D9269F51DA22DECF10F014
:101B3800DECF11F0DECF12F0DECF13F0CEEC50F096
:101B48000EC0BCF00FC0BDF010C0BEF011C0BFF099
:101B58000001BC51BD11BE11BF1101E17AD7B851C6
:101B6800BC27B951BD23000EBE23BF23A2C0A5F0D8
:101B7800A3C0A6F0090EA76FD890A633A533A72F48
:101B8800FBD7A5C0BAF0A6C0BBF0BA51BB1101E1A2
:101B9800A2D0BA51B825A56FBB51B921A66F20EEC6
:101BA80009F0C651D926C751DA22A551DE5CA651E3
:101BB800DE5810E220EE09F0C651D926C751DA22C4
:101BC800DECFA5F0DDCFA6F0B851A55DBA6FB9514B
:101BD800A659BB6FB6C01DF0B7C01EF0BCC01FF041
:101BE800BDC020F0BEC021F0BFC022F0BAC023F0B3
:101BF800BBC024F020EE01F0C651D926C751DA2225
:101C0800DF50BCEC56F0000901E0D8D00001BA5111
:101C1800A56FBB51A66FA76BA86B20EE2BF0C65122
:101C2800D926C751DA22DECFA9F0DECFAAF0DECF5F
:101C3800ABF0DECFACF0BC51A95DAD6FBD51AA5978
:101C4800AE6FBE51AB59AF6FBF51AC59B06FA55114
:101C5800AD5DA651AE59A751AF59A851B0592CE264
:101C68002F0EC6250E6E000EC7210F6E20EE2BF02C
:101C7800C651D926C751DA22DECFA5F0DDCFA6F0AE
:101C8800BC51A55FBD51A65B090ED890A537A637F4
:101C9800E82EFBD7A551B625106EA651B721116EB7
:101CA800020E136E126A1AEC64F020EE03F0C651AD
:101CB800D926C751DA22DF6ABAC0A5F0BBC0A6F0A0
:101CC800090ED890A537A637E82EFBD7A5C0C4F0D3
:101CD800A6C0C5F0A7D020EE0AF09E51D9269F5184
:101CE800DA2210EE10F09E51E1269F51E222DE50DA
:101CF800E65CDE50E658DE50E658DE50E65818E35B
:101D0800C6C027F0C7C028F07AEC48F0000901E007
:101D180055D0000120EE2BF0C651D926C751DA2242
:101D2800BCC0DEFFBDC0DEFFBEC0DEFFBFC0DEFF41
:101D380020EE18F09E51D9269F51DA22BCC0DEFF52
:101D4800BDC0DEFFBEC0DEFFBFC0DEFFA569010E5D
:101D5800A66F20EE10F09E51D9269F51DA22DECFD1
:101D6800A7F0DDCFA8F0A551A717A651A817A7512E
:101D78000008C46FA851D8A0E82A0208C56FC4514A
:101D8800A25DC551A35904E2A2C0C4F0A3C0C5F026
:101D9800C6C03AF0C7C03BF020EE18F09E51D926D5
:101DA8009F51DA22DECF3CF0DECF3DF0DECF3EF0B1
:101DB800DECF3FF01BEC5BF0000902E000015AD6D1
:101DC8000001A569010EA66F20EE10F09E51D926DC
:101DD8009F51DA22DECFA7F0DDCFA8F0A551A717D3
:101DE800A651A817C6C0A9F0C7C0AAF0A751A9272D
:101DF800A851AA232F0EA9250E6E000EAA210F6E38
:101E0800B6C010F0B7C011F0C4C012F0C5C013F0CE
:101E18001AEC64F020EE03F0C651D926C751DA2235
:101E2800010EDF6EC451A25FC551A35BA451D96EE8
:101E3800DA6AC451DE26C551DD22C451B627C55120
:101E4800B72320EE10F09E51D9269F51DA22C451B3
:101E5800DE26C551DE22000EDE22DE2220EE10F044
:101E68009E51D9269F51DA2210EE0AF09E51E126A2
:101E78009F51E222DE50E65CDE50E658DE50E6581E
:101E8800DE50E65820EE0AF0D8A020EE10F09E5161
:101E9800D9269F51DA22DECFB1F0DECFB2F0DECF05
:101EA800B3F0DECFB4F020EE0AF09E51D9269F5150
:101EB800DA22B1C0DEFFB2C0DEFFB3C0DEFFB4C0BD
:101EC800DEFFA251A31101E02CD520EE0EF09E51A9
:101ED800D9269F51DA22000EDB8C000C0F6A0E6A9D
:101EE800CEEC67F00101FA6F636B0F010D6B156B98
:101EF8001D6B226B070E8C6E010E0101FB6F696B67
:101F08000F0E0F01596F116B196B216B266B2E6B1E
:101F18000E6B166B1E6B236B2B6B886889688A683F
:101F28008A8E889088928382020E026EE2EC66F0B6
:101F380088948384888C839C889E838E8B68896828
:101F4800060E00019C6FF90E9D6FA90E9E6FFF0E85
:101F58009F6FA30EA06FFE0EA16F2E0EA26FFF0E35
:101F6800A36FF0EC67F08A98858841EC66F04F0E15
:101F780000019C6FFB0E9D6FFAC19EF09F6BF0EC09
:101F880067F00101FA2901E1FA6B0F0EFA1741EC2B
:101F980050F00101FA6F670E00019C6FFB0E9D6FF8
:101FA800FAC19EF09F6BF0EC67F00400520E01013D
:101FB800B16F2B0EB06F000EE82EFED7B02FFCD7F6
:101FC800B12FFAD700F0D250F00B0109D26ED09E93
:101FD8000E01C691CF0ECF16CF82CF80C2890F01D6
:101FE800138113891489F28E0E01BA8979EC5FF096
:101FF8008392839449EC56F049EC56F0000E0E6E2D
:10200800340E1FEC63F0490E126EFF0E136E01ECD6
:102018005FF0A90E126EFF0E136E01EC5FF0000E5A
:102028000E6E390E1FEC63F08FA22FD0290E01011E
:10203800B16F960EB06F7F0EE82EFED7B02FFCD78B
:10204800B12FFAD7000E0E6E800E1FEC63F0160E3D
:10205800126EFE0E136E01EC5FF017D0580E0001E1
:102068009C6FFE0E9D6F8FCF9EF09F6BF0EC67F01C
:10207800290E0101B16F960EB06F7F0EE82EFED7C4
:10208800B02FFCD7B12FFAD704008FB2E7D78380DF
:10209800040098EC4EF00101B66FA6EC38F001018F
:1020A800B66FFB050EE167510CE1430E00019C6F12
:1020B800FD0E9D6FF0EC67F0020E0101676F220EB6
:1020C800666FFB510EE167510CE1330E00019C6F06
:1020D800FD0E9D6FF0EC67F0010E0101676F040EB5
:1020E800666F625102E04CEC45F0CFC193FF57ECAC
:1020F80032F0CBEC58F0000E0E6E800E1FEC63F041
:10210800F7EC66F0000E0E6E800E1FEC63F0010116
:10211800FA510F0D350EF324126E0D0EF420136EC6
:1021280001EC5FF0010169BFD5EC49F00101B56B25
:10213800BA6B000EB86F010EB76FB8BF05D0B851B3
:1021480066E1040EB75D63E20F0EB703F3CFB0F19B
:10215800F4CFB1F1B803F350B127250EB0250E6EB8
:102168000E0EB1210F6EF9EC63F00F5003E1030E70
:102178000E5C49E3A00E00019C6FFD0E9D6F0F0ED3
:102188000101B703F3CFB0F1F4CFB1F1B803F350C5
:10219800B127250EB02500019E6F0E0E0101B12159
:1021A80000019F6FF0EC67F0220E0101B703F3CF37
:1021B800B0F1F4CFB1F1B803F350B127000EB02558
:1021C8000001CE6F030E0101B1210001CF6F0F0E88
:1021D8000101B703F3CFB2F1F4CFB3F1B803F35071
:1021E800B327250EB2250001D06F0E0E0101B321D1
:1021F8000001D16F030ED26F7EEC15F00101B66FAE
:10220800B651CEEC62F00101B74BB82B96D76405F6
:1022180002E1070E8C6E020E641901E051D10F0124
:10222800108B070E2D6F4CD1849284948EA88994BC
:1022380092EC63F02150221001E107D1BAC1B4F148
:10224800B90E0E6E010E0F6E3EEC5EF00101BA6F14
:10225800B9B9BA9F69511CE0350EBA1907E1340EB5
:1022680000019C6FF90E9D6FF0EC67F0370E0001CE
:102278009C6FFF0E9D6FBAC19EF09F6B0101010E0E
:10228800B9A9000E0001A06FA16BF0EC67F004D0B3
:102298006A0EE82EFED700D00101FB5109E10D0EB0
:1022A8000101B06F760EE82EFED7B02FFCD700F0F4
:1022B8000101B9A931D0600EBA192EE15F0EB41927
:1022C8002BE1510E00019C6FFF0E9D6FF0EC67F043
:1022D80002500209026EF20E9C6FFE0E9D6F67C1DE
:1022E8009EF09F6B66C1A0F0A16BF0EC67F02BEE3F
:1022F80035F067C1DFFF2BEE36F066C1DFFF838460
:10230800020EFBEC5DF08394029201016C6B8FEC82
:1023180067F00101BA6BD4D0FB5147E0B951100BFB
:102328000001ED6F000EEE6F0101BA51A5EC3EF011
:10233800EDC0BBF1EEC0BCF1080E0101BB19BC1128
:1023480001E100F0070E0101BB19BC1102E19EEC8E
:1023580061F0BB05BC1102E1B5EC5BF0020E0101B6
:10236800BB19BC1102E164EC3CF0030E0101BB197E
:10237800BC1104E12FEC22F00101B56F050EBB1969
:10238800BC1104E1B5EC40F00101B56F090EBB19B1
:10239800BC1102E127EC59F00A0E0101BB19BC116E
:1023A80001E08ED0E0EC54F08BD0B9C121F0226A64
:1023B800BA5146EC18F021C0BBF122C0BCF1070E9F
:1023C8000101BB19BC1102E13AEC61F0020EBB1924
:1023D800BC1102E126EC60F0BB05BC1102E1EEEC99
:1023E8001FF0030EBB19BC1102E19EEC57F0040E5E
:1023F800BB19BC1102E14FEC65F0050EBB19BC110D
:1024080002E158EC51F0060E0101BB19BC1102E1C2
:102418001DEC68F0080EBB19BC1102E1BFEC3FF0DF
:10242800090EBB19BC1102E1D4EC55F00A0E0101EA
:10243800BB19BC1102E19BEC64F00C0E0101BB1945
:10244800BC113EE1B4EC35F03BD041EC50F0010159
:10245800636F645135E0FA51631932E0838E000EE0
:102468000E6EC00E1FEC63F0F7EC66F0000E0E6EF9
:10247800C00E1FEC63F0E70E126EFE0E136E01EC39
:102488005FF063C1FAF1000E00016D6F030E6E6F0D
:1024980015EC65F0A6EC38F00101625102E04CEC55
:1024A80045F0070E00018A6FFC0E8B6FFAC18CF0A5
:1024B8008D6BB6EC67F0FB5103E0FA51AAEC67F0BC
:1024C8008FB22ED0050E0101B5192AE0ADD6580EEF
:1024D80000019C6FFE0E9D6F8FCF9EF09F6BF0ECFE
:1024E80067F0290E0101B16F960EB06F7F0EE82ECE
:1024F800FED7B02FFCD7B12FFAD70400000E0E6E0E
:10250800C00E1FEC63F0F7EC66F0000E0E6EC00E06
:102518001FEC63F0590E126EFF0E136E01EC5FF0A4
:102528008FB2D5D7090E0101B16F1E0EB06FE40E40
:10253800E82EFED7B02FFCD7B12FFAD700F083943E
:1025480083920001B16BB26B360EB36FF90EB46FA4
:10255800B56BDFEC5CF09CD59EC00FF09FC010F00F
:10256800BC0E116E82EC59F00001BE6FBE5108E13D
:1025780020EE0FF09E51D9269F51DA22DF50BE6F10
:10258800BE5102E0BE51120020EE0AF09E51D9263B
:102598009F51DA22A051DE5CA151DE58A251DE58CB
:1025A800A351DE5816E220EE0EF09E51D9269F5117
:1025B800DA22DFB20ED020EE0AF09E51D9269F51C2
:1025C800DA22DECFA0F0DECFA1F0DECFA2F0DECFA0
:1025D800A3F020EE10F09E51D9269F51DA22DECFCB
:1025E800B4F0DECFB5F0DECFB6F0DECFB7F0B86B23
:1025F800B96BBA6BBB6B20EE10F09E51D9269F5178
:10260800DA22B8C0DEFFB9C0DEFFBAC0DEFFBBC049
:10261800DEFFA051A111A211A31101E100D220EE09
:1026280009F0BC51D926BD51DA22DECFA4F0DDCFA6
:10263800A5F0A451A66FA551A76FA86BA96B090EA9
:10264800D890A637A737A837A937E82EF9D7A6C054
:10265800BFF0A7C0C0F0A8C0C1F0A9C0C2F0B45173
:10266800B511B611B71101E196D0FF0EA0250E6E77
:10267800FF0EA1210F6EFF0EA221106EFF0EA321E7
:10268800116EBFC012F0C0C013F0C1C014F0C2C0B8
:1026980015F03EEC5FF00EC0A4F00FC0A5F010C01E
:1026A800A6F011C0A7F0FF0E0001B4250E6EFF0EB4
:1026B800B5210F6EFF0EB621106EFF0EB721116EF9
:1026C800BFC012F0C0C013F0C1C014F0C2C015F0F2
:1026D8003EEC5FF00E500001A45D0F50A55910505C
:1026E800A6591150A75957E3FF0EBF25A46FFF0E37
:1026F800C021A56FFF0EC121A66FFF0EC221A76FD3
:10270800A41DA86FA51DA96FA61DAA6FA71DAB6F55
:10271800FF0EB425AC6FFF0EB521AD6FFF0EB621CD
:10272800AE6FFF0EB721AF6FA851AC15B06FA951AE
:10273800AD15B16FAA51AE15B26FAB51AF15B36FEE
:1027480020EE10F09E51D9269F51DA22B0C0DEFF4C
:10275800B1C0DEFFB2C0DEFFB3C0DEFF20EE10F076
:102768009E51D9269F51DA22DE50A05FDE50A15B30
:10277800DE50A25BDD50A35B20EE14F09E51D926FB
:102788009F51DA22DECFC3F0DECFC4F0DECFC5F032
:10279800DECFC6F060D020EE06F09E51D9269F51BC
:1027A800DA22DECFC3F0DECFC4F0DECFC5F0DECF55
:1027B800C6F0C351C411C511C6113FE19EC081F0D6
:1027C8009FC082F0836B846B856B866B8EEC2AF0DE
:1027D80081C0C3F082C0C4F083C0C5F084C0C6F015
:1027E800C305C411C511C61109E120EE0FF09E51B1
:1027F800D9269F51DA22020EDF6E020CC3290FE19F
:10280800C4290DE1C5290BE1C62909E120EE0FF025
:102818009E51D9269F51DA22010EDF6E010C20EE5F
:1028280006F09E51D9269F51DA22C3C0DEFFC4C0EC
:10283800DEFFC5C0DEFFC6C0DEFF20EE14F09E51ED
:10284800D9269F51DA22C3C0DEFFC4C0DEFFC5C04F
:10285800DEFFC6C0DEFFC351C411C511C61101E0B9
:1028680085D0DDD0BF51A05FC051A15BC151A25B33
:10287800C251A35B20EE10F09E51D9269F51DA2257
:10288800BF51DE26C051DE22C151DE22C251DE22F6
:1028980020EE0EF09E51D9269F51DA22DFA220D0D9
:1028A8009EC081F09FC082F0C3C083F0C4C084F092
:1028B800C5C085F0C6C086F08EEC2AF081C0C3F092
:1028C80082C0C4F083C0C5F084C0C6F0C351C4112F
:1028D800C511C6111BE1A06BA16BA26BA36B50D0F5
:1028E8009EC045F09FC046F0C3C047F0C4C048F042
:1028F800C5C049F0C6C04AF098EC30F045C0C3F0F6
:1029080046C0C4F047C0C5F048C0C6F00001C3299E
:1029180007E1C42905E1C52903E1C62901E176D704
:10292800C651C511C41104E1020EC35D01E25DD7B1
:1029380020EE13F0BC51D926BD51DA22DE50C35D1A
:10294800DE50C459DE50C559DE50C65901E34DD793
:1029580020EE14F09E51D9269F51DA22C3C0DEFF23
:10296800C4C0DEFFC5C0DEFFC6C0DEFFA051BF5D2C
:10297800A151C059A251C159A351C25901E272D7FC
:1029880020EE10F09E51D9269F51DA22A051DE2662
:10299800A151DE22A251DE22A351DE22A051A46F52
:1029A800010EA115A56FA66BA76BA411A611A711FF
:1029B80036E0BCC00EF0BDC00FF0C3C010F0C4C0FC
:1029C80011F0C5C012F0C6C013F0CEEC50F00EC026
:1029D800B8F00FC0B9F010C0BAF011C0BBF00001D8
:1029E800B851B911BA11BB1101E1FFD6A0C0A4F0CA
:1029F800A1C0A5F0A2C0A6F0A3C0A7F00A0E05D0FA
:102A0800D890A733A633A533A433E82EF9D7A45119
:102A1800B827A551B923A651BA23A751BB2320EE45
:102A280010F09E51D9269F51DA2210EE0AF09E51DD
:102A3800E1269F51E222DE50E65CDE50E658DE5089
:102A4800E658DE50E6581CE220EE10F09E51D926DA
:102A58009F51DA2210EE0AF09E51E1269F51E222A0
:102A6800DECFE6FFDECFE6FFDECFE6FFDECFE6FF16
:102A780020EE0EF09E51D9269F51DA22000EDB8CF3
:102A880020EE10F09E51D9269F51DA22FF0EDE1457
:102A9800A46F010EDE14A56F000EDE14A66F000EE3
:102AA800DE14A76FA451A511A611A71101E16AD5DB
:102AB80020EE18F09E51D9269F51DA22B851DE181F
:102AC8000AE1B951DE1807E1BA51DE1804E1BB5139
:102AD800DE1801E157D520EE18F09E51D9269F51F6
:102AE800DA22B8C0DEFFB9C0DEFFBAC0DEFFBBC065
:102AF800DEFF48D5CE51CF1101E1090C3F0ED217A8
:102B0800D00E7C6F810E7D6F010E7E6FD2C07FF07C
:102B1800ADEC00F00101836F835101E0A8D281C1BF
:102B280084F182C185F1840E0001C06F010EC16F6E
:102B3800D0C0C2F0D1C0C3F026EC46F00101836FCB
:102B4800835104E1ABAF02D0060E836FD2C0D3F03D
:102B58001C0E0001D31701E1D1D0010183510FE010
:102B6800040E831909E1840E0001C46F010EC56FBC
:102B78006DEC58F00101836F0001D2870DD088C138
:102B8800D3F0110E0001D31702E0070E03D0D2A52F
:102B980003D0080E0101836F0101835101E0BDD00C
:102BA8000001D2A7BAD081C115F082C116F09EC12A
:102BB80017F09FC118F0B3EC5FF015C071F116C0A3
:102BC80072F117C073F118C074F10E0E01019E2541
:102BD8000E6E000E9F210F6E106A116A210E126E82
:102BE800500E136E04EC61F0010120EE0BF09E51C3
:102BF800D9269F51DA22200EDF6E81C112F082C1E0
:102C080013F09EC114F09FC115F0166A176A186A6E
:102C1800196A7BEC64F01C0E01019E250E6E000EF5
:102C28009F210F6E106A116A126A136A04EC61F030
:102C3800010120EE03F08151D9268251DA22010EDA
:102C4800DF6E715172117311741167E020EE2BF071
:102C58008151D9268251DA22DECF75F1DECF76F1A5
:102C6800DECF77F1DECF78F1840E0001816F010E9F
:102C7800826F71C183F072C184F073C185F074C131
:102C880086F0876B886B896B8A6BF3EC46F00101E1
:102C9800836F835142E181C13AF082C13BF075C133
:102CA8003CF076C13DF077C13EF078C13FF01BECB7
:102CB8005BF00101836FFF0E71250001D36FFF0EDA
:102CC800010172210001D46FFF0E0101732100017F
:102CD800D56FFF0E010174210001D66F010120EEAE
:102CE8000BF08151D9268251DA22D3C0DEFFD4C03D
:102CF800DEFFD5C0DEFFD6C0DEFF0FD00101835155
:102D08000CE188A902D0040E07D00001D2A305D097
:102D1800010188A102D0070E836F0101835123E1CD
:102D28000001D2B7D28D010120EE2BF08151D926B6
:102D38008251DA22000110EE1CF0CE51E126CF516B
:102D4800E222DECFE6FFDECFE6FFDECFE6FFDECF14
:102D5800E6FF20EE20F0CE51D926CF51DA229EC1CF
:102D6800DEFF9FC1DDFF0101835101E080D181C1F8
:102D780015F082C116F09EC117F09FC118F0B3EC90
:102D88005FF0000120EE06F0CE51D926CF51DA22AD
:102D980015C0DEFF16C0DEFF17C0DEFF18C0DEFF5D
:102DA8001C0E01019E250E6E000E9F210F6ED8ECA1
:102DB80059F0000120EE0AF0CE51D926CF51DA227F
:102DC8000EC0DEFF0FC0DEFF10C0DEFF11C0DEFF49
:102DD800CEC0D9FFCFC0DAFF81C1DEFF82C1DDFFDF
:102DE800010120EE05F08151D9268251DA22000135
:102DF80010EE02F0CE51E126CF51E222DECFE6FFFF
:102E0800DDCFE5FF20EE0EF0CE51D926CF51DA22E4
:102E1800D2C0DFFF20EE0FF0CE51D926CF51DA22F3
:102E2800DF6A20EE18F0CE51D926CF51DA22DE6AB9
:102E3800DE6ADE6ADD6A20EE10F0CE51D926CF5167
:102E4800DA22DE6ADE6ADE6ADD6AD2AB10D120EEF3
:102E58000AF0CE51D926CF51DA22DE50DE10DE102C
:102E6800DE1001E104D120EE0AF0CE51D926CF516F
:102E7800DA2210EE10F0CE51E126CF51E222DECF59
:102E8800E6FFDECFE6FFDECFE6FFDECFE6FF01019D
:102E980020EE09F08151D9268251DA22DECFD3F013
:102EA800DDCFD4F00001D351D56FD451D66FD76B95
:102EB800D86B090ED890D537D637D737D837E82EFC
:102EC800F9D7D5C06DF1D6C06EF1D7C06FF1D8C0B3
:102ED80070F120EE06F0CE51D926CF51DA22DECF9E
:102EE8007DF1DECF7EF1DECF7FF1DECF80F120EE07
:102EF8000AF0CE51D926CF51DA22DECF79F1DECFD2
:102F08007AF1DECF7BF1DECF7CF132D0CEC045F056
:102F1800CFC046F07DC147F07EC148F07FC149F07F
:102F280080C14AF098EC30F045C07DF146C07EF192
:102F380047C07FF148C080F1010180517F117E11A7
:102F480005E1020E7D5D02E2020E836F7D2908E134
:102F58007E2906E17F2904E1802902E1010E836FC1
:102F68006D51795F6E517A5B6F517B5B70517C5B01
:102F78000101835109E179516D5D7A516E597B5197
:102F88006F597C517059C2E3000120EE14F0CE5104
:102F9800D926CF51DA227DC1DEFF7EC1DEFF7FC197
:102FA800DEFF80C1DEFF0101835161E1795100013B
:102FB800D36F010E01017A150001D46FD56BD66B62
:102FC800D311D511D61153E081C10EF082C10FF093
:102FD8007DC110F07EC111F07FC112F080C113F0E5
:102FE800CEEC50F00EC075F10FC076F110C077F13D
:102FF80011C078F10101755176117711781103E14B
:10300800020E836F34D079C1D3F07AC1D4F07BC17A
:10301800D5F07CC1D6F00A0E06D00001D890D63380
:10302800D533D433D333E82EF8D7010175510001D5
:10303800D325D76F010176510001D421D86F010142
:1030480077510001D521D96F010178510001D621AE
:10305800DA6F20EE18F0CE51D926CF51DA22D7C038
:10306800DEFFD8C0DEFFD9C0DEFFDAC0DEFF010117
:10307800835106E0CEC0D9FFCFC0DAFFDE6ADD6A31
:1030880083511200276E2150100B256E225002E04A
:10309800CBEC58F0266A255001E120D2279E040E79
:1030A800271802E1505003E1140E271807E1010127
:1030B800486B496B226A070E216E070C3F0E2718D2
:1030C80007E1506A0101486B496B216A226A1200C4
:1030D8005F0E271807E101015C6B486B496B216A99
:1030E800226A12003F0E27640BD05F0E276008D0BB
:1030F800400E271805E001015C6B216A226A120064
:10310800400E27180AE1010E01015C6F506A0101A7
:10311800486B496B216A226A1200200E271801E0C9
:10312800DDD1010E506EF3D7600E27180CE10101B6
:103138005C5109E05A51080ED8B4030E266E0101FD
:10314800486B496B33D2600E271809E1505007E0ED
:1031580001015A5102E0090EF1D7050EEFD7680EAA
:10316800271809E1505007E01A0E0101496F900E27
:103178005FD183801BD2680E271805E101015C51DD
:1031880002E0020EDBD76A0E271807E1505005E06F
:103198001A0E0101496FF40E4BD16C0E271807E186
:1031A800505005E01A0E0101496F2C0E41D1700EE6
:1031B800271808E101015C5105E0040E266E486BF2
:1031C800496BD7D7700E271801E0F0D1505001E1B4
:1031D800EDD11B0E0101496F620E2AD18380275061
:1031E8000CE121AA05D0266A0101486B496B83903E
:1031F8001A0E0101496FAF0E486F020E271805E13C
:103208001A0E0101496F920E486F050E271805E145
:103218001A0E0101496FAE0E486F070E271805E117
:103228001A0E0101496FB80E486F080E271805E1FC
:103238001A0E0101496FCC0E486F030E271802E0E1
:1032480027280CE18380680E236EE40EE82EFED753
:10325800232EFCD700D0266A839071D7140E271826
:1032680005E11A0E0101496F9E0E486F160E2718C8
:1032780001E09CD11A0E0101496FA40ECAD0050EB7
:10328800271805E11A0E0101496FF50E486F080E5F
:10329800271801E08BD11A0E0101496FCC0E486F37
:1032A800010E5A6F83D127C053F01A0E0101496FDE
:1032B800950EAFD02750246E236A53500C0D000E84
:1032C800F324D96E010EF420DA6E23C0DEFF24C089
:1032D800DDFF1A0E0101496F960E9BD02750236E11
:1032E800246A53500C0D000EF324D96E010EF420FD
:1032F800DA6E23C0DEFF24C0DDFF1A0E0101496F1C
:10330800970E87D053500C0D020EF324D96E010E80
:10331800F420DA6E27C0DFFF1A0E0101496F980EFC
:1033280078D053500C0D030EF324D96E010EF420FF
:10333800DA6E27C0DFFF0101486B496B010E37D0F9
:103348001A0E0101496FB90E73D01A0E0101496FA7
:10335800BA0E5FD01A0E0101496FBB0E486F240EDA
:1033680000019C6FFE0E9D6FF0EC67F001015B6B36
:10337800486B496B55D00101486B496B240E00011D
:103388009C6FFE0E9D6FF0EC67F04AD0FD0E0001B9
:103398009C6FFE0E9D6FF0EC67F00101486B496B66
:1033A800010E586F3DD00101486B496B060E266E21
:1033B800FDD027C053F00101486B496B266A30D015
:1033C80001015A6B1A0E496FF70E486F29D01A0E71
:1033D8000101496FF70E1DD08390270E0101496F37
:1033E8000F0E17D0180E271801E0E0D01A0E0101B1
:1033F800496F2D0E0ED01A0E0101496F2E0E09D0FD
:103408001A0E0101496F2F0E04D01A0E0101496FDF
:10341800300E486FCBD00101486B496B0A0E266EFF
:103428008390C4D0040E266E270E0101496F0F0E3B
:10343800486F9FD68380010104D08390010E01015B
:103448005A6F486B496B266AB1D08390010E01010F
:103458005A6F486B496B266A53500C0D000EF324C3
:10346800D96E010EF420DA6EDE6ADD6A53500C0D57
:10347800020EF324D96E010EF420DA6E2744E846D2
:10348800030BDF6E53500C0D030EF324D96E010E9F
:10349800F420DA6E27503F0BDF6E8D0E00019C6F13
:1034A800FC0E9D6F27C09EF09F6B53500C0D020EB3
:1034B800F324D96E010EF420DA6EDF50A06FA16BF1
:1034C80053500C0D030EF324D96E010EF420DA6E5E
:1034D800DF50A26FA36BF0EC67F068D048C123F00F
:1034E80049C124F0245007E01A0A09E0010A54E00F
:1034F8003C0A5AE05BD0235001E116D657D023503E
:103508002C0A01E16FD7010A01E175D7030A01E12D
:1035180077D7010A01E179D71F0A01E17CD7A00A10
:1035280001E15CD6020A01E1BED6070A01E1C2D672
:10353800030A01E1D3D6010A01E1E4D60F0A01E149
:10354800F0D6060A01E122D73A0A01E12CD70A0A85
:1035580001E173D7010A01E178D7170A01E1F0D632
:10356800010A01E1F2D6030A01E1F4D6010A01E1F8
:1035780002D7790A01E105D60E0A01E11AD7380AFD
:1035880001E17DD6010A01E11BD7030A01E11FD73A
:10359800010A01E121D70AD02350580A01E142D794
:1035A8003A0A01E147D702D023500F0A26C021F07A
:1035B800226A1200730EF66EF80EF76E0900F5CF48
:1035C800E5F00A00F5CFE6F00001E96BEC6B0101CC
:1035D800F06B030ECF6105D09650CF19F00BCF19C1
:1035E80005D0CFC193FF9650F00B0A09966ECD6AAD
:1035F800CE6A0FD1ED6B350E176E0B0E186EE50EF9
:10360800196E4BEC5CF017C0EAF018C0EBF0EAC09A
:10361800D9FFEBC0DAFF3B0EDE1801E0F5D0F9D098
:10362800ED5113E1EAC012F0EBC013F05EEC60F06C
:103638000001EC6F800EEC6503D0EC51800FE96F50
:10364800030EE965D5D0E96BD3D0ED0511E1010191
:10365800FA510001EC1903E07F0EEC1909E1EAC008
:1036680012F0EBC013F05EEC60F00101676FC0D0A0
:10367800020EED1911E10101FA510001EC1903E004
:103688007F0EEC1909E1EAC012F0EBC013F05EEC12
:1036980060F00101666FACD0020EED652CD0080E0B
:1036A800ED6129D00101FA510001EC190CE07F0EFF
:1036B800EC1909E0810EEC1906E0820EEC1903E022
:1036C800830EEC1918E1E951050DD10EF324E76FCB
:1036D800010EF420E86FEAC012F0EBC013F05EECC4
:1036E80060F00001C26FED51E725C36F000EE821BD
:1036F800C46FFD0E5DD0070EED652CD01B0EED617D
:1037080029D00101FA510001EC190CE07F0EEC19E7
:1037180009E0810EEC1906E0820EEC1903E0830E35
:10372800EC1918E1E951130DAA0EF324E76F030E03
:10373800F420E86FEAC012F0EBC013F05EEC60F022
:103748000001C26FED51E725C36F000EE821C46F79
:10375800F80E2ED01A0EED6533D0280EED6130D05C
:103768000101FA510001EC190CE07F0EEC1909E097
:10377800810EEC1906E0820EEC1903E0830EEC19B9
:103788001FE1E9510D0D980EF324E76F020EF420A6
:10379800E86FEAC012F0EBC013F05EEC60F00001D5
:1037A800C26FED51E725C36F000EE821C46FE50E27
:1037B800C325D96EFF0EC421DA6EC2C0DFFF18D050
:1037C800280EED1915E10101FA510001EC1903E089
:1037D8007F0EEC190DE1F00E0E6E010E0F6EEAC0B1
:1037E80010F0EBC011F0136A080E126EFDEC61F0D8
:1037F8000001ED2B176A186AE50E196E4BEC5CF0A8
:1038080017C0EAF018C0EBF00001EA51EB1101E033
:1038180007D7350E00019F6F0B0EA06FA26B910E9C
:10382800A16F000EA36F030EA46F95EC5CF09F517F
:10383800A01101E0DFD6ED6BED510D0DA20EF324C2
:10384800D96E020EF420DA6EDF50C26FC2C0C3F028
:10385800C46BC56BC66BC5C0C6F0C4C0C5F0C3C0D9
:10386800C4F0C36BED510D0DA10EF324D96E020EF9
:10387800F420DA6EDF50C76FC7C0C8F0C96BCA6BD7
:10388800CB6BC9C0CBF0C8C0CAF0C96BC86BED51CF
:103898000D0DA00EF324D96E020EF420DA6EDF505F
:1038A800CC6FCCC0CDF0CE6BCF6BD06BCDC0D0F091
:1038B800CF6BCE6BCD6BC851CD25D16FC951CE2101
:1038C800D26FCA51CF21D36FCB51D021D46FC351FE
:1038D800D125D56FC451D221D66FC551D321D76F09
:1038E800C651D421D86FED510D0DA30EF324D96E16
:1038F800020EF420DA6EDF50D525D96F000ED621DE
:10390800DA6F000ED721DB6F000ED821DC6FD9C02B
:10391800DDF0DAC0DEF0DBC0DFF0DCC0E0F0E16B48
:10392800E0BFE169E1C0E2F0E1C0E3F0E1C0E4F04A
:10393800ED511E0D0F0EF324D96E020EF420DA6E2F
:10394800DDC0DEFFDEC0DEFFDFC0DEFFE0C0DEFF81
:10395800E1C0DEFFE2C0DEFFE3C0DEFFE4C0DEFF61
:10396800ED51130DAE0EF324D96E030EF420DA6E6A
:10397800DF50C36FC26BED51130DAF0EF324D96E38
:10398800030EF420DA6EDF50C46FC56BC251C42732
:10399800C351C523ED511E0D1C0EF324D96E020E22
:1039A800F420DA6EC4C0DEFFC5C0DDFFED511E0D88
:1039B8001C0EF324D96E020EF420DA6EDECFC2F0AC
:1039C800DDCFC3F0C2C00EF0C3C00FF0106A116A99
:1039D800126A136A146A156AED511E0D0F0EF3244C
:1039E800D96E020EF420DA6EDECFC4F0DECFC5F059
:1039F800DECFC6F0DECFC7F0DECFC8F0DECFC9F02D
:103A0800DECFCAF0DECFCBF0C4C016F0C5C017F0C9
:103A1800C6C018F0C7C019F0C8C01AF0C9C01BF05A
:103A2800CAC01CF0CBC01DF0B5EC5DF00EC0CCF0E8
:103A38000FC0CDF010C0CEF011C0CFF012C0D0F042
:103A480013C0D1F014C0D2F015C0D3F00001ED516D
:103A58001E0D0F0EF324D96E020EF420DA6ECCC0C0
:103A6800DEFFCDC0DEFFCEC0DEFFCFC0DEFFD0C0A0
:103A7800DEFFD1C0DEFFD2C0DEFFD3C0DEFF4C0EBA
:103A88009C6FFA0E9D6FEDC09EF09F6BED511E0D61
:103A98001C0EF324D96E020EF420DA6EDECFA0F0ED
:103AA800DDCFA1F0F0EC67F0ED2B030EED65C4D689
:103AB800D30E9C6FFA0E9D6FF00E9E6F010E9F6FD6
:103AC800F0EF67F076C091F077C092F07AC0D9FF36
:103AD8007BC0DAFFDE6ADD6A74C00FF075C010F0D3
:103AE8009D0E116E82EC59F000018C6F8C510AE129
:103AF80020EE0FF07451D9267551DA22DF508C6F01
:103B08008C5102E08C51120020EE0EF07451D9262F
:103B18007551DA22DFA0070C20EE10F07451D92677
:103B28007551DA22DECF7CF0DECF7DF0DECF7EF07D
:103B3800DECF7FF020EE0AF07451D9267551DA22D3
:103B4800DECF80F0DECF81F0DECF82F0DECF83F0F3
:103B58007C51805D886F7D518159896F7E51825972
:103B68008A6F7F5183598B6F78517C6F79517D6F44
:103B78007E6B7F6B7C51885D7D5189597E518A5956
:103B88007F518B5901E321D288C078F089C079F040
:103B98001CD220EE10F07451D9267551DA22FF0E8E
:103BA800DE147C6F010EDE147D6F000EDE147E6F56
:103BB800000EDE147F6F7C517D117E117F1101E0B4
:103BC80083D120EE10F07451D9267551DA22DECF58
:103BD8007CF0DECF7DF0DECF7EF0DECF7FF00A0E08
:103BE80005D0D8907F337E337D337C33E82EF9D7E8
:103BF8008069816920EE09F09D51D9269E51DA220B
:103C0800DECF82F0DDCF83F080518227815183237C
:103C18007C518215936F7D518315946F931166E1E2
:103C280020EE10F07451D9267551DA22DE50DE10DC
:103C3800DE10DE100FE120EE06F07451D926755122
:103C4800DA22DECF8DF0DECF8EF0DECF8FF0DECF42
:103C580090F01CD074C045F075C046F020EE14F00A
:103C68007451D9267551DA22DECF47F0DECF48F0FD
:103C7800DECF49F0DECF4AF098EC30F045C08DF049
:103C880046C08EF047C08FF048C090F000019051B8
:103C98008F118E110CE1020E8D5D09E220EE0FF0FE
:103CA8007451D9267551DA22020EDF6E020C8D2965
:103CB8000FE18E290DE18F290BE1902909E120EE12
:103CC8000FF07451D9267551DA22010EDF6E010CFE
:103CD80020EE14F07451D9267551DA228DC0DEFF1A
:103CE8008EC0DEFF8FC0DEFF90C0DEFF9DC00EF0ED
:103CF8009EC00FF020EE14F07451D9267551DA22C7
:103D0800DECF10F0DECF11F0DECF12F0DECF13F0F1
:103D1800CEEC50F00EC095F00FC096F010C097F0A2
:103D280011C098F00001955196119711981101E171
:103D3800B5D79351952794519623000E972398232E
:103D480078C07CF079C07DF0090E7E6FD8907D3305
:103D58007C337E2FFBD77CC099F07DC09AF09951B7
:103D68009A1101E1A3D0995193257C6F9A5194211E
:103D78007D6F20EE09F09D51D9269E51DA227C51A3
:103D8800DE5C7D51DE5810E220EE09F09D51D92607
:103D98009E51DA22DECF7CF0DDCF7DF093517C5D41
:103DA800996F94517D599A6F91C01DF092C01EF081
:103DB80095C01FF096C020F097C021F098C022F05F
:103DC80099C023F09AC024F020EE01F09D51D92625
:103DD8009E51DA22DF502CEC5AF0000901E0ACD0F9
:103DE800000120EE03F09D51D9269E51DA22DF50C2
:103DF8004EE099517C6F9A517D6F7E6B7F6B20EE00
:103E08002BF09D51D9269E51DA22DECF80F0DECFED
:103E180081F0DECF82F0DECF83F09551805D846F34
:103E280096518159856F97518259866F9851835958
:103E3800876F7C51845D7D5185597E5186597F51AC
:103E4800875925E220EE2BF09D51D9269E51DA2282
:103E5800DECF7CF0DDCF7DF095517C5F96517D5BA8
:103E6800090ED8907C377D37E82EFBD77C519125F9
:103E78000E6E7D5192210F6E2F0E9D25106E000E35
:103E88009E21116E020E136E126A1AEC64F099C02C
:103E98007CF09AC07DF0090ED8907C377D37E82EEB
:103EA800FBD77CC09BF07DC09CF072D020EE18F050
:103EB8007451D9267551DA2295C0DEFF96C0DEFF0F
:103EC80097C0DEFF98C0DEFF7C69010E7D6F20EE93
:103ED80010F07451D9267551DA22DECF7EF0DDCF8D
:103EE8007FF07C517E177D517F177E5100089B6FB4
:103EF8007F51D8A0E82A02089C6F9B51785D9C519D
:103F0800795904E278C09BF079C09CF09DC03AF0E2
:103F18009EC03BF020EE18F07451D9267551DA2274
:103F2800DECF3CF0DECF3DF0DECF3EF0DECF3FF01F
:103F38001BEC5BF0000902E00001C1D691C00EF055
:103F480092C00FF000017C69010E7D6F20EE10F029
:103F58007451D9267551DA22DECF7EF0DDCF7FF09D
:103F68007C517E177D517F179DC080F09EC081F0E7
:103F78007E5180277F5181232F0E8025106E000EE1
:103F88008121116E9BC012F09CC013F01AEC64F0F2
:103F98009B51785F9C51795B7AC0D9FF7BC0DAFF6F
:103FA8009B51DE269C51DD229B5191279C519223E7
:103FB80020EE10F07451D9267551DA229B51DE2675
:103FC8009C51DE22000EDE22DE227851791101E0BA
:103FD800E0D5000C53500C0D000EF324D96E010EE1
:103FE800F420DA6E0001C969CA6953500C0D080E35
:103FF800F324E16E010EF420E26EE6CFCBF0E5CFBC
:10400800CCF0C951CB27CA51CC23DE50CB5DCC5163
:10401800800ACD6FDE50800ACD594AE353500C0D0B
:10402800020EF324D96E010EF420DA6EDF50C76F4A
:10403800C86BC969CA6953500C0D0A0EF324D96EAE
:10404800010EF420DA6EDF50CB6FCC6BC951CB2751
:10405800CA51CC23C751CB5DCC51800ACD6FC85112
:10406800800ACD5925E353500C0D030EF324D96E65
:10407800010EF420DA6EDF50C76FC86BC969CA69D0
:1040880053500C0D0B0EF324D96E010EF420DA6E8A
:10409800DF50CB6FCC6BC951CB27CA51CC23C7514A
:1040A800CB5DCC51800ACD6FC851800ACD5961E2F1
:1040B8001F0E0101596F010E5B6F83905D0E0001A9
:1040C8009C6FF90E9D6F53500C0D000EF324D96EA2
:1040D800010EF420DA6EDECF9EF0DDCF9FF0535054
:1040E8000C0D080EF324D96E010EF420DA6EDECF23
:1040F800C7F0DDCFC8F0FF0EC725A06FFF0EC8219F
:10410800A16F53500C0D020EF324D96E010EF4204A
:10411800DA6EDF50A26FA36B53500C0D0A0EF32416
:10412800D96E010EF420DA6EDF50C96FFF0EC92573
:10413800A46FA56BFF0EA52353500C0D030EF3249B
:10414800D96E010EF420DA6EDF50A66FA76B5350BC
:104158000C0D0B0EF324D96E010EF420DA6EDF502D
:10416800CA6FFF0ECA25A86FA96BFF0EA923F0EC32
:1041780067F053500C0D030EF324D96E010EF42092
:10418800DA6EDF50C76FC7C0C8F0C96BCA6BCB6B9C
:10419800CAC0CBF0C9C0CAF0C8C0C9F0C86B535078
:1041A8000C0D0B0EF324D96E010EF420DA6EDF50DD
:1041B800CC6FCCC0CDF0CE6BCF6BD06B53500C0D09
:1041C800020EF324D96E010EF420DA6EDF50D16F9F
:1041D800D1C0D2F0D36BD46BD56BD4C0D5F0D3C0DB
:1041E800D4F0D2C0D3F0D26BD251CD03F3CFD6F0F6
:1041F800F4CFD7F0D86BD96BCE03F350D727F45050
:10420800D823000ED923D351CD03F350D727F45028
:10421800D823000ED923D251CF03F350D827F45016
:10422800D923D351CE03F350D827F450D923D451EE
:10423800CD03F350D827F450D923D051D203F350EB
:10424800D927D351CF03F350D927D451CE03F350F4
:10425800D927D551CD03F350D92753500C0D0A0E49
:10426800F324D96E010EF420DA6EDF50DA6FDAC06B
:10427800DBF0DC6BDD6BDE6B53500C0D0B0EF324A7
:10428800D96E010EF420DA6EDF50DF6FDFC0E0F088
:10429800E16BE26BE36B53500C0D000EF324D96E07
:1042A800010EF420DA6EDECFE4F0DDCFE5F0E4C0F5
:1042B800E6F0E5C0E7F0000EE7BFFF0EE86FE96F34
:1042C800E651E003F3CFEAF0F4CFEBF0EC6BED6BE3
:1042D800E103F350EB27F450EC23000EED23E751F4
:1042E800E003F350EB27F450EC23000EED23E651E6
:1042F800E203F350EC27F450ED23E751E103F350C8
:10430800EC27F450ED23E851E003F350EC27F45088
:10431800ED23E351E603F350ED27E751E203F350B1
:10432800ED27E851E103F350ED27E951E003F3509D
:10433800ED27ECC0EDF0EBC0ECF0EAC0EBF0EA6B77
:10434800EA51DB03F3CFEEF0F4CFEFF0F06BF16B53
:10435800DC03F350EF27F450F023000EF123EB5168
:10436800DB03F350EF27F450F023000EF123EA515A
:10437800DD03F350F027F450F123EB51DC03F35045
:10438800F027F450F123EC51DB03F350F027F450FD
:10439800F123DE51EA03F350F127EB51DD03F3502B
:1043A800F127EC51DC03F350F127ED51DB03F35017
:1043B800F127D651EE25F26FD751EF21F36FD8517F
:1043C800F021F46FD951F121F56FC851F225F76F3B
:1043D800C951F321F86FCA51F421F96FCB51F52176
:1043E800FA6F5350220D000EF3249E6F030EF42033
:1043F8009F6FF7C0A0F0F8C0A1F0F9C0A2F0FAC012
:10440800A3F0B0EC12F0F66FF65111E01F0E9C6F9E
:10441800FB0E9D6FF7C09EF0F8C09FF0F9C0A0F0AA
:10442800FAC0A1F0F6C0A2F0A36BF0EC67F053500D
:104438000C0D040EF324D96E010EF420DA6EF7C0C9
:10444800DEFFF8C0DEFFF9C0DEFFFAC0DEFF0101C3
:104458005B6B83901200838E8380A5EC41F0FA6F2A
:10446800FA5118E053501E0D1B0EF324D96E020E9C
:10447800F420DA6E53501E0D1B0EF324E16E020E6B
:10448800F420E26EE7500409DF6E8AEC66F0000162
:10449800FA511200010162514EE0385139113A11B6
:1044A8003B1149E0535047E153501E0D070EF324CA
:1044B800D96E020EF420DA6E38C176F139C177F17F
:1044C8003AC178F1756B000E7525796F010E76216A
:1044D8007A6F000E77217B6F000E78217C6F7D6BE1
:1044E8007E6B7F6B806BDE50791925E1DE507A197F
:1044F80022E1DE507B191FE1DE507C191CE1DE5001
:104508007D1919E1DE507E1916E1DE507F1913E19D
:10451800DE50801910E1350E2B6E0B0E2C6E625199
:104528005BEC55F00292000EFBEC5DF00292516AD2
:1045380083905150120053501E0D170EF324D96E5C
:10454800020EF420DA6EDE50DE10DE1002E1DE0428
:1045580010E053501E0D170EF324D96E020EF420EE
:10456800DA6EDE280DE1DE280BE1DE2809E1DE281F
:1045780007E10001F069F169F269F369FB6B2ED07C
:1045880053501E0D170EF324D96E020EF420DA6E66
:10459800DECF6DF1DECF6EF1DECF6FF1DECF70F1E1
:1045A8006EC16DF16FC16EF170C16FF1706B6DC14D
:1045B800F0F06EC1F1F06FC1F2F070C1F3F053503A
:1045C8001E0D170EF324D96E020EF420DA6EDECF1C
:1045D8006DF1DDCF6EF16D510001FB6FFC6B029246
:1045E800F66BF76BF86BF96BF46BF56BCED08EA8A6
:1045F8008EAA0AD0C60E00019C6FFE0E9D6FF0ECCD
:1046080067F0BCD08394BCD0F4C06DF1F5C06EF1F6
:10461800000E6EBFFF0E6F6F706FFF0E0001F0256A
:104628000101716FFF0E0001F1210101726FFF0E90
:104638000001F2210101736FFF0E0001F321010156
:10464800746F6D51711910E16E5172190DE16F514E
:1046580073190AE17051741907E10001FB51FC114B
:1046680003E102500209026E5350220D000EF3249A
:104678000001746F030EF420756F350E766F0B0E04
:10468800776F010E796F786BFD0E7A6F7B6B66EC36
:104698001DF0FF6FFF5101E0E5D6FD51FE1101E16C
:1046A800E1D6D00E01016D6FC90EE82EFED76D2F31
:1046B800FCD700D08EA88EAA08D0D10E00019C6F1E
:1046C800FE0E9D6FF0EC67F059D00001FD51FBEC38
:1046D8005DF00001FD51F627FE51F723000EF82387
:1046E800F92353501E0D070EF324D96E020EF42041
:1046F800DA6E000EDE2401016D6F010EDE206E6F92
:10470800000EDE206F6F000EDE20706F000EDE20C0
:10471800716F000EDE20726F000EDE20736F000EC8
:10472800DE20746F53501E0D070EF324D96E020E4F
:10473800F420DA6E6DC1DEFF6EC1DEFF6FC1DEFFF1
:1047480070C1DEFF71C1DEFF72C1DEFF73C1DEFF23
:1047580074C1DEFF8EA88EAA08D0DC0E00019C6F03
:10476800FE0E9D6FF0EC67F009D08EBC0BD0110ED9
:1047780000019C6FFF0E9D6FF0EC67F0516A42D705
:10478800839086D00001F44BF52BF4C06DF1F5C091
:104798006EF1000E01016EBFFF0E6F6F706F0001AA
:1047A800F05101016D5D0001F15101016E590001E7
:1047B800F25101016F590001F3510101705901E2F1
:1047C80016D70001FB51FC1160E05350220D000E7A
:1047D800F324746F030EF420756F350E766F0B0E8D
:1047E800776FFBC078F0FCC079F0FD0E7A6F7B6BB9
:1047F80066EC1DF0FF6FFF5101E034D6025002094C
:10480800026EFB51FBEC5DF00001FD51F627FE51F5
:10481800F723000EF823F92353501E0D070EF32437
:10482800D96E020EF420DA6E000EDE2401016D6FDF
:10483800010EDE206E6F000EDE206F6F000EDE2090
:10484800706F000EDE20716F000EDE20726F000E9A
:10485800DE20736F000EDE20746F53501E0D070E9E
:10486800F324D96E020EF420DA6E6DC1DEFF6EC13C
:10487800DEFF6FC1DEFF70C1DEFF71C1DEFF72C1F6
:10488800DEFF73C1DEFF74C1DEFF0292516A78D782
:10489800839E4FD6020E806F65516411631104E147
:1048A800020E625D01E211D220EE13F06051D926AA
:1048B8006151DA22DE50625DDE506359DE50645980
:1048C800DE50655901E2EED100D262C07EF063C0CD
:1048D8007FF0D8907F316B6F7E316A6F6A517E2787
:1048E8006B517F2360C03AF061C03BF020EE1FF0AF
:1048F8006051D9266151DA22DECF6AF0DECF6BF043
:10490800DECF6CF0DECF6DF07EC06EF07FC06FF052
:10491800090E706FD8906F336E33702FFBD76E51BE
:104928006A253C6E6F516B213D6E000E6C213E6E08
:10493800000E6D213F6E1BEC5BF00001806F805113
:1049480001E0C3D16A69010E6B6F7EC06CF07FC055
:104958006DF06A516C176B516D1760C06EF061C0D5
:104968006FF06C516E276D516F232F0E6E257C6F83
:10497800000E6F217D6F7E4B7F2B62B104D066C025
:1049880078F0796B1AD066516A6F6B6B6A3B6B3B38
:10499800F00E6B176A510F0B6B13F00E6A177CC081
:1049A800D9FF7DC0DAFFDF500F0B6C6F6D6B6A515A
:1049B8006C11786F6B516D11796F7CC0D9FF7DC018
:1049C800DAFF78C0DFFF20EE03F06051D92661518D
:1049D800DA22010EDF6E60C03AF061C03BF020EED3
:1049E8001FF06051D9266151DA22DECF6AF0DECF9E
:1049F8006BF0DECF6CF0DECF6DF07EC06EF07FC066
:104A08006FF0090E706FD8906F336E33702FFBD72D
:104A18006E516A253C6E6F516B213D6E000E6C2104
:104A28003E6E000E6D213F6E1BEC5BF00001806F47
:104A3800805101E04AD16A69010E6B6F7EC06CF04B
:104A48007FC06DF06A516C176B516D1760C06EF0C6
:104A580061C06FF06C516E276D516F232F0E6E255C
:104A68007C6F000E6F217D6F62B10CD067C06AF059
:104A78000F0E6A177CC0D9FF7DC0DAFFDF50F00B3C
:104A88006A1112D066C06AF067C06BF068C06CF03B
:104A980069C06DF0050E05D0D8906D336C336B335B
:104AA8006A33E82EF9D76A517A6F7B6B7CC0D9FFDD
:104AB8007DC0DAFF7AC0DFFF4FD060C03AF061C036
:104AC8003BF020EE1FF06051D9266151DA22DECF8B
:104AD8006AF0DECF6BF0DECF6CF0DECF6DF06351A5
:104AE8006E6F64516F6F6551706F716B6A516E258F
:104AF8003C6E6B516F213D6E6C5170213E6E6D5155
:104B080071213F6E1BEC5BF00001806F805101E06A
:104B1800DCD06A69010E6B6F62C06CF063C06DF027
:104B2800D8906C376D376A516C176B516D1760C030
:104B38006EF061C06FF06C516E276D516F232F0EB0
:104B48006E250E6E000E6F210F6E66C010F067C0E6
:104B580011F020EC67F0A4D020EE03F06051D926C4
:104B68006151DA22010EDF6EB0D060C03AF061C048
:104B78003BF020EE1FF06051D9266151DA22DECFDA
:104B88006AF0DECF6BF0DECF6CF0DECF6DF062C086
:104B98006EF063C06FF064C070F065C071F0080E0D
:104BA80005D0D890713370336F336E33E82EF9D750
:104BB8006A516E253C6E6B516F213D6E6C517021B0
:104BC8003E6E6D5171213F6E1BEC5BF00001806FF2
:104BD80080517BE16A69010E6B6F62C06CF063C043
:104BE8006DF0D8906C376D37D8906C376D376A5147
:104BF8006C176B516D1760C06EF061C06FF06C512F
:104C08006E276D516F232F0E6E250E6E000E6F21CD
:104C18000F6ED8EC59F00001706B716B726BF00E6F
:104C28001114736F6651746F6751756F6851766FA1
:104C38000F0E6915776F70517411666F7151751188
:104C4800676F72517611686F73517711696F6A696E
:104C5800010E6B6F62C06CF063C06DF0D8906C375A
:104C68006D37D8906C376D376A516C176B516D176B
:104C780060C06EF061C06FF06C516E276D516F238C
:104C88002F0E6E250E6E000E6F210F6E66C010F08F
:104C980067C011F068C012F069C013F004EC61F04D
:104CA80000015AD760C0D9FF61C0DAFFDF506A6FD0
:104CB8006B6B6B510AE16A51010A01E106D6030ADE
:104CC80001E1FBD6010A01E150D7805112002D6E97
:104CD8001EC044F01FC045F02D5001E0040C010E29
:104CE800426E55B0030CE9D1C2EC67F0000901E14E
:104CF800FDD1426AFBD1176A186A196A1A6A090E45
:104D080087EC65F0000901E0F1D12E0E0E6E0F6AF6
:104D1800116A100E106ECEEC61F0000901E1E6D1C7
:104D28002E44E846030BE8064DE135C020F03F0E5F
:104D3800201620C021F0226A236A246A22C024F0A7
:104D480021C023F0226A216A3650266E256A375020
:104D5800276E286A255027262650282227502124E6
:104D6800296E285022202A6E000E23202B6E000E5A
:104D780024202C6E29283E6E000E2A203F6E000E3D
:104D88002B20406E000E2C20416E3EC020F03FC00C
:104D980021F040C022F041C023F00A0ED8902036FE
:104DA800213622362336E82EF9D71EC0D9FF1FC078
:104DB800DAFF20C0DEFF21C0DEFF22C0DEFF23C0F5
:104DC800DEFF97D7206A38AE01D0202A010E2016C0
:104DD80033C021F00F0E21163750030B020DF3508C
:104DE80021242024020F436E3450030B206E216AC5
:104DF8000A0ED89020362136E82EFBD73550226E81
:104E0800236AD89022362336D89022362336364461
:104E1800E846030B246E256A2250242623502522B7
:104E28002050242621502522242A000E252224C081
:104E38003EF025C03FF0406A416A43C020F0F70EBB
:104E480020263EC021F03FC022F040C023F041C0E0
:104E580024F0202A05D0D89021362236233624364D
:104E6800202EF9D734D054A43FD0176A186A196A8B
:104E78001A6A8D0E87EC65F0000901E037D10CEC59
:104E880068F02E0E0E6E0F6A116A100E106ECEECC0
:104E980061F0000901E12AD1300E436E03D00CEC19
:104EA80068F043064350FBE138C020F0203A0F0E6B
:104EB8002016100E216E226A236A246A202A05D041
:104EC800D8902136223623362436202EF9D71EC014
:104ED800D9FF1FC0DAFF21C0DEFF22C0DEFF23C0DA
:104EE800DEFF24C0DEFF05D7176A186A196A1A6A36
:104EF800090E87EC65F0000901E0F8D02E0E0E6E61
:104F08000F6A116A100E106ECEEC61F0000901E113
:104F1800EDD054A232D03BC020F0060E216ED890BE
:104F28002032212EFCD7FF0E202638503F0B226E50
:104F3800236AD890223623363944010B2226000EE4
:104F48002322222A2322202A03D0D890223623364D
:104F5800202EFBD72250246E2350256E266A276AFE
:104F68001EC0D9FF1FC0DAFF24C0DEFF25C0DEFF48
:104F780026C0DEFF27C0DEFFBCD63950030B206EEB
:104F8800216AD89020362136D89020362136D890FC
:104F9800203621363938E842070B2026000E212218
:104FA800202A21223840E8423F0B1F0B226E236A39
:104FB800222A000E232220502202F3CF24F0F4CF1D
:104FC80025F02302F350252621502202F3502526EE
:104FD8002450266E2550276E286A296A1EC0D9FFDC
:104FE8001FC0DAFF26C0DEFF27C0DEFF28C0DEFFB5
:104FF80029C0DEFF7ED644C0D9FF45C0DAFF54C0C1
:10500800DFFF77D6176A186A196A1A6A090E87ECD9
:1050180065F000096BE144C00EF045C00FF0116A5D
:10502800100E106ECEEC61F0000901E062D65ED081
:10503800176A186A196A1A6A0A0E87EC65F0000975
:1050480055E144C00EF045C00FF0116A100E106E05
:10505800CEEC61F0E9D7176A186A196A1A6A3A0E2B
:1050680087EC65F0000942E1040E436E0AD00CECAF
:1050780068F044C0D9FF45C0DAFFDF6E444A452ACC
:105088004306435001E135D6F2D7176A186A196A00
:105098001A6A8D0E87EC65F0000928E10CEC68F0BF
:1050A80044C00EF045C00FF0116A400E106ECEECF1
:1050B80061F0BAD7040E426E19D01D50206E216AD5
:1050C8002150F8E1205001E10FD6010A01E113D681
:1050D800020A01E1C8D6090A8EE0010A93E0070A2C
:1050E800A7E0010AB8E0030AD0E0E4D719EC68F0B9
:1050F800425012001BC0F6FF1CC0F7FF0800F5CF96
:105108009BF01B4A1C2A00019B5101E11200250E4D
:105118009B1904E09B51E5EC67F0ECD7946B956B19
:10512800966B976B1BC0F6FF1CC0F7FF0800F5CF06
:105138009BF01B4A1C2A300E9B190DE1976B010E40
:10514800966F1BC0F6FF1CC0F7FF0800F5CF9BF059
:105158001B4A1C2A06D02D0E9B1903E1976B020EE1
:10516800EFD72A0E9B1943E11D50D96EDA6A020E59
:10517800DF26DF5CD96EDA6ADECF8CF0DECF8DF009
:105188008DAF0BD08C5100088C6F8D51D8A0E82AB8
:1051980000088D6F976B020E966F8CC094F08DC0CF
:1051A80095F01BC0F6FF1CC0F7FF0800F5CF9BF079
:1051B8001B4A1C2A22D00A0E9403F3CF1EF0F4CF08
:1051C8001FF09503F3501F269B511E26000E1F2229
:1051D800D00E1E24946FFF0E1F20956F1BC0F6FF84
:1051E8001CC0F7FF0800F5CF9BF01B4A1C2A2F0EA6
:1051F8009B6503D0390E9B65DED76C0E9B1903E0C7
:105208004C0E9B190AE196851BC0F6FF1CC0F7FFE0
:105218000800F5CF9BF01B4A1C2A9B5101E11200A4
:105228009BC09AF0600E9A6575D0200E9A5F72D076
:105238001D50D96EDA6A020EDF26DF5CD96EDA6A93
:10524800DECF84F0DECF85F0926B936B03D0000144
:10525800924B932B925184251E6E935185211F6E7C
:105268001EC0F6FF1FC0F7FF000EF86E0E0EF764A3
:1052780003D00800F55005D0F6CFE9FFF7CFEAFFD5
:10528800EF50000904E0E3D7200EE5EC67F00001D9
:1052980096B30BD092511E6E93511F6E924B932B67
:1052A80094511E5C95511F58EFE384C00FF085C0E0
:1052B80010F052EC62F003D0200EE5EC67F000012C
:1052C80092511E6E93511F6E924B932B94511E5CFC
:1052D80095511F5801E30ED7EFD71D50D96EDA6AE2
:1052E800DF50DF2ADF2AD96EDA6ADF50E5EC67F093
:1052F80001D7876B020E08D0876B080E05D0876B25
:105308000A0E02D0876B100E866F1AD09B51E5ECFF
:1053180067F0F0D69A511E6E1F6A1F50F7E11E50B3
:10532800420AE7E0010AD9E0070AE9E00B0AE4E0EB
:105338001C0A01E17DD7060AE2E00D0AE3E0E6D7A0
:1053480096A511D01D50D96EDA6A040EDF26DF5CEF
:10535800D96EDA6ADECF8EF0DECF8FF0DECF90F036
:10536800DECF91F027D0440E9A1913E01D50D96E64
:10537800DA6ADF50DF2ADF2AD96EDA6ADECF1EF05A
:10538800DDCF1FF01EC08EF01FC08FF0906B916BA9
:1053980011D01D50D96EDA6ADF50DF2ADF2AD96EA4
:1053A800DA6ADECF8EF0DDCF8FF0000E8FBFFF0EF2
:1053B800906F916F440E9A190CE191AF0AD08E6DDF
:1053C8008F1FD8B08F2B901FD8B0902B000E9157FD
:1053D8009689986B996B8EC088F08FC089F090C0C1
:1053E8008AF091C08BF088C00EF089C00FF08AC097
:1053F80010F08BC011F086C012F087C013F0146A49
:10540800156A6DEC61F00E5000019A6F88C00EF0BD
:1054180089C00FF08AC010F08BC011F086C012F05E
:1054280087C013F0146A156A3EEC5FF00EC088F06E
:105438000FC089F010C08AF011C08BF0090E00016E
:105448009A650BD0780E9B1903E0816B070E02D08A
:10545800816B270E806F80519A279851600FD96E03
:10546800DA6A9A51300FDF6E984B992B885189115F
:105478008A118B1105E0995103E1200E985DB3E381
:1054880096A908D09851600FD96EDA6A2D0EDF6E92
:10549800984B992B98C092F099C093F096B103D08D
:1054A800836B200E02D0836B300E826F82C09AF01D
:1054B80003D09A51E5EC67F0000196B30BD09251F6
:1054C8001E6E93511F6E924B932B94511E5C9551F7
:1054D8001F58EFE39807D8A099079851600FD96E25
:1054E800DA6ADF50E5EC67F000019851991104E0A1
:1054F800F1D7200EE5EC67F0000192511E6E935132
:105508001F6E924B932B94511E5C95511F5801E3CB
:10551800F1D5EFD781C0D9FF82C0DAFFDECF98F08E
:10552800DDCF99F0835184118511861128E120EE91
:105538000BF09851D9269951DA22DECF90F0DECFC0
:1055480091F0DECF92F0DECF93F09051911192114D
:1055580093110FE020EE13F09851D9269951DA22D1
:10556800DE50905DDE509159DE509259DE509359CD
:1055780052E3010E906F916B926B936B4CD081C08C
:1055880045F082C046F083C047F084C048F085C02B
:1055980049F086C04AF098EC30F045C09AF046C011
:1055A8009BF047C09CF048C09DF000019D519C11A4
:1055B8009B1109E1020E9A5D06E2010E816F826B72
:1055C800836B846B000C9A290FE19B290DE19C29C0
:1055D8000BE19D2909E19AC081F09BC082F09CC033
:1055E80083F09DC084F0120020EE13F09851D92664
:1055F8009951DA22DE509A5DDE509B59DE509C5953
:10560800DE509D59E8E383C090F084C091F085C0D6
:1056180092F086C093F020EE0FF09851D926995158
:10562800DA22DE50DE10DE10DE1005E1816B826BBF
:10563800836B846B1200946B956B966B976B83519D
:10564800901909E18451911906E1855192197DE17A
:1056580086519319D8A479D09029946F000E91217E
:10566800956F000E9221966F000E9321976F20EE92
:1056780013F09851D9269951DA22DE50945DDE5004
:105688009559DE509659DE50975905E3020E946FEE
:10569800956B966B976B81C045F082C046F094C0BD
:1056A80047F095C048F096C049F097C04AF098EC8A
:1056B80030F045C09AF046C09BF047C09CF048C007
:1056C8009DF000019A059B119C119D1184E09A2977
:1056D80007E19B2905E19C2903E19D2901E17BD78D
:1056E8009A519B119C119D1130E020EE0BF09851BE
:1056F800D9269951DA22DECF9AF0DECF9BF0DECFA1
:105708009CF0DECF9DF09D519C119B1103E1020E90
:105718009A5D17E320EE13F09851D9269951DA22B1
:10572800DE509A5DDE509B59DE509C59DE509D59E3
:1057380008E29AC090F09BC091F09CC092F09DC086
:1057480093F0946B956B966B976B9451951196119A
:10575800971162E190C094F091C095F092C096F0D4
:1057680093C097F0942B000E95239623972320EE51
:1057780013F09851D9269951DA22DE50945DDE5003
:105788009559DE509659DE5097590DE3020E946FE5
:10579800956B966B976B93519211911104E1020EE0
:1057A800905D01E243D781C045F082C046F094C0C5
:1057B80047F095C048F096C049F097C04AF098EC79
:1057C80030F045C09AF046C09BF047C09CF048C0F6
:1057D8009DF000019A519B119C119D111DE09A05A5
:1057E8009B119C119D1101E1F6D69A2907E19B298D
:1057F80005E19C2903E19D2901E1EDD69051941919
:10580800B1E191519519AEE192519619ABE19351DD
:10581800971901E10BD7A6D798C060F099C061F03D
:1058280094C062F095C063F096C064F097C065F0CC
:1058380066696769686969694EEC24F08F6F8F51F2
:105848001CE1835184118511861117E098C060F01E
:1058580099C061F083C062F084C063F085C064F0D1
:1058680086C065F094C066F095C067F096C068F091
:1058780097C069F04EEC24F08F6F8F5143E120EE12
:105888000BF09851D9269951DA2294C0DEFF95C0C1
:10589800DEFF96C0DEFF97C0DEFF20EE0FF09851C6
:1058A800D9269951DA2210EE13F09851E126995130
:1058B800E222FE0EE6248B6FFF0EE6208C6FFF0EB1
:1058C800E6208D6FFF0EE6208E6FDE508B5DDE507A
:1058D8008C59DE508D59DE508E590BE320EE0FF0B7
:1058E8009851D9269951DA22DE06000EDE5ADE5A80
:1058F800DE5A20EE04F09851D9269951DA22000E8A
:10590800DB800DD08F0507E0010E946F000E956BBC
:10591800966B976B04D0946995699669976994C05A
:1059280081F095C082F096C083F097C084F0120091
:10593800000E0001746F030E756F350E766F0B0E37
:10594800776F020E796F786BF30E7A6F7B6B66EC6C
:105958001DF00101686F630E00019C6FFD0E9D6FC5
:10596800F3C09EF0F4C09FF0F0EC67F0F56BF66BB7
:10597800F16BF26BF76BF86BF751D30FD96EDA6AEC
:10598800DF6AF751E20FD96EDA6A000EDF6EF74B65
:10599800F82BF8BFF1D7F85103E10F0EF75DECE3F0
:1059A800F96BFA6B43D1350EF925D96E0B0EFA2136
:1059B800DA6E0D0EDE1801E0FED0910E0E6EFF0EAF
:1059C8000F6ED30E106E00EC5CF00E500F1007E156
:1059D800E20E156EE4EC52F015500101FB6F8B0ED0
:1059E8000E6EFF0E0F6ED30E106E00EC5CF00E50B4
:1059F8000F1007E1E20E156EE4EC52F015500101AC
:105A0800696F700E0E6EFF0E0F6ED30E106E00ECE7
:105A18005CF00E500F1007E1E20E156EE4EC52F048
:105A280015500101646FD50E0E6EFF0E0F6ED30E6A
:105A3800106E00EC5CF00E500F1007E1E20E156ED0
:105A4800E4EC52F015500101626FDD0E0E6EFF0E90
:105A58000F6ED30E106E00EC5CF00E500F1007E1C5
:105A6800E20E156EE4EC52F015500101CF6FD90E1D
:105A78000E6EFF0E0F6ED30E106E00EC5CF00E5023
:105A88000F1008E1E20E156EE4EC52F015C052F169
:105A980016C053F10001FB6BFC6BC40E8A6F8B6B55
:105AA800770E8C6FFF0E8D6FFBC08EF0FCC08FF0F1
:105AB800F7EC64F0C40E0E6E0F6AD30E106E00EC95
:105AC8005CF00E500F1018E10F0E0001FB03F3CF2E
:105AD800C2F0F4CFC3F0FC03F350C327350EC22540
:105AE8000E6E0D0EC3210F6EE20E106E116A136A50
:105AF8000F0E126EFDEC61F00001FB4BFC2BFCBF9E
:105B0800CCD7FC5103E1100EFB5DC7E3FC6B010E23
:105B1800FB6FC40E8A6F8B6B7E0E8C6FFF0E8D6FC2
:105B2800FBC08EF0FCC08FF0F7EC64F0C40E0E6E74
:105B38000F6AD30E106E00EC5CF00E500F1018E1D7
:105B48000F0E0001FB03F3CFC2F0F4CFC3F0FC0348
:105B5800F350C327250EC2250E6E0E0EC3210F6EFD
:105B6800E20E106E116A136A0F0E126EFDEC61F0F0
:105B78000001FB4BFC2BFCBFCCD7FC5103E1040E0E
:105B8800FB5DC7E3F76BF86BF751D30FD96EDA6A91
:105B9800DF6AF751E20FD96EDA6A000EDF6EF74B53
:105BA800F82BF8BFF1D7F85103E10F0EF75DECE3DE
:105BB800F16BF26B15D0350EF925D96E0B0EFA2163
:105BC800DA6E0A0EDE1830E0350EF925D96E0B0EA6
:105BD800FA21DA6E200EDE1806E1F26B010EF16F83
:105BE800F56BF66B21D0F151F21109E0350EF9256C
:105BF800D96E0B0EFA21DA6EF551E20F08D0350E88
:105C0800F925D96E0B0EFA21DA6EF551D30FE16E34
:105C1800E26ADFCFE7FFF6BF05D0F65105E10F0EC8
:105C2800F55D02E2F54BF62BF94BFA2BF351F95DD2
:105C3800F451FA5901E2B7D6530E9C6FFD0E9D6FD1
:105C480064C19EF09F6BF0EC67F0CD0E9C6FFD0E6B
:105C58009D6FFBC19EF09F6BF0EC67F0AF0E9C6FE1
:105C6800FD0E9D6F69C19EF09F6BF0EC67F0BE0E54
:105C78009C6FFD0E9D6FCFC19EF09F6BF0EC67F09F
:105C8800440E9C6FFC0E9D6F52C19EF053C19FF055
:105C9800F0EC67F0FB6BFC6BC00E9C6FFC0E9D6F0D
:105CA800FBC09EF0FCC09FF00F0EFB03F3CFC2F0C9
:105CB800F4CFC3F0FC03F350C327350EC225A06F01
:105CC8000D0EC321A16FF0EC67F0FB4BFC2BFCBF62
:105CD800E3D7FC5103E1100EFB5DDEE3FA6B010E26
:105CE800F96FD10E9C6FFC0E9D6FF9C09EF0FAC043
:105CF8009FF00F0EF903F3CFC2F0F4CFC3F0FA030D
:105D0800F350C327250EC225A06F0E0EC321A16F25
:105D1800F0EC67F0F94BFA2BFABFE3D7FA5103E13D
:105D2800040EF95DDEE3340E9C6FF90E9D6FF0EF03
:105D380067F053500C0D030EF324D96E010EF420B6
:105D4800DA6EDF2A53500C0D030EF324D96E010EC0
:105D5800F420DA6EDF500001C76FC86BC969CA69E1
:105D680053500C0D0B0EF324D96E010EF420DA6E8D
:105D7800DF50CB6FCC6BC951CB27CA51CC23C7514D
:105D8800CB5DCC51800ACD6FC851800ACD594BE20A
:105D980053500C0D030EF324D96E010EF420DA6E65
:105DA800DF6A53500C0D020EF324D96E010EF42055
:105DB800DA6EDF2A53500C0D020EF324D96E010E51
:105DC800F420DA6EDF50C76FC86BC969CA695350CF
:105DD8000C0D0A0EF324D96E010EF420DA6EDF5092
:105DE800CB6FCC6BC951CB27CA51CC23C751CB5DE4
:105DF800CC51800ACD6FC851800ACD5914E2535056
:105E08000C0D020EF324D96E010EF420DA6EDF6A4F
:105E180053500C0D000EF324D96E010EF420DA6EE7
:105E2800DE2A000EDD2253500C0D030EF324D96E2A
:105E3800010EF420DA6EDF50C76FC7C0C8F0C96B17
:105E4800CA6BCB6BCAC0CBF0C9C0CAF0C8C0C9F016
:105E5800C86B53500C0D0B0EF324D96E010EF420B1
:105E6800DA6EDF50CC6FCCC0CDF0CE6BCF6BD06B81
:105E780053500C0D020EF324D96E010EF420DA6E85
:105E8800DF50D16FD1C0D2F0D36BD46BD56BD4C0F7
:105E9800D5F0D3C0D4F0D2C0D3F0D26BD251CD0359
:105EA800F3CFD6F0F4CFD7F0D86BD96BCE03F3503D
:105EB800D727F450D823000ED923D351CD03F3505C
:105EC800D727F450D823000ED923D251CF03F3504B
:105ED800D827F450D923D351CE03F350D827F45000
:105EE800D923D451CD03F350D827F450D923D05116
:105EF800D203F350D927D351CF03F350D927D45124
:105F0800CE03F350D927D551CD03F350D927535099
:105F18000C0D0A0EF324D96E010EF420DA6EDF5050
:105F2800DA6FDAC0DBF0DC6BDD6BDE6B53500C0D27
:105F38000B0EF324D96E010EF420DA6EDF50DF6FFA
:105F4800DFC0E0F0E16BE26BE36B53500C0D000E29
:105F5800F324D96E010EF420DA6EDECFE4F0DDCF43
:105F6800E5F0E4C0E6F0E5C0E7F0000EE7BFFF0E9D
:105F7800E86FE96FE651E003F3CFEAF0F4CFEBF016
:105F8800EC6BED6BE103F350EB27F450EC23000EC0
:105F9800ED23E751E003F350EB27F450EC23000E18
:105FA800ED23E651E203F350EC27F450ED23E751DB
:105FB800E103F350EC27F450ED23E851E003F350EC
:105FC800EC27F450ED23E351E603F350ED27E751B6
:105FD800E203F350ED27E851E103F350ED27E951CF
:105FE800E003F350ED27ECC0EDF0EBC0ECF0EAC0B5
:105FF800EBF0EA6BEA51DB03F3CFEEF0F4CFEFF00E
:10600800F06BF16BDC03F350EF27F450F023000E34
:10601800F123EB51DB03F350EF27F450F023000E8C
:10602800F123EA51DD03F350F027F450F123EB514B
:10603800DC03F350F027F450F123EC51DB03F35069
:10604800F027F450F123DE51EA03F350F127EB5126
:10605800DD03F350F127EC51DC03F350F127ED5148
:10606800DB03F350F127D651EE25F26FD751EF211C
:10607800F36FD851F021F46FD951F121F56FC85160
:10608800F225F66FC951F321F76FCA51F421F86F61
:10609800CB51F521F96F53500C0D040EF324D96E32
:1060A800010EF420DA6EF6C0DEFFF7C0DEFFF8C09E
:1060B800DEFFF9C0DEFF5350220D000EF3249E6F61
:1060C800030EF4209F6F53500C0D040EF324D96E69
:1060D800010EF420DA6EDECFA0F0DECFA1F0DECF25
:1060E800A2F0DECFA3F0B0EC12F04B6E4B5019E0EB
:1060F8001F0E9C6FFB0E9D6F53500C0D040EF32466
:10610800D96E010EF420DA6EDECF9EF0DECF9FF05E
:10611800DECFA0F0DECFA1F04BC0A2F0A36BF0EC75
:1061280067F001015B6B120045C0D9FF46C0DAFF7A
:10613800DECF72F0DDCF73F04A504910481003E10A
:10614800020E475C10E3000120EE13F07251D926CD
:106158007351DA22DE50475CDE504858DE50495809
:10616800DE504A5808E3010E00016C6F000E6D6B9B
:106178006E6B6F6B8FD16C696D696E696F6976D163
:1061880047C070F048C071F0D8907131616F7031BC
:10619800606F605170276151712372C03AF073C00B
:1061A8003BF020EE1FF07251D9267351DA22DECF70
:1061B80060F0DECF61F0DECF62F0DECF63F070C05A
:1061C80064F071C065F0090E666FD890653364336A
:1061D800662FFBD7645160253C6E655161213D6E89
:1061E800000E62213E6E000E63213F6E1BEC5BF0D9
:1061F800000901E04FD100016069010E616F70C0B4
:1062080062F071C063F0605162176151631772C028
:1062180064F073C065F062516427635165232F0EE3
:106228006425D96E000E6521DA6EDF506A6F6B6BDC
:10623800704B712B72C03AF073C03BF020EE1FF028
:106248007251D9267351DA22DECF60F0DECF61F0C9
:10625800DECF62F0DECF63F070C064F071C065F02D
:10626800090E666FD89065336433662FFBD7645187
:1062780060253C6E655161213D6E000E62213E6EC7
:10628800000E63213F6E1BEC5BF0000901E002D1B8
:1062980000016069010E616F70C062F071C063F047
:1062A800605162176151631772C064F073C065F082
:1062B80062516427635165232F0E6425D96E000E41
:1062C8006521DA6EDF50676F666B66516A13675136
:1062D8006B1347B006D06A51686F0F0E6B15696F64
:1062E8000FD06AC060F06BC061F0040E626FD89086
:1062F80061336033622FFBD760C068F061C069F01A
:1063080068C06CF069C06DF04ED072C03AF073C0CE
:106318003BF020EE1FF07251D9267351DA22DECFFE
:1063280060F0DECF61F0DECF62F0DECF63F0485080
:10633800646F4950656F4A50666F676B605164259A
:106348003C6E615165213D6E625166213E6E63511E
:1063580067213F6E1BEC5BF0000901E09BD0000158
:106368006069010E616F47C062F048C063F0D89061
:1063780062376337605162176151631772C064F006
:1063880073C065F062516427635165232F0E64253D
:106398000E6E000E65210F6E0EEC66F00EC06CF0EE
:1063A8000FC06DF000016E6B6F6B74D072C03AF065
:1063B80073C03BF020EE1FF07251D9267351DA22D8
:1063C800DECF60F0DECF61F0DECF62F0DECF63F0CB
:1063D80047C064F048C065F049C066F04AC067F03D
:1063E800080E05D0D8906733663365336433E82EDA
:1063F800F9D7605164253C6E615165213D6E62514B
:1064080066213E6E635167213F6E1BEC5BF000090D
:1064180041E100016069010E616F47C062F048C048
:1064280063F0D89062376337D8906237633760512A
:1064380062176151631772C064F073C065F06251EE
:106448006427635165232F0E64250E6E000E6521A7
:106458000F6ED8EC59F00E5000016C6F0F506D6F35
:1064680010506E6F0F0E11146F6F14D072C0D9FFD9
:1064780073C0DAFFDF50606F616B615101E073D662
:106488006051010A01E17CD6030A01E13ED7010A05
:106498008DE069D66CC045F06DC046F06EC047F01F
:1064A8006FC048F01200536A01015D6B536A030E16
:1064B800536401D0A8D1535003E1266A276A03D058
:1064C800276A010E266E53501E0D1B0EF324D96E3B
:1064D800020EF420DA6EDF6A53501E0D000EF3240C
:1064E800D96E020EF420DA6EDF6A53501E0D070EC5
:1064F800F324D96E020EF420DA6E070EDE6AE8067F
:10650800FDE20D0E2602F3CFC2F0F4CFC3F027024E
:10651800F3500001C327A20EC225D96E020EC32173
:10652800DA6EDF50C46FC4C0C5F0C66BC76BC86BEA
:10653800C7C0C8F0C6C0C7F0C5C0C6F0C56B0D0E51
:106548002602F3CFC9F0F4CFCAF02702F350CA27C6
:10655800A10EC925D96E020ECA21DA6EDF50CB6FA3
:10656800CBC0CCF0CD6BCE6BCF6BCDC0CFF0CCC059
:10657800CEF0CD6BCC6B0D0E2602F3CFD0F0F4CF5E
:10658800D1F02702F350D127A00ED025D96E020EE4
:10659800D121DA6EDF50D26FD2C0D3F0D46BD56B75
:1065A800D66BD3C0D6F0D56BD46BD36BCC51D32577
:1065B800D76FCD51D421D86FCE51D521D96FCF51B6
:1065C800D621DA6FC551D725DB6FC651D821DC6FCC
:1065D800C751D921DD6FC851DA21DE6F0D0E2602B1
:1065E800F3CFDFF0F4CFE0F02702F350E027A30E5B
:1065F800DF25D96E020EE021DA6EDF50DB25E16F70
:10660800000EDC21E26F000EDD21E36F000EDE21BB
:10661800E46FE1C0E5F0E2C0E6F0E3C0E7F0E4C013
:10662800E8F0E96BE8BFE969E9C0EAF0E9C0EBF036
:10663800E9C0ECF053501E0D0F0EF324D96E020E74
:10664800F420DA6EE5C0DEFFE6C0DEFFE7C0DEFF5D
:10665800E8C0DEFFE9C0DEFFEAC0DEFFEBC0DEFF18
:10666800ECC0DEFF53501E0D1C0EF324D96E020E33
:10667800F420DA6EDECFC2F0DDCFC3F0C2C00EF078
:10668800C3C00FF0106A116A126A136A146A156A95
:1066980053501E0D0F0EF324D96E020EF420DA6E3D
:1066A800DECFC4F0DECFC5F0DECFC6F0DECFC7F058
:1066B800DECFC8F0DECFC9F0DECFCAF0DECFCBF038
:1066C800C4C016F0C5C017F0C6C018F0C7C019F08E
:1066D800C8C01AF0C9C01BF0CAC01CF0CBC01DF05E
:1066E800B5EC5DF00EC0CCF00FC0CDF010C0CEF010
:1066F80011C0CFF012C0D0F013C0D1F014C0D2F046
:1067080015C0D3F053501E0D0F0EF324D96E020E90
:10671800F420DA6ECCC0DEFFCDC0DEFFCEC0DEFFD7
:10672800CFC0DEFFD0C0DEFFD1C0DEFFD2C0DEFFAB
:10673800D3C0DEFF53501E0D170EF324D96E020E80
:10674800F420DA6EDE6ADE6ADE6A010EDD6E0E0E97
:1067580000019C6FFA0E9D6F53C09EF09F6B5350C3
:106768001E0D0F0EF324D96E020EF420DA6EDECF62
:10677800C2F0DECFC3F0DECFC4F0DECFC5F0DECF8F
:10678800C6F0DECFC7F0DECFC8F0DECFC9F0C2C09A
:10679800A0F0C3C0A1F0C4C0A2F0C5C0A3F0C6C099
:1067A800A4F0C7C0A5F0C8C0A6F0C9C0A7F0535050
:1067B8001E0D0F0EF324D96E020EF420DA6EDECF12
:1067C800CAF0DECFCBF0DECFCCF0DECFCDF0DECF1F
:1067D800CEF0DECFCFF0DECFD0F0DECFD1F0CAC022
:1067E800A8F0CBC0A9F0CCC0AAF0CDC0ABF0CEC009
:1067F800ACF0CFC0ADF0D0C0AEF0D1C0AFF0F0EC8F
:1068080067F0532A54D60101606B526A5F6B4E6A77
:106818004F6A020E516E5E6F8390020C9EC0D9FFC4
:106828009FC0DAFFDECFB2F0DDCFB3F020EE0EF07E
:106838009E51D9269F51DA22DECFA2F0DECFA3F0F7
:10684800DECFA4F0DECFA5F0200EA225AE6F000E9D
:10685800A321AF6F000EA421B06F000EA521B16F68
:10686800B15103E1200EB05D0AE320EE16F09E510F
:10687800D9269F51DA22DE6ADE6ADE6ADD6A20EEF8
:1068880016F09E51D9269F51DA22DE50DE10DE1016
:10689800DE1001E1040CAE51A26F010EAF15A36F1B
:1068A800A46BA56BA211A411A51101E029D120EEBA
:1068B80016F09E51D9269F51DA22DE2A000EDE22DA
:1068C800DE22DE2220EE12F09E51D9269F51DA22D6
:1068D800DE50DE10DE10DE102CE120EE07F0B251A3
:1068E800D926B351DA22DECFA2F0DDCFA3F0A25130
:1068F800A46FA351A56FA66BA76BAEC0A8F0AFC0DD
:10690800A9F0B0C0AAF0B1C0ABF0060E05D0D8907F
:10691800AB33AA33A933A833E82EF9D7A451A85D1D
:10692800A551A959A651AA59A751AB5901E2E8D0D6
:106938006ED0A269A36920EE09F0B251D926B351ED
:10694800DA22DECFA4F0DDCFA5F0A251A427A3510F
:10695800A523AEC0A6F0AFC0A7F0B0C0A8F0B1C0E4
:10696800A9F00A0E05D0D890A933A833A733A633C7
:10697800E82EF9D7A451A615AA6FA551A715AB6F94
:10698800AC6BAD6BAA11AC11AD1101E0B9D09EC0D2
:1069980045F09FC046F020EE12F09E51D9269F5137
:1069A800DA22DECF47F0DECF48F0DECF49F0DECF87
:1069B8004AF098EC30F045C0B4F046C0B5F047C096
:1069C800B6F048C0B7F00001B751B611B51104E1EF
:1069D800020EB45D01E2020CB42907E1B52905E114
:1069E800B62903E1B72901E1010C20EE13F0B251F9
:1069F800D926B351DA22DE50B45DDE50B559DE50E7
:106A0800B659DE50B75950E3A051A1110BE120EE61
:106A180016F09E51D9269F51DA22DE6ADE6ADE6AB6
:106A2800DD6A040C9EC081F09FC082F020EE12F057
:106A38009E51D9269F51DA22DECF83F0DECF84F033
:106A4800DECF85F0DECF86F08EEC2AF081C0B4F080
:106A580082C0B5F083C0B6F084C0B7F0B451B511A8
:106A6800B611B71101E1070CB405B511B611B7118C
:106A780001E1020CB42907E1B52905E1B62903E1D2
:106A8800B72901E1010CB2C03AF0B3C03BF0B4C081
:106A98003CF0B5C03DF0B6C03EF0B7C03FF062EC88
:106AA80052F0000901E0010C000120EE12F09E51A5
:106AB800D9269F51DA22B4C0DEFFB5C0DEFFB6C0CA
:106AC800DEFFB7C0DEFFB2C00EF0B3C00FF0B4C037
:106AD80010F0B5C011F0B6C012F0B7C013F0CEEC8C
:106AE80050F0000120EE16F09E51D9269F51DA226F
:106AF8000EC0DEFF0FC0DEFF10C0DEFF11C0DEFFDC
:106B080020EE0EF09E51D9269F51DA22AEC0DEFF4C
:106B1800AFC0DEFFB0C0DEFFB1C0DEFFA269010E6C
:106B2800A36FAEC0A4F0AFC0A5F0A251A417A351A3
:106B3800A517B2C0A6F0B3C0A7F0A451A627A551C7
:106B4800A7232F0EA627000EA72320EE1AF09E518A
:106B5800D9269F51DA22A6C0DEFFA7C0DDFF000CB0
:106B680053500C0D030EF324D96E010EF420DA6E87
:106B7800DF506D6F6DC16EF16F6B706B716B70C1B3
:106B880071F16FC170F16EC16FF16E6B53500C0DE6
:106B98000B0EF324D96E010EF420DA6EDF50726FFB
:106BA80072C173F1746B756B766B53500C0D020EDA
:106BB800F324D96E010EF420DA6EDF50776F77C1B7
:106BC80078F1796B7A6B7B6B7AC17BF179C17AF159
:106BD80078C179F1786B78517303F3CF7CF1F4CFF6
:106BE8007DF17E6B7F6B7403F3507D27F4507E2319
:106BF800000E7F2379517303F3507D27F4507E23D1
:106C0800000E7F2378517503F3507E27F4507F23BD
:106C180079517403F3507E27F4507F237A5173031C
:106C2800F3507E27F4507F2376517803F3507F2763
:106C380079517503F3507F277A517403F3507F27F6
:106C48007B517303F3507F2753500C0D0A0EF32426
:106C5800D96E010EF420DA6EDF50806F80C181F1A9
:106C6800826B836B846B53500C0D0B0EF324D96E1F
:106C7800010EF420DA6EDF50856F85C186F1876BCF
:106C8800886B896B53500C0D000EF324D96E010EDE
:106C9800F420DA6EDECF8AF1DDCF8BF18AC18CF178
:106CA8008BC18DF1000E8DBFFF0E8E6F8F6F8C51D3
:106CB8008603F3CF90F1F4CF91F1926B936B870336
:106CC800F3509127F4509223000E93238D5186039D
:106CD800F3509127F4509223000E93238C5188038C
:106CE800F3509227F45093238D518703F350922742
:106CF800F45093238E518603F3509227F450932334
:106D080089518C03F35093278D518803F3509327AF
:106D18008E518703F35093278F518603F35093279F
:106D280092C193F191C192F190C191F1906B905100
:106D38008103F3CF94F1F4CF95F1966B976B8203AF
:106D4800F3509527F4509623000E97239151810311
:106D5800F3509527F4509623000E97239051830300
:106D6800F3509627F450972391518203F3509627B6
:106D7800F450972392518103F3509627F4509723A8
:106D880084519003F350972791518303F350972729
:106D980092518203F350972793518103F350972719
:106DA8007C519425986F7D519521996F7E5196213C
:106DB8009A6F7F5197219B6F6E5198250001DC6F68
:106DC80001016F5199210001DD6F010170519A2174
:106DD8000001DE6F010171519B210001DF6F5350EB
:106DE800220D000EF3249E6F030EF4209F6FDCC06B
:106DF800A0F0DDC0A1F0DEC0A2F0DFC0A3F0B0ECCF
:106E080012F0DB6FDB5111E01F0E9C6FFB0E9D6FC4
:106E1800DCC09EF0DDC09FF0DEC0A0F0DFC0A1F0B6
:106E2800DBC0A2F0A36BF0EC67F07F0E9C6FFE0E48
:106E38009D6FF0EC67F0839053500C0D040EF32413
:106E4800D96E010EF420DA6EDCC0DEFFDDC0DEFF95
:106E5800DEC0DEFFDFC0DEFF01015B6B5A6BBFEFF8
:106E68003FF074C0D9FF75C0DAFFDECF8CF0DDCFFC
:106E78008DF0795109E1200E785DD8B0020C76C00A
:106E88007AF01F0E7A1701E0020C20EE0EF0745112
:106E9800D9267551DA2276C0DEFF77C0DEFF78C0CA
:106EA800DEFF79C0DEFF20EE06F07451D926755159
:106EB800DA22DECF88F0DECF89F0DECF8AF0DECFAF
:106EC8008BF0885189118A118B1115E18CC0D9FF7B
:106ED8008DC0DAFF020EDF640ED020EE23F08C5155
:106EE800D9268D51DA22DECF88F0DECF89F0DECFC9
:106EF8008AF0DECF8BF0885189118A118B1140E11D
:106F080020EE07F08C51D9268D51DA22DECF7AF0A7
:106F1800DDCF7BF07A517C6F7B517D6F7E6B7F6B11
:106F280076C080F077C081F078C082F079C083F0B5
:106F3800060E05D0D8908333823381338033E82E10
:106F4800F9D77C51805D7D5181597E5182597F519D
:106F5800835901E3020C20EE23F08C51D9268D5180
:106F6800DA2210EE16F07451E1267551E222DECFD6
:106F7800E6FFDECFE6FFDECFE6FFDECFE6FF87D017
:106F880020EE09F08C51D9268D51DA22DECF7AF025
:106F9800DDCF7BF07A517C6F7B517D6F7E6B7F6B91
:106FA800090ED8907C377D377E377F37E82EF9D7A2
:106FB8007CC084F07DC085F07EC086F07FC087F0FD
:106FC80040D074C045F075C046F088C047F089C00D
:106FD80048F08AC049F08BC04AF098EC30F045C0C0
:106FE80088F046C089F047C08AF048C08BF000019D
:106FF800882907E1892905E18A2903E18B2901E12B
:10700800010C8B518A11891104E1020E885DD8A008
:10701800020C20EE13F08C51D9268D51DA22DE5065
:10702800885DDE508959DE508A59DE508B5901E35C
:10703800020C8451765F8551775B8651785B875166
:10704800795B8451765D8551775986517859875196
:107058007959B7E28CC00EF08DC00FF088C010F0DF
:1070680089C011F08AC012F08BC013F0CEEC50F03A
:10707800000120EE16F07451D9267551DA220EC09F
:10708800DEFF0FC0DEFF10C0DEFF11C0DEFF20EE06
:1070980012F07451D9267551DA2288C0DEFF89C0F2
:1070A800DEFF8AC0DEFF8BC0DEFF20EE16F07451D3
:1070B800D9267551DA22DE50DE10DE10DE1001E12D
:1070C800020C76C07AF077C07BF078C07CF079C08B
:1070D8007DF00A0E05D0D8907D337C337B337A332C
:1070E800E82EF9D720EE16F07451D9267551DA2218
:1070F8007A51DE267B51DE227C51DE227D51DE2252
:107108007A69010E7B6F76C07CF077C07DF07A518A
:107118007C177B517D178CC07EF08DC07FF07C5131
:107128007E277D517F232F0E7E27000E7F2320EEA2
:107138001AF07451D9267551DA227EC0DEFF7FC05D
:10714800DDFF000C000E0001F36F250EF26F000E3C
:10715800F16F050EF06F0101FB5105E1000E000112
:10716800F36F280EF26F010164510DE1FA6B350ED1
:1071780000018A6F0D0E8B6F720E8C6FFE0E8D6F75
:10718800F7EC64F00DD02E0E00019C6FFA0E9D6F87
:1071980064C19EF09F6BFAC1A0F0A16BF0EC67F0A0
:1071A800EB0E9C6FFD0E9D6F0101FA510F0D350E10
:1071B800F32400019E6F0D0EF4209F6FF0EC67F032
:1071C800050E0001EF6F0F0EEE6FF10EE82EFED7E1
:1071D800EE2FFCD7EF2FFAD7CCD0AF0E0F6EFC0EE8
:1071E800106E52EC62F0030E0101CF6105D096508B
:1071F800CF19F00BCF1905D0CFC193FF9650F00BE4
:107208000A09966E000E0001CE6F030ECF6F650E51
:10721800D06FFE0ED16F010ED26F7EEC15F001011A
:10722800686F6851CEEC62F0010168510AE1DEEC4A
:107238001AF0000E6D6F030E6E6F15EC65F001010C
:10724800686F6851CEEC62F0F36B280EF26F8DD048
:107258000101FA510F0D350EF324D96E0D0EF420ED
:10726800DA6E200EDE1806E1FA2B0F0EFA657DD0D5
:10727800FA6B7BD0AD0E00019C6FFB0E9D6F010178
:10728800FA510F0D350EF32400019E6F0D0EF420F8
:107298009F6FF0EC67F0000ECE6F030ECF6F010109
:1072A800FA510F0D350EF3240001D06F0D0EF420A6
:1072B800D16F030ED26F7EEC15F00101686F685133
:1072C800CEEC62F00101685104E10001F36B3C0E61
:1072D800F26F040E0101681904E10001F36B410E1D
:1072E800F26F050E0001EF6F0F0EEE6FF10EE82E34
:1072F800FED7EE2FFCD7EF2FFAD737D0570E9C6F5B
:10730800FC0E9D6F0101FA510F0D350EF32400019B
:107318009E6F0D0EF4209F6FF0EC67F026D0570E8D
:107328009C6FFC0E9D6F0101FA510F0D350EF32471
:1073380000019E6F0D0EF4209F6FF0EC67F015D0E2
:10734800F2C0EEF0F3C0EFF0EF510FE1EE51250A75
:1073580001E143D70D0A01E17BD7050A06E01F0AC0
:1073680004E00E0ACBE07D0ADAE00001F007D8A0BD
:10737800F1070001F1BF08D0F15102E1F00504E383
:107388003C0EF219F311DCE1030E010164193BE133
:10739800839E000E0E6EC00E1FEC63F0F7EC66F0D5
:1073A800000E0E6EC00E1FEC63F03C0E0001F219C9
:1073B800F31116E10101F0510CE0F00E126E010E0E
:1073C800136E01EC5FF0950E126EFE0E136E01EC5B
:1073D8005FF0970E126EFF0E136E01EC5FF0000C5B
:1073E800350E8A6F0D0E8B6F400E8C6FFF0E8D6FF2
:1073F80068C18EF08F6BF7EC64F0350E126E0D0ECF
:10740800136E01EC5FF0000C350E0101796F0B0E65
:107418007A6FE9C00EF0EAC00FF0F9EC63F00E5095
:1074280001016D6FC70E00019E6F9F6BA06BA16B72
:10743800A26BA36BB0EC12F00101766F76510DE0F0
:10744800ED0E00019C6FFA0E9D6FF0EC67F00001E5
:10745800C76BC86BC96BCA6B1200C70E0001746F8B
:10746800756B79C176F07AC177F0010E796F786B18
:10747800740E7A6F010E7B6F66EC1DF00101766F5A
:10748800765108E0960E00019C6FFB0E9D6FF0ECA4
:1074980067F0DDD779C1D9FF7AC1DAFF800EDE182F
:1074A80008E09E0E00019C6FFC0E9D6FF0EC67F0EB
:1074B800CED720EE0AF07951D9267A51DA22DF5058
:1074C8000001EC6FEB6B010120EE0BF07951D9262E
:1074D8007A51DA22DF500001EB250101726F000EAC
:1074E8000001EC210101736F7F0E00019C6FFB0E00
:1074F8009D6F72C19EF073C19FF0F0EC67F0C70EEC
:107508009E6F9F6B010172510001EC6FEB6BEBC03A
:10751800A0F0ECC0A1F0A26BA36BB0EC12F00101DB
:10752800766F765194E1C70E0001746F756B79C15F
:1075380076F07AC177F0010E796F786B740E7A6FF6
:10754800010E7B6F66EC1DF00101766F765101E04C
:107558007ED7776B786BE9C00EF0EAC00FF077C181
:10756800EBF078C1ECF0050ED8900001EB37EC3762
:10757800E82EFAD7EB5101017925106E0001EC5184
:1075880001017A21116E6DC112F0136A27EC5DF0CA
:107598000E500F105DE177C1EBF078C1ECF0050EED
:1075A800D8900001EB37EC37E82EFAD779C1EDF027
:1075B8007AC1EEF0EB51ED27EC51EE230E0EED25DE
:1075C800D96E000EEE21DA6EDF50F06FEF6B77C1E7
:1075D800F1F078C1F2F0050ED890F137F237E82EC5
:1075E800FBD779C1F3F07AC1F4F0F151F327F251E6
:1075F800F4230F0EF325D96E000EF421DA6EDF5056
:10760800F56FF66BEF51F527F051F623F5C06EF1E3
:10761800F6C06FF10101000E6FBFFF0E706F716F42
:10762800730E00019C6FFD0E9D6F6EC19EF06FC1C1
:107638009FF070C1A0F071C1A1F0F0EC67F06EC1CD
:10764800C7F06FC1C8F070C1C9F071C1CAF01200AB
:10765800774B782B78BF7FD7785105E10F0E775D90
:1076680001E3F5D678D7F3D61850D96EDA6ADECFAB
:1076780022F0DDCF23F01C0E1624266E000E1720F4
:10768800276E26C00EF027C00FF0116A200E106E6C
:10769800136A0B0E126E5AEC67F0286A296A246A7C
:1076A800256A216A080E206E24502224196E25505E
:1076B80023201A6E19C0F6FF1AC0F7FF000EF86EE5
:1076C8000E0EF76403D00800F55005D0F6CFE9FF99
:1076D800F7CFEAFFEF502A6E244A252A210E2A60A6
:1076E80001D0BED02F0E2A1806E05C0E2A1803E03F
:1076F80036D0244A252A24502224196E25502320C6
:107708001A6E19C0F6FF1AC0F7FF000EF86E0E0EBB
:10771800F76403D00800F55005D0F6CFE9FFF7CF9E
:10772800EAFFEF502F0AE5E024502224196E255075
:1077380023201A6E19C0F6FF1AC0F7FF000EF86E64
:107748000E0EF76403D00800F55005D0F6CFE9FF18
:10775800F7CFEAFFEF505C0A01E082D0CAD72E0EBD
:107768002A1805E02050285C215029580FE30B0EF9
:1077780020182110D8B4060C2E0E2A1801E0060C89
:10778800296A080E286E216A0B0E8DD72A50F7EC4D
:1077980062F00E500F1044E024502224196E255038
:1077A80023201A6E19C0F6FF1AC0F7FF000EF86EF4
:1077B8000E0EF76403D00800F55005D0F6CFE9FFA8
:1077C800F7CFEAFFEF501F6E244A252A1F5096EC88
:1077D80060F00E500F10D8B4060C19681A6820C053
:1077E8001BF021C01CF019501B261A501C221B50DC
:1077F800285C1C50295801E3060C28502624D96E11
:1078080029502720DA6E2AC0DFFF284A292A285063
:107818002624D96E29502720DA6E1FC0DFFF1DD01D
:10782800910E0E6EFD0E0F6E2AC010F0116A6BECF1
:1078380065F00E500F1001E0060C600E2A6405D0AA
:107848007B0E2A6002D0200E2A5E28502624D96E8C
:1078580029502720DA6E2AC0DFFF284A292A24D790
:1078680024502224196E255023201A6E1850D96EE0
:10787800DA6A19C0DEFF1AC0DDFF2850291001E1BD
:10788800060C26C0D9FF27C0DAFFE50EDE1806E190
:1078980026C0D9FF27C0DAFF050EDF6E200E2A6446
:1078A80003D01D6A1E6A03D01E6A040E1D6E20EEE8
:1078B8000BF02650D9262750DA221DC0DFFF000C16
:1078C8000F0E5316EC0E00019C6FF90E9D6F53C0FE
:1078D8009EF09F6B53501E0D1B0EF324D96E020EA3
:1078E800F420DA6EDF50A06FA16BF0EC67F0025065
:1078F8000209026E350E0E6E0B0E0F6E116A106ABB
:10790800010E136E126AE5EC4CF0040E531804E1F4
:107918000F0EE8CF35FB04D02BEE35F053C0DFFF58
:10792800FF0EE8CF36FB02011B5102E0000E0BD020
:10793800395102E0010E07D0575102E0020E03D080
:10794800755103E0030EE8CF36FB050E53605BD09C
:1079580053501E0D1B0EF324D96E020EF420DA6E5E
:10796800DFA403D0810EE8CF37FB53501E0D1B0E4A
:10797800F324D96E020EF420DA6EDFA803D0020ECB
:10798800E8CF37FB53501E0D1B0EF324D96E020EA1
:10799800F420DA6EDFA003D0020EE8CF39FB535093
:1079A8001E0D1B0EF324D96E020EF420DA6EDFA230
:1079B80003D0020EE8CF39FB53501E0D1B0EF324E3
:1079C800D96E020EF420DA6EDFA603D0800EE8CF5F
:1079D80038FB53501E0D1B0EF324D96E020EF420F3
:1079E800DA6EDFAA03D0040EE8CF37FB53501E0D22
:1079F8001B0EF324D96E020EF420DA6EDFAC03D02E
:107A0800020EE8CF3AFB8FA403D0080EE8CF3BFB69
:107A1800236A246A300E2324D96E010E2420DA6EDC
:107A2800DF1C226E370E2324D96E0B0E2420DA6E4B
:107A3800370E2324E16E0B0E2420E26EE750221449
:107A4800DF6E234A242A24BEE5D7245003E1070E1B
:107A5800235CE0E3516A020E01015D6548D0535092
:107A68001E0D010EF324D96E020EF420DA6EDF50DB
:107A7800216E21C03FFB53501E0D020EF324D96E18
:107A8800020EF420DA6EDF50216E21C040FB535005
:107A98001E0D030EF324D96E020EF420DA6EDF50A9
:107AA800216E21C041FB53501E0D040EF324D96EE4
:107AB800020EF420DA6EDF50216E21C042FB5350D3
:107AC8001E0D050EF324D96E020EF420DA6EDF5077
:107AD800216E21C043FB53501E0D060EF324D96EB0
:107AE800020EF420DA6EDF50216E21C044FB5350A1
:107AF8001E0D1B0EF324D96E020EF420DA6E000E52
:107B0800DF6E140EFBEC5DF002928390120001010F
:107B18006B6B546B556BFF0E2124256EFF0E2220D4
:107B2800266E898689808982898489888B68849071
:107B380084928494849883500F011391350EE82E13
:107B4800FED700F007D0FD0E00019C6FFF0E9D6F61
:107B5800F0EC67F08EA8F7D7E1D08EA88EAA14D0E3
:107B6800FB5112E1545155110FE0E20E00019C6FD8
:107B7800FC0E9D6F54C19EF055C19FF0F0EC67F06C
:107B8800630E01016B6FD0D0100E3C6F270E3D6F56
:107B98003E6B3F6BABD08EB28EA410D03C07000E6C
:107BA8003D5B3E5B3F5B3C2906E13D2904E13E2904
:107BB80002E13F29D8A4B2D0620E84D0010E82D04F
:107BC8008EA8ACD0020E7ED0350E5425D96E0B0E81
:107BD8005521DA6EDF1C866E5451251805E1555182
:107BE800261802E102B2899A544B552B8B6A030E70
:107BF8006B6F100E3C6F270E3D6F3E6B3F6B06D0D0
:107C08008EA204D08990050E6B6F0ED03C07000E33
:107C18003D5B3E5B3F5B3C29F3E13D29F1E13E29B9
:107C2800EFE13F297BE0ECD7100E3C6F270E3D6F4C
:107C38003E6B3F6B0DD08EA40BD0898A89808B68F0
:107C48002150545D22505559BDE3630E01013AD0CD
:107C58003C07000E3D5B3E5B3F5B3C29ECE13D2968
:107C6800EAE13E29E8E13F2959E0E5D78EB20DD097
:107C78003C07000E3D5B3E5B3F5B3C294FE13D29E5
:107C88004DE13E294BE13F2949E1040E1BD0899083
:107C9800050E6B6F100E3C6F270E3D6F3E6B3F6BF2
:107CA8003DD089848EB40DD03C07000E3D5B3E5B11
:107CB8003F5B3C2933E13D2931E13E292FE13F2952
:107CC8002DE1060E6B6F2AD0898A89808B68215036
:107CD800545D2250555901E271D7B7D7A30E000160
:107CE8009C6FFF0E9D6FF0EC67F0AFD76B51236E62
:107CF800246A245013E1235001E14DD7010A01E120
:107D08005FD7030A01E160D7010AB0E0070ABFE0C4
:107D1800010AC7E0030AD8E0640AE0E0630E010143
:107D28006B1902E08EBC19D7898089828984898879
:107D3800898A8B680F01138154C121F055C122F043
:107D480012000001F26FEE5102E057EC32F0000130
:107D5800F16BED5101E1F6D0040EF21902E1525037
:107D680003E1140EF21909E101015F6B4E6A4F6AD3
:107D78000001EE6B070EED6F070C3F0EF21907E1DD
:107D8800526A01015F6B0001ED6BEE6B12005F0E32
:107D9800F21907E10101606B5F6B0001ED6BEE6B9F
:107DA80012003F0EF26506D05F0EF26103D0400E5E
:107DB800F219F0E1400EF21909E1010E0101606FBC
:107DC80001015F6B0001ED6BEE6B1200200EF219E2
:107DD80003E1010E526EF4D7650EF21909E1525013
:107DE80007E04E6A4F6A010E01015F6F8380EAD790
:107DF8006E0EF21909E1525003E10101605104E0ED
:107E08008380020E01015F6F700E0001F21907E115
:107E18000101605104E04E6A4F6A030E5F6F700EF5
:107E28000001F21908E1525006E083804E6A4F6A59
:107E3800040E01010FD0720EF21901E083D05250E6
:107E480001E180D0838001015D6B1C0E4F6E2A0E0C
:107E58004E6E050E5F6FB6D7F251E5EC08F00001E3
:107E6800F16F84D0BC0E4E1809E1020E4F1806E1DE
:107E780064EC3CF001015F6B516AA4D7F251B4EC99
:107E88004FF00001F16F01015F6B70D08380350EF8
:107E98000E6E0B0E0F6E116A106A010E136E126AC7
:107EA800E5EC4CF002500209026E2BEE35F051C0A1
:107EB800DFFF01014A4B4B2B52514A1903E1535141
:107EC8004B1903E05251531101E0889C010EFBEC61
:107ED8005DF00292080E0001F16F01015F6B516ABB
:107EE80045D08390F16B42D0080EF21915E18390CA
:107EF800536AF16B516A030E01015D6513D00F0ED1
:107F08005D1910E0010E516E02011B5110091B6F23
:107F180009D04E6A4F6A2AD0090EF21906E18390F9
:107F2800F16B516A01015F6BF4D71F0EF2651ED029
:107F3800300EF2611BD0F2510F0B01015D6F000191
:107F4800F16BCDD701015F510001EF6FF06BF0517C
:107F58000DE1EF510BE0010A01E17ED7030A82E04F
:107F6800010A94E0070ABDE0010ABEE0F1C0EDF0A5
:107F78000001EE6B12000001D16B010ED06F838EF1
:107F88008380D26BD36BD46BD56BE1D05350220D69
:107F9800000EF324746F030EF420756F350E766FA0
:107FA8000B0E776F010E796F786BD80E7A6F7B6B3B
:107FB80066EC1DF0DA6FDA5118E0180E0101596FFE
:107FC800010E5B6F0001D96BD86FCA0E9C6FF90E5A
:107FD8009D6F53C09EF09F6BDAC0A0F0A16BD8C014
:107FE800A2F0D9C0A3F0F0EC67F00101625135E0CE
:107FF800385139113A113B1130E053500C0D040E31
:10800800F324D96E010EF420DA6E38C1C7F039C1F5
:10801800C8F03AC1C9F00001C66B000EC625CA6F88
:10802800010EC721CB6F000EC821CC6F000EC921ED
:10803800CD6FDE50CA1911E1DE50CB190EE1DE50CA
:10804800CC190BE1DE50CD1908E1350E2B6E0B0E65
:108058002C6E010162515BEC55F0029201015951FD
:1080680003E002500209026ED8C021F0D9C022F004
:108078008BEC3DF021C0D6F022C0D7F0F00E000105
:108088009C6FFE0E9D6FF0EC67F0D651D227D7514A
:10809800D323000ED423D5238EBC8EA85DD0D8510F
:1080A800D61903E1D951D7190CE0310E9C6FFE0E99
:1080B8009D6FD6C09EF0D7C09FF0F0EC67F0839418
:1080C8004BD08FEC67F092EC63F02150221004E063
:1080D800010E01015B6F40D00001CF6B050ECE6F22
:1080E8001CD0D00E0001C26FC90EE82EFED7C22FD9
:1080F800FCD700D092EC63F0215022100EE0000172
:10810800D06BD16BF30E9C6FFC0E9D6FCEC09EF0B2
:10811800CFC09FF0F0EC67F008D00001CE07D8A0E0
:10812800CF07CE29DEE1CF29DCE18EB808D0250EB5
:108138009C6FFF0E9D6FF0EC67F0D06BD16B92ECEB
:1081480063F02150221003E00001D06BD16B0001D5
:10815800D051D11101E01AD701015B6B839E839046
:108168001200838E8380516AA5EC41F001019B6F58
:108178009B5102E09B5112006C6B936B946B956B57
:10818800966B996B010E986F9E6BD0D09C6B9D6B14
:108198001CD092EC63F02150221015E09E0E0E6E5A
:1081A800010E0F6E3EEC5EF00101976F000E6C251C
:1081B800D96EDA6A040EDA2297C1DFFF6C2B9C4B6A
:1081C8009D2B9EBB05D08EAC03D001019D05E1E33C
:1081D80001019C5193279D519423000E95239623CA
:1081E80053501E0D170EF324D96E020EF420DA6ECA
:1081F800DE50935DDE509459DE509559DE50965905
:1082080002E3986B996B9EAB02D0986B996B8EBC0E
:1082180002D0986B996B9D0519E2000E6C250E6EC5
:108228000F6A040E0F22FF0E6C25D96EDA6A030E50
:10823800DA22DF50106E116A6C510008126E000EBF
:10824800D8A0E82A0108136EE5EC4CF00101625150
:1082580045E0385139113A113B1140E053503EE1A5
:1082680053501E0D070EF324D96E020EF420DA6E59
:1082780038C188F139C189F13AC18AF1876B000E9A
:1082880087258B6F010E88218C6F000E89218D6FD9
:10829800000E8A218E6F8F6B906B916B926BDE5004
:1082A8008B191CE1DE508C1919E1DE508D1916E18D
:1082B800DE508E1913E1DE508F1910E1DE5090194F
:1082C8000DE1DE5091190AE1DE50921907E1000E26
:1082D800256E040E266E62516EEC5DF0DDEC51F0F9
:1082E80001019A6F6C6B9A5121E0370E00019C6F67
:1082F800FB0E9D6F9AC19EF09F6BF0EC67F0010E2C
:10830800516E53501E0D1B0EF324D96E020EF4202D
:10831800DA6E53501E0D1B0EF324E16E020EF4208C
:10832800E26EE7500409DF6E51501200985199111E
:1083380001E02CD78FA402D0010E516E8390839E4A
:10834800000C53501E0D070EF324D96E020EF420B4
:10835800DA6EDECFEBF0DECFECF0DECFEDF0DECF85
:10836800EEF053501E0D070EF324D96E020EF420C2
:10837800DA6E53501E0D0F0EF324E16E020EF42038
:10838800E26EDE50E65CDE50E658DE50E658DE501F
:10839800E658DE50E658DE50E658DE50E658DE5025
:1083A800E65815E2010E516E53501E0D1B0EF324B4
:1083B800D96E020EF420DA6E53501E0D1B0EF324F4
:1083C800E16E020EF420E26EE7500409DF6E5350AE
:1083D8001E0D070EF324D96E020EF420DA6EDECFDE
:1083E800C7F0DECFC8F0DECFC9F0DECFCAF0DECFEF
:1083F800CBF0DECFCCF0DECFCDF0DECFCEF05350D9
:108408001E0D170EF324D96E020EF420DA6EDECF9D
:10841800CFF0DECFD0F0DECFD1F0DECFD2F000014A
:10842800CF51D36FD051D46FD151D56FD251D66FB0
:10843800D76BD86BD96BDA6BC751D325DB6FC851B3
:10844800D421DC6FC951D521DD6FCA51D621DE6F29
:10845800CB51D721DF6FCC51D821E06FCD51D92135
:10846800E16FCE51DA21E26F53501E0D0F0EF32447
:10847800D96E020EF420DA6EDB51DE5CDC51DE5878
:10848800DD51DE58DE51DE58DF51DE58E051DE584E
:10849800E151DE58E251DE5815E2010E516E53509B
:1084A8001E0D1B0EF324D96E020EF420DA6E535003
:1084B8001E0D1B0EF324E16E020EF420E26EE7504F
:1084C8000409DF6E516A5350220D000EF3249E6F8B
:1084D800030EF4209F6FEBC0A0F0ECC0A1F0EDC03C
:1084E800A2F0EEC0A3F0B0EC12F0EF6FEF5115E080
:1084F800010E516E53501E0D1B0EF324D96E020E41
:10850800F420DA6E53501E0D1B0EF324E16E020E9A
:10851800F420E26EE7500409DF6E515012008EA677
:1085280004D0940E216EFE0E03D0B80E216EFF0EFD
:10853800226E8EAA04D0940E236EFE0E03D0B30EC4
:10854800236EFF0E246E8EA804D0940E256EFE0EA8
:1085580003D0C10E256EFE0E266E8EAE04D0940E8C
:10856800276EFE0E03D0BD0E276EFF0E286E8EAC52
:1085780004D0940E296EFE0E03D0AE0E296EFF0EA7
:108588002A6E8EA404D0940E2B6EFE0E03D0C70E56
:108598002B6EFF0E2C6E8EA204D0940E2D6EFE0E46
:1085A80003D0CC0E2D6EFF0E2E6E8EA004D0940E2E
:1085B8002F6EFE0E03D0C20E2F6EFF0E306E90AEE1
:1085C80004D0940E316EFE0E03D0FA0E316EFF0EFB
:1085D800326E90AC04D0940E336EFE0E03D0F70EBC
:1085E800336EFF0E346E90AA04D0940E356EFE0ED4
:1085F80003D0F40E356EFF0E366E90A804D0940E9C
:10860800376EFE0E03D0F10E376EFF0E386E90A651
:1086180004D0940E396EFE0E03D0EE0E396EFF0EA6
:108628003A6E90A404D0940E3B6EFE0E03D0EB0E6F
:108638003B6EFF0E3C6E90A204D0940E3D6EFE0E73
:1086480003D0E80E3D6EFF0E3E6E90A004D0940E4F
:108658003F6EFE0E03D0E50E3F6EFF0E406EBA0E63
:1086680000019C6FF80E9D6F901C9E6F9F6B8ECFC4
:10867800A0F0A16B3FC0A2F040C0A3F03DC0A4F0A1
:108688003EC0A5F03BC0A6F03CC0A7F039C0A8F09A
:108698003AC0A9F037C0AAF038C0ABF035C0ACF08A
:1086A80036C0ADF033C0AEF034C0AFF031C0B0F07A
:1086B80032C0B1F02FC0B2F030C0B3F02DC0B4F06A
:1086C8002EC0B5F02BC0B6F02CC0B7F029C0B8F05A
:1086D8002AC0B9F027C0BAF028C0BBF025C0BCF04A
:1086E80026C0BDF023C0BEF024C0BFF021C0C0F03A
:1086F80022C0C1F0F0EF67F0070E0E241D6E000EC9
:108708000F201E6E0EC0D9FF0FC0DAFFDF50126EA9
:1087180012380F0B0A0DF3CF13F0F4CF14F00EC07C
:10872800D9FF0FC0DAFFDF500F0B1326000E1422FB
:1087380013281B6E000E14201C6E206A010E1F6E7B
:10874800216A226A236A246AB2D01F50201054E09A
:1087580021C012F022C013F023C014F024C015F079
:108768000A0E1202F3CF16F0F4CF17F0186A196A3E
:108778001302F3501726F4501822000E1922120281
:10878800F3501726F4501822000E19220A0E14026C
:10879800F3501826F4501922000E1302F35018262D
:1087A800F4501922000E1202F3501826F450192220
:1087B8000A0E1502F3501926000E1402F35019265A
:1087C800000E1302F3501926000E1202F350192658
:1087D8001DC0D9FF1EC0DAFFDF501A6E1A380F0B02
:1087E8001624216E000E1720226E000E1820236E0C
:1087F800000E1920246E54D021C012F022C013F0AC
:1088080023C014F024C015F00A0E1202F3CF16F09C
:10881800F4CF17F0186A196A1302F3501726F450A8
:108828001822000E19221202F3501726F4501822AB
:10883800000E19220A0E1402F3501826F4501922B9
:10884800000E1302F3501826F4501922000E1202DB
:10885800F3501826F45019220A0E1502F35019265F
:10886800000E1402F3501926000E1302F3501926B5
:10887800000E1202F35019261DC0D9FF1EC0DAFFE0
:10888800DF500F0B1624216E000E1720226E000EEB
:108898001820236E000E1920246E1D06D8A01E066F
:1088A8001F502010010ED8A4000E1F6E206A1B0650
:1088B800D8A01C061B2802E11C28D8A446D721C032
:1088C8000EF022C00FF023C010F024C011F01200E7
:1088D80046C027F047C028F07AEC48F0486E485068
:1088E80001E0D4D046C0D9FF47C0DAFF030EDE1836
:1088F80001E0BCD020EE04F04650D9264750DA22D9
:10890800DE0401E0B3D02F0E46240E6E000E472081
:108918000F6E116A106A020E136E126A5AEC67F033
:108928002D0E46240E6E020E47200F6EAA0E116EF3
:10893800550E106E20EC67F02F0E46240E6E000EBA
:1089480047200F6E520E106E116E610E126E410EA0
:10895800136E04EC61F0130E46240E6E020E4720CF
:108968000F6E720E106E116E410E126E610E136E46
:1089780004EC61F0170E46240E6E020E47200F6EAF
:1089880020EE0FF04650D9264750DA22DECF10F0FD
:10899800DECF11F0DECF12F0DECF13F004EC61F081
:1089A8001B0E46240E6E020E47200F6E20EE0BF0B3
:1089B8004650D9264750DA22DECF10F0DECF11F02C
:1089C800DECF12F0DECF13F004EC61F020EE1BF0E6
:1089D8004650D9264750DA22DECF60F0DECF61F06C
:1089E800DECF62F0DECF63F0010E00016025646F18
:1089F800000E6121656F000E6221666F000E632113
:108A0800676F20EE2BF04650D9264750DA2264C013
:108A1800DEFF65C0DEFF66C0DEFF67C0DEFF2F0E2B
:108A280046241D6E000E47201E6E20EE2BF0465089
:108A3800D9264750DA22DECF1FF0DECF20F0DECF76
:108A480021F0DECF22F0246A010E236E20EE01F021
:108A58004650D9264750DA22DF50BCEC56F020EEBB
:108A680004F04650D9264750DA22DF6A1D6A1E6A8A
:108A78001F6A20EE01F04650D9264750DA22DF500F
:108A88006BEC26F0000902E0010E486E4850120017
:108A98006251D8B41200230E00019C6FFD0E9D6F29
:108AA800F0EC67F07EEC5AF021C07DF122C07EF137
:108AB80023C07FF124C080F101017D517E117F1117
:108AC800801117E1DB0E00019C6FFB0E9D6F7DC1CD
:108AD8009EF07EC19FF07FC1A0F080C1A1F0F0ECB4
:108AE80067F00A0E116E000E126A136A146A7CECA3
:108AF80062F00101816B826BE10E00019C6FFF0E39
:108B08009D6F7D0E01018125D96E010E8221DA6EDD
:108B1800DF5000019E6F9F6BF0EC67F00101814B05
:108B2800822B82BFE9D7825103E1040E815DE4E321
:108B3800340E00019C6FF90E9D6FF0EC67F0B90ED2
:108B48009C6FFA0E9D6FF0EC67F023EE00F000EEDC
:108B5800C7F0210EDBCFEBFFE806FCE2D50EE96F8C
:108B6800FF0EEA6F08EC3AF0C7C038F1C8C039F117
:108B7800C9C03AF1CAC03BF10101385139113A1163
:108B88003B11D8B412009F0E00019C6FFA0E9D6F26
:108B980038C19EF039C19FF03AC1A0F03BC1A1F0A5
:108BA800F0EC67F0000E9E6F030E9F6F38C1F8F06F
:108BB80039C1F9F03AC1FAF0F76B000EF725A06F4A
:108BC800010EF821A16F000EF921A26F000EFA2103
:108BD800A36FB0EC12F00101686F000E0001746F12
:108BE800030E756F350E766F0B0E776F796B080E67
:108BF800786F7B0E7A6F010E7B6F66EC1DF00101BA
:108C0800686F836B846B9A0E00019C6FFC0E9D6FDE
:108C1800350E01018325D96E0B0E8421DA6EDF50E3
:108C280000019E6F9F6BF0EC67F00101834B842B72
:108C380084BFE9D7845105E1080E835DD8B01200DE
:108C4800E2D71200C0C0D9FFC1C0DAFFDECFCAF038
:108C5800DDCFCBF003D00001C24BC32BC2C0F6FF5F
:108C6800C3C0F7FF000EF86E0E0EF76403D00800BD
:108C7800F55005D0F6CFE9FFF7CFEAFFEF502F0AFE
:108C8800EAE0C2C0F6FFC3C0F7FF000EF86E0E0E92
:108C9800F76403D00800F55005D0F6CFE9FFF7CF09
:108CA800EAFFEF505C0AD7E0000120EE06F0C05161
:108CB800D926C151DA22DE6ADE6ADE6ADD6AC2C0FE
:108CC800F6FFC3C0F7FF000EF86E0E0EF76403D070
:108CD8000800F55005D0F6CFE9FFF7CFEAFFEF50CF
:108CE8000001C46F200EC46114D020EE27F0C051DB
:108CF800D926C151DA22800EDF6EC0C074F0C1C01F
:108D080075F0000E766F776F786F796F35EC37F006
:108D180023D0C0C016F0C1C017F0C20E186E38ECD0
:108D28003BF00001CD6FCD5158E1C0C0B8F0C1C0D3
:108D3800B9F07BEC4DF0CD6F20EE27F0C051D9266D
:108D4800C151DA22DF50CC6FCD5108E0040ECD19A5
:108D580044E1CCB542D0050ECD6F3FD0CCB53DD067
:108D680020EE04F0C051D926C151DA22DFA8F3D78A
:108D7800CAC015F0CBC016F0C469010EC56F20EE4D
:108D88000EF0C051D926C151DA22DECFC6F0DDCFB0
:108D9800C7F0C451C617C551C717CAC0C8F0CBC061
:108DA800C9F0C651C827C751C9232F0EC825176E49
:108DB800000EC921186EB3EC5FF0000120EE06F03A
:108DC800C051D926C151DA2215C0DEFF16C0DEFF18
:108DD80017C0DEFF18C0DEFF9CD7CD51120081C03E
:108DE800D9FF82C0DAFFDECF98F0DDCF99F0865147
:108DF8008511841104E1020E835DD8A0020C20EED7
:108E080013F09851D9269951DA22DE50835DDE504D
:108E18008459DE508559DE50865901E3020C87518A
:108E2800881189118A1117E098C060F099C061F023
:108E380087C062F088C063F089C064F08AC065F0BA
:108E480066696769686969694EEC24F0976F97519C
:108E580002E09751120081C045F082C046F083C0FD
:108E680047F084C048F085C049F086C04AF098ECC5
:108E780030F045C093F046C094F047C095F048C024
:108E880096F00001935194119511961170E0930595
:108E980094119511961101E1020C932907E1942987
:108EA80005E1952903E1962901E1010C98C060F0DC
:108EB80099C061F083C062F084C063F085C064F03B
:108EC80086C065F0666B676B686B696B4EEC24F067
:108ED800976F9751BEE120EE13F09851D92699511A
:108EE800DA22FE0EDE248B6FFF0EDE208C6FFF0E63
:108EF800DE208D6FFF0EDE208E6F20EE0FF0985172
:108F0800D9269951DA228B51DE5C8C51DE588D516D
:108F1800DE588E51DE5813E220EE0FF09851D92614
:108F28009951DA22DE2A000EDE22DE22DE2220EE2F
:108F380004F09851D9269951DA22000EDB8093C0AB
:108F480083F094C084F095C085F096C086F020EE3A
:108F580013F09851D9269951DA22DE50835DDE50FC
:108F68008459DE508559DE50865901E274D7000CC9
:108F78001E6E1E5001E0010C55A202D05550120081
:108F8800000E0CEC67F00A0E296E03D00CEC68F0AA
:108F980029062950FBE1266A000E176A186A196A21
:108FA8001A6A87EC65F0E80601E097D0AA0E176EFA
:108FB800010E186E196A1A6A080E87EC65F0E80641
:108FC80051E1296A29501F0FD96EDA6A0CEC68F052
:108FD800DF6E292A030E2964F5D721047EE1AA0E43
:108FE80022187BE1030E286EE80E276E15D0176A4B
:108FF800186A196A400E1A6EA90E87EC65F0000906
:109008000EE0150E1D6EC60EE82EFED71D2EFCD7DF
:1090180000D02706D8A0280627502810E8E12750B6
:1090280028105BE0176A186A196A1A6A3A0E87EC00
:1090380065F0000952E1296A29501F0FD96EDA6AD2
:109048000CEC68F0DF6E292A030E2964F5D71FBCE3
:1090580003D0246A040E02D0246A0C0E236E23C0A7
:1090680026F03BD0176A186A196A1A6AA90E87ECA3
:1090780065F01D6E020E1D6003D0266EA90E02D08B
:10908800010E266E256E030E286EE80E276E14D08C
:10909800176A186A196A1A6A255087EC65F0000978
:1090A8000EE0150E1D6EC60EE82EFED71D2EFCD73F
:1090B80000D02706D8A0280627502810E9E1275015
:1090C80028100AE0176A020E186E196A1A6A100E3A
:1090D80087EC65F0000901E0266A26C054F019EC17
:1090E80068F0265001E14AD7559048D7396A20EEF2
:1090F80003F02750D9262850DA22DF5001E1A7D003
:109108002F0E27241D6E000E28201E6E20EE2BF039
:109118002750D9262850DA22DECF1FF0DECF20F0E4
:10912800DECF21F0DECF22F0246A010E236E20EE7E
:1091380001F02750D9262850DA22DF50BCEC56F02F
:10914800000901E082D020EE03F02750D9262850EC
:10915800DA22DF6A20EE17F02750D9262850DA22C3
:1091680010EE1FF02750E1262850E222E6CF2DF01E
:10917800E6CF2EF0E6CF2FF0E6CF30F010EE2BF052
:109188002750E1262850E222E6CF31F0E6CF32F030
:10919800E6CF33F0E6CF34F02D50315C356E2E50EB
:1091A8003258366E2F503358376E30503458386E28
:1091B800DE50355CDE503658DE503758DE503858B1
:1091C80046E220EE02F02750D9262850DA22020E75
:1091D800DE183DE12F0E27241D6E000E28201E6E7E
:1091E80020EE17F02750D9262850DA22DECF29F0B2
:1091F800DECF2AF0DECF2BF0DECF2CF020EE2BF0E6
:109208002750D9262850DA22DECF2DF0DECF2EF0D7
:10921800DECF2FF0DECF30F029502D241F6E2A50DC
:109228002E20206E2B502F20216E2C503020226EA5
:10923800246A010E236E20EE01F02750D92628500B
:10924800DA22DF50BCEC56F002D0010E396E3950EC
:10925800120049C00FF04AC010F0690E116E82EC7E
:1092680059F00001686F685101E099D020EE0EF0C6
:109278004950D9264A50DA22DFAC91D069C03AF079
:109288006AC03BF020EE1CF04950D9264A50DA2239
:10929800DECF3CF0DECF3DF0DECF3EF0DECF3FF05C
:1092A8001BEC5BF00001686F685179E120EE20F05B
:1092B8004950D9264A50DA22DECF6BF0DDCF6CF068
:1092C80020EE0BF06B51D9266C51DA22000EDB8AA6
:1092D80049C0D9FF4AC0DAFFDECF12F0DDCF13F064
:1092E8006BC014F06CC015F020EE06F04950D9267A
:1092F8004A50DA22DECF16F0DECF17F0DECF18F0B4
:10930800DECF19F07BEC64F01C0E00016B250E6EAD
:10931800000E6C210F6E20EE0AF04950D9264A50F3
:10932800DA22DECF10F0DECF11F0DECF12F0DECF82
:1093380013F004EC61F0160E00016B250E6E000EA2
:109348006C210F6E106A116A210E126E500E136E88
:1093580004EC61F0120E00016B250E6E000E6C21FC
:109368000F6E000E116A106A20EC67F0000120EE03
:1093780003F06951D9266A51DA22010EDF6E69C0FD
:1093880046F06AC047F06CEC44F00001686F20EECC
:109398000EF04950D9264A50DA22BF0EDF1668511E
:1093A800120089688B68F29E8E280BE1060E000178
:1093B8009C6FFB0E9D6F8ECF9EF09F6BF0EC67F05D
:1093C8000AD0820E00019C6FF90E9D6F8ECF9EF021
:1093D8009F6BF0EC67F090280AE1C40E9C6FFB0EBF
:1093E8009D6F8ECF9EF09F6BF0EC67F009D0A70EB3
:1093F8009C6FF90E9D6F8ECF9EF09F6BF0EC67F01F
:10940800290E426E960E416E7F0EE82EFED7412E33
:10941800FCD7422EFAD700F04B0E00019C6FFE0ECF
:109428009D6FF0EC67F089988498090E426E1E0EC5
:10943800416EE40EE82EFED7412EFCD7422EFAD715
:1094480000D03E0E00019C6FFE0E9D6FF0EC67F0A1
:10945800899A849A090E426E1E0E416EE40EE82E19
:10946800FED7412EFCD7422EFAD700D0AF0E00010E
:109478009C6FFE0E9D6FF0EC67F088908D909028A1
:109488000AE0C40E9C6FFB0E9D6F90CF9EF09F6B01
:10949800F0EC67F009D0370E9C6FF90E9D6F90CFF6
:1094A8009EF09F6BF0EC67F08D80A30E426E570E16
:1094B800416E020EE82EFED7412EFCD7422EFAD777
:1094C80000D089688B688A6883928382290E426EED
:1094D800960E416E7F0EE82EFED7412EFCD7422E07
:1094E800FAD700F093EC42F0EFD71F6A1DAE12D006
:1094F8001D1E1C1E1B1E1A1E191E181E171E166C5A
:10950800000E1722182219221A221B221C221D22A1
:10951800010E1F6E15AE12D0151E141E131E121E3C
:10952800111E101E0F1E0E6C000E0F22102211228B
:109538001222132214221522010E1F1A206A216AF0
:10954800226A236A246A256A266A276A165017102F
:10955800181019101A101B101C101D1045E0010ED0
:109568001E6E0AD0D89016361736183619361A369F
:109578001B361C361D361E2A1DAEF4D7D890203651
:1095880021362236233624362536263627361650F7
:109598000E5C17500F5818501058195011581A507F
:1095A80012581B5013581C5014581D50155811E3CD
:1095B80016500E5E17500F5A1850105A1950115A5B
:1095C8001A50125A1B50135A1C50145A1D50155A2F
:1095D8002080D8901D321C321B321A3219321832B0
:1095E800173216321E2ECAD71F5010E0271E261E0D
:1095F800251E241E231E221E211E206C000E212241
:1096080022222322242225222622272220C00EF0CD
:1096180021C00FF022C010F023C011F024C012F0B6
:1096280025C013F026C014F027C015F012001768E3
:1096380018680E50D96EDA6ADECF19F0DDCF1AF04D
:1096480019C014F01AC015F019501A1003E10E6869
:109658000F68120014C0F6FF15C0F7FF000EF86E71
:109668000E0EF76403D00800F55005D0F6CFE9FFD9
:10967800F7CFEAFFEF50166E144A152A200E16642B
:1096880003D03A0E1618E6E13A0E161868E1000EF5
:10969800136E010E126E19C0F6FF1AC0F7FF000E06
:1096A800F86E0E0EF76403D00800F55005D0F6CF1B
:1096B800E9FFF7CFEAFFEF50106E2F0E106439D094
:1096C80019C0F6FF1AC0F7FF000EF86E0E0EF76409
:1096D80003D00800F55005D0F6CFE9FFF7CFEAFF31
:1096E800EF50106E3A0E106024D0020E1924106E3E
:1096F800000E1A20116E145010181BE11550111885
:1097080018E119C0F6FF1AC0F7FF000EF86E0E0E2A
:10971800F76403D00800F55005D0F6CFE9FFF7CF7E
:10972800EAFFEF50106ED00E1024126E136AFF0E6F
:10973800132213BE04D013500DE112040BE212C021
:1097480017F013C018F00E50D96EDA6A14C0DEFF95
:1097580015C0DDFF17C00EF018C00FF012000E6A1A
:109768000F6A120060C045F061C046F0476A486A57
:10977800496A4A6A63EC54F045C078F046C079F00B
:10978800020E0001781979110DE0795106E1030EF6
:10979800785D03E26251631105E178C060F079C039
:1097A80061F012007A6B7B6B7AC064F07BC065F065
:1097B800643B653BF00E651764510F0B6513F00EA3
:1097C800641760C066F061C067F064516627655130
:1097D8006723F50E66250E6E010E67210F6ED8EC15
:1097E80059F000017A51040DF350680FD96EDA6A06
:1097F8000EC0DEFF0FC0DEFF10C0DEFF11C0DEFFAF
:109808007A4B7B2B7B5103E1040E7A5DCDE36251E9
:10981800631103E17A6B7B6B06D0FF0E62257A6FCA
:10982800FF0E63217B6F7A51040DF350680FD96ED8
:10983800DA6ADE50DE10DE10DE1004E1796B030E0A
:10984800786F18D060C045F061C046F07A51040DB9
:10985800F350680FD96EDA6ADECF47F0DECF48F0F2
:10986800DECF49F0DECF4AF063EC54F045C078F023
:1098780046C079F00001625163118FE1795103E12B
:10988800020E785D8AE37A4B7B2B7B5186E1040ECE
:109898007A5D83E2C8D72F6C696664617461302E83
:1098A80062696E20002F6C696664617461312E6292
:1098B800696E20002F6C696664617461322E62697A
:1098C8006E20002F6C696664617461332E62696E64
:1098D80020002F6C696664617461342E62696E20A1
:1098E800002F6C696664617461352E62696E2000B0
:1098F8002F6C696664617461362E62696E20002F70
:109908006C696664617461372E62696E20002F6C21
:10991800696664617461382E62696E20002F6C6913
:109928006664617461392E62696E20002F6C696605
:1099380064617461612E62696E20002F6C696664CF
:10994800617461622E62696E20002F6C69666461C1
:109958007461632E62696E20002F6C69666461749D
:1099680061642E62696E20002F6C6966646174619F
:10997800652E62696E20002F6C6966646174616689
:109988002E62696E20000000000000000000000048
:1099980000000000000000000000000000000000BF
:1099A80000000000000000000000000000000000AF
:1099B800000000000000000000000000000000009F
:1099C80000000EC018F00FC019F01250131001E17A
:1099D800120018C0D9FF19C0DAFF10C0DFFF1250FB
:1099E8001824146E13501920156EFF0E1424D96E06
:1099F800FF0E1520DA6E10C0DFFF135004E1030ECE
:109A0800125C01E2120020EE01F01850D92619501C
:109A1800DA2210C0DFFF20EE02F01850D9261950C4
:109A2800DA2210C0DFFF12501824146E13501920C8
:109A3800156EFE0E1424D96EFF0E1520DA6E10C0B6
:109A4800DFFF12501824146E13501920156EFD0EE6
:109A58001424D96EFF0E1520DA6E10C0DFFF1350E4
:109A680004E1070E125C01E2120020EE03F0185028
:109A7800D9261950DA2210C0DFFF12501824146EAC
:109A880013501920156EFC0E1424D96EFF0E1520E4
:109A9800DA6E10C0DFFF135004E1090E125C01E218
:109AA800120018C014F019C015F0141E151E144A1F
:109AB800152A030E1414166E176A16501826175016
:109AC80019221650125E1750135AFC0E12160BD09C
:109AD80018C0D9FF19C0DAFF10C0DFFF1206D8A0DE
:109AE8001306184A192A12501310F2E11200B8C0CE
:109AF800D9FFB9C0DAFFDECFBCF0DDCFBDF0B8C00A
:109B080074F0B9C075F0000E766F776F786F796F63
:109B180035EC37F0BF6FBF5103E00001BF511200B1
:109B2800BCC03AF0BDC03BF020EE16F0B851D926C3
:109B3800B951DA22DECF3CF0DECF3DF0DECF3EF089
:109B4800DECF3FF01BEC5BF00001BF6FBF51E5E1DA
:109B580020EE1AF0B851D926B951DA22DECFBAF080
:109B6800DDCFBBF0BAC0D9FFBBC0DAFFDF50BE6F94
:109B7800BE5103E1040EBF6FD0D720EE04F0B851F8
:109B8800D926B951DA2210EE1AF0B851E126B951A6
:109B9800E22200EE0BF0E650E926E550EA22EF500B
:109BA8003F0BDF6E20EE1AF0B851D926B951DA22F0
:109BB80010EE0BF0DE50E126DD50E222E7B618D0B9
:109BC80020EE1AF0B851D926B951DA22DECF0EF0BC
:109BD800DDCF0FF01C0EB825106E000EB921116EE6
:109BE800136A0B0E126ECEEC60F00E500F1095E05B
:109BF800B8C09EF0B9C09FF00001A16BA06B12EC39
:109C080034F00001BF6FBF5188E18AD71BC00EF046
:109C18001CC00FF0116A106A136A080E126EE5EC88
:109C28004CF0266A020E256E25501B24D96E26504C
:109C38001C20DA6E25501B24216E26501C20226E13
:109C48002128E16E000E2220E26EE750236E233AAF
:109C5800F00E2316231625501B24E16E26501C20D7
:109C6800E26EE750246E24380F0B2310DF6E254A6E
:109C7800262A26BED9D7265003E1070E255CD4E351
:109C880025501B24D96E26501C20DA6E1DC00EF0FC
:109C98001EC00FF01FC010F020C011F00A0E126E87
:109CA800136A146A156A6DEC61F00E3AF00E0E161E
:109CB80025501B24E16E26501C20E26EE750216ED1
:109CC80021380F0B0E10DF6E1BC0D9FF1CC0DAFF46
:109CD800DF2A1DC00EF01EC00FF01FC010F020C0FC
:109CE80011F00A0E126E136A146A156A3EEC5FF0E0
:109CF8000EC01DF00FC01EF010C01FF011C020F0E4
:109D08001D501E101F1020108CE11BC0D9FF1CC055
:109D1800DAFFDF06090EDF64090C1BC0D9FF1CC07F
:109D2800DAFF100EDF6E100C000E0101AF6F0A0E85
:109D3800AE6F000EAD6F050EAC6F7DD00101AF6B3D
:109D4800140EAE6F70D0300E0F6EFC0E106E52EC0B
:109D580062F08FB204D00101AF6B1E0EAE6F090E18
:109D68000001FE6F1E0EFD6FE40EE82EFED7FD2FDC
:109D7800FCD7FE2FFAD700F056D0970E0F6EFE0EC6
:109D8800106E52EC62F0060E0001B16F090EB26F50
:109D9800360EB36FF90EB46FB56BDFEC5CF00101F2
:109DA800686F6851CEEC62F001016851D8E1AF6B81
:109DB800230ED4D7DC0E0F6EFD0E106E52EC62F03F
:109DC800000E0001CE6F030ECF6FE50ED06F010EAF
:109DD800D16F010ED26F7EEC15F00101686F6851EA
:109DE800CEEC62F0010168510AE19CEC2CF0000E07
:109DF8006D6F030E6E6F15EC65F00101686F6851A9
:109E0800CEEC62F0010CAEC1FDF0AFC1FEF0000176
:109E1800FE5109E1FD510A0A91E01E0A94E00A0A7E
:109E2800ACE03D0AC7E0140E0101AE19AF1103E022
:109E3800AC07D8A0AD07ADBF000CAD51E4E1AC054F
:109E4800E2E2000C1F6A15AE12D0151E141E131E76
:109E5800121E111E101E0F1E0E6C000E0F22102255
:109E680011221222132214221522010E1F6E1DAE7A
:109E780010D01D1E1C1E1B1E1A1E191E181E171E72
:109E8800166C000E1722182219221A221B221C22D5
:109E98001D2216501710181019101A101B101C101C
:109EA8001D103BE0010E1E6E0AD0D89016361736EC
:109EB800183619361A361B361C361D361E2A1DAEA4
:109EC800F4D716500E5C17500F58185010581950E8
:109ED80011581A5012581B5013581C5014581D5022
:109EE800155810E316500E5E17500F5A1850105A96
:109EF8001950115A1A50125A1B50135A1C50145AFE
:109F08001D50155AD8901D321C321B321A32193284
:109F18001832173216321E2ED4D71F5010E0151ED5
:109F2800141E131E121E111E101E0F1E0E6C000E84
:109F38000F221022112212221322142215220EC0DF
:109F48000EF00FC00FF010C010F011C011F012C0C9
:109F580012F013C013F014C014F015C015F012005D
:109F68002968820E9C6FFD0E9D6F4EC09EF04FC0FB
:109F78009FF04AC1A0F04BC1A1F0F0EC67F08380DC
:109F880003D02D0EE5EC67F08EA88EAA03D0290623
:109F98002928F7E153501E0D070EF324D96E020E3F
:109FA800F420DA6EDECF21F0DECF22F0DECF23F010
:109FB800DECF24F0DECF25F0DECF26F0DECF27F08F
:109FC800DECF28F021C00FF022C010F023C011F01E
:109FD80024C012F025C013F026C014F027C015F0D5
:109FE80028C016F0CDEC5AF00D0EE5EC67F00A0E1D
:109FF800E5EC67F0010152514A1903E153514B193D
:10A0080003E05251531112E0889C10D0030E0AD07D
:10A01800050E2A6E4E6A4F6A2ED00A0E03D0010E24
:10A0280001D0020E2A6E27D02A6A25D04EC021F010
:10A038004FC022F0225009E0020A0EE00E0A10E09A
:10A04800010A12E02A0A14E0EFD72150DFE00A0AD9
:10A05800DDE01E0ADDE0E8D72150BC0AE2E0E4D7E3
:10A0680021501C0ADAE0E0D72150AC0AD8E0DCD74E
:10A0780021500F0AD9E12A501200FAC123F079D0F1
:10A088006DEC67F0236EFA1901E182D0290E226E79
:10A09800960E216E7F0EE82EFED7212EFCD7222E9B
:10A0A800FAD700F075D06DEC63F0246E245070E0A0
:10A0B80024A002D00101612B24A202D00101610772
:10A0C8000F0E01016117000E0E6EC00E1FEC63F03B
:10A0D800F7EC66F0000E0E6EC00E1FEC63F0010187
:10A0E80061510F0D350EF324126E0D0EF420136E10
:10A0F80001EC5FF0110E226E3C0E216ECB0EE82EA5
:10A10800FED7212EFCD7222EFAD700F024A440D067
:10A118000F6A0E6A61C110F032EC65F01C0E000186
:10A128009C6FFC0E9D6F61C19EF09F6BF0EC67F019
:10A1380061C123F0000E0E6E800E1FEC63F0F7EC89
:10A1480066F0000E0E6E800E1FEC63F00101615187
:10A158000F0D350EF324126E0D0EF420136E01EC64
:10A168005FF0000E0E6EC00E1FEC63F0F7EC66F0A9
:10A178000FD001016451216E226A225009E1215059
:10A18800010A01E17DD7030A01E17AD7010A8BE0D0
:10A1980023501200020E105E000E115A125A135A62
:10A1A80020EE13F00E50D9260F50DA22FE0EDE24D0
:10A1B800146EFF0EDE20156EFF0EDE20166EFF0EEB
:10A1C800DE20176E1450105C155011581650125896
:10A1D8001750135805E30E6A0F6A106A116A1200C5
:10A1E80020EE27F00E50D9260F50DA22DECF14F0D9
:10A1F800DECF15F0DECF16F0DECF17F020EE09F037
:10A208000E50D9260F50DA22DECF18F0DDCF19F024
:10A2180018501A6E19501B6E1C6A1D6A1A501002CB
:10A22800F3CF1EF0F4CF1FF0206A216A1102F35019
:10A238001F26F4502022000E21221B501002F3503A
:10A248001F26F4502022000E21221A501202F35029
:10A258002026F45021221B501102F3502026F450DE
:10A2680021221C501002F3502026F45021221350B2
:10A278001A02F35021261B501202F35021261C50BB
:10A288001102F35021261D501002F35021261450BC
:10A298001E240E6E15501F200F6E16502020106EB3
:10A2A80017502120116E1200838E83800001FB6BF2
:10A2B800FC6BC4EC5EF025C0FDF026C0FEF0040E79
:10A2C8000001FE5D07E3000EFD25FB6FFC0EFE217D
:10A2D800FC6F04D0FDC0FBF0FEC0FCF00101625130
:10A2E80033E0385139113A113B112EE053500C0D1F
:10A2F800040EF324D96E010EF420DA6E38C172F11F
:10A3080039C173F13AC174F1716B000E7125756F23
:10A31800010E7221766F000E7321776F000E742183
:10A32800786FDE50751910E1DE5076190DE1DE50B8
:10A3380077190AE1DE50781907E1000E256E040E40
:10A34800266E62516EEC5DF08FB415D05350220D1D
:10A35800000EF32400019E6F030EF4209F6F000E81
:10A36800A06F040EA16F010EA36FA26BFB0EA46F6A
:10A3780033EC0CF0FA6F0001FA5109E0130E9C6FF0
:10A38800FD0E9D6FFAC09EF09F6BF0EC67F09DECA0
:10A398002EF05B6B8390839E7C0E00019C6FFC0EFD
:10A3A8009D6FCECF9EF09F6BCDCFA0F0A16BF0EF4D
:10A3B80067F053501E0D070EF324D96E020EF420D9
:10A3C800DA6EDECF6DF1DECF6EF1DECF6FF1DECF6C
:10A3D80070F1DECF71F1DECF72F1DECF73F1DECF37
:10A3E80074F16DC10EF06EC10FF06FC110F070C145
:10A3F80011F071C112F072C113F073C114F074C17D
:10A4080015F053501E0D1C0EF324D96E020EF420C5
:10A41800DA6EDECF75F1DDCF76F175C116F076C153
:10A4280017F0186A196A1A6A1B6A1C6A1D6A06EC10
:10A4380058F00EC077F10FC078F110C079F111C053
:10A448007AF112C07BF113C07CF114C07DF115C004
:10A458007EF177C1F0F078C1F1F079C1F2F07AC1FC
:10A46800F3F0A5EC41F0F66FF65102E0F651120058
:10A478008FB414D05350220D000EF3249E6F030E98
:10A48800F4209F6F000EA06F040EA16F010EA36F42
:10A49800A26BF40EA46F33EC0CF0F76FF7510BE0DE
:10A4A800130E9C6FFD0E9D6FF7C09EF09F6BF0EC36
:10A4B80067F0F7511200E5EC53F0000C3AC027F0B2
:10A4C8003BC028F07AEC48F0000901E0010C3AC0E2
:10A4D8000EF03BC00FF03CC010F03DC011F03EC084
:10A4E80012F03FC013F0CEEC50F00EC044F00FC095
:10A4F80045F010C046F011C047F020EE2BF03A505E
:10A50800D9263B50DA2244C0DEFF45C0DEFF46C0F4
:10A51800DEFF47C0DEFF2F0E3A240E6E000E3B20F2
:10A528000F6E116A106A020E136E126A5AEC67F007
:10A538002F0E3A24426E000E3B20436E496A010EEC
:10A54800486E4A6A4B6A04D048504A2649504B2202
:10A5580020EE09F03A50D9263B50DA22DE504A5C08
:10A56800DE504B581FE242C01DF043C01EF04A5057
:10A5780044241F6E4B504520206E000E4620216E4D
:10A58800000E4720226E48C023F049C024F020EE78
:10A5980001F03A50D9263B50DA22DF50BCEC56F095
:10A5A8000009D2E020EE09F03A50D9263B50DA22D1
:10A5B8004A50DE1803E14B50DE18D8A4010C000CF9
:10A5C800226A236A1B6A1C6A01D0152A010E216EB1
:10A5D8001550D96EDA6A200EDE1813E0F70E176EE2
:10A5E80018681550D96EDA6ADF50196E1A6A175052
:10A5F800192618501A221A5003E1050E195C01E3B6
:10A60800216A21C01DF01E6A1D501E1006E0DDD70C
:10A618001C6A010E1B6E152A25D01550D96EDA6AF0
:10A62800DF50176E186A18501DE117502B0AF3E017
:10A63800060AEEE017D00A0E2202F3CF17F0F4CF85
:10A6480018F02302F35018261550D96EDA6ADF5035
:10A65800175E000E185A300E1724226E000E1820AE
:10A66800236ED9D7D00E176E18681550D96EDA6ACE
:10A67800DF50196E1A6A1750192618501A221A50E4
:10A6880005E10A0E195C02E2010E01D0000E1F6EF0
:10A69800206A1F502010CFE11B501C100DE122C072
:10A6A80017F023C018F0171E181E174A182A17C0CB
:10A6B80015F018C016F0120022C015F023C016F0CD
:10A6C8001200818E819C9E0EF66E980EF76E000E1B
:10A6D800F86E0DEE35F011EE2CF00900F5CFEEFF17
:10A6E800E550E150FAE1E250F8E18E0EF66EC60E42
:10A6F800F76E000EF86E03EEAAF010EE4CF00900AB
:10A70800F5CFEEFFE550E150FAE1E80EF66ECB0E1C
:10A71800F76E000EF86E02EE98F010EE34F00900B5
:10A72800F5CFEEFFE550E150FAE1740EF66EC90E72
:10A73800F76E000EF86E01EEBDF010EE3DF0090068
:10A74800F5CFEEFFE550E150FAE1560EF66ED00E69
:10A75800F76E000EF86E0900F5CF55F005EE00F023
:10A7680018EE35F0EE6AE550E150FCE1E250FAE10E
:10A7780004EE00F011EE00F0EE6AE550E150FCE165
:10A78800E250FAE103EE00F0AA0EEE6AE806FDE1F7
:10A7980002EE00F0980EEE6AE806FDE101EE00F028
:10A7A8006D0EEE6AE806FDE100EE4CF0090EEE6A69
:10A7B800E806FDE156905692000EF86E000172EF21
:10A7C8000FF053501E0D070EF324D96E020EF4201D
:10A7D800DA6EDECFC7F0DECFC8F0DECFC9F0DECF4D
:10A7E800CAF0DECFCBF0DECFCCF0DECFCDF0DECFBF
:10A7F800CEF053501E0D1C0EF324D96E020EF42019
:10A80800DA6EDECFCFF0DDCFD0F0CF51C725D16FD4
:10A81800D051C821D26F000EC921D36F000ECA21B2
:10A82800D46F000ECB21D56F000ECC21D66F000E51
:10A83800CD21D76F000ECE21D86F53501E0D070EB5
:10A84800F324D96E020EF420DA6ED1C0DEFFD2C036
:10A85800DEFFD3C0DEFFD4C0DEFFD5C0DEFFD6C02A
:10A86800DEFFD7C0DEFFD8C0DEFF53501E0D070E37
:10A87800F324D96E020EF420DA6EDECFD9F0DECFE3
:10A88800DAF0DECFDBF0DECFDCF05350220D000E25
:10A89800F3249E6F030EF4209F6FD9C0A0F0DAC096
:10A8A800A1F0DBC0A2F0DCC0A3F0B0EC12F0DD6FC9
:10A8B800DD5103E0010E516E010C516A120020EEC9
:10A8C80003F04550D9264650DA22DF6A20EE2BF0F5
:10A8D8004550D9264650DA22DE68DE68DE68DD6833
:10A8E80045C03AF046C03BF047C03CF048C03DF098
:10A8F80049C03EF04AC03FF01BEC5BF0000904E0A1
:10A90800466A040E456E040C2D0E45240E6E020E8A
:10A9180046200F6E0EEC66F0550E0E1803E1AA0ED7
:10A928000F1804E0466A030E456E030C20EE2FF064
:10A938004550D9264650DA22E90EDE1812E020EEFC
:10A948002FF04550D9264650DA22EB0EDE1809E0E2
:10A9580020EE2FF04550D9264650DA22E80EDE18B0
:10A9680027E1650E45240E6E000E46200F6ED10EAF
:10A97800106EFF0E116E136A030E126ECEEC60F0AD
:10A988000E500F1003E1456A466A1200810E4524F5
:10A998000E6E000E46200F6E850E106EFF0E116EA5
:10A9A800136A050E126ECEEC60F00E500F10EBE03D
:10A9B800466A020E456E020C256A286A8380850E57
:10A9C80000019C6FFA0E9D6FCECF9EF09F6BCDCF8E
:10A9D800A0F0A16BF0EC67F019D0270E0E6E0F6A8D
:10A9E8003EEC5EF0266E1B0E00019C6FFF0E9D6F05
:10A9F800252A25C09EF09F6B26C0A0F0A16BF0EC25
:10AA080067F027AA03D026C028F005D092EC63F09F
:10AA180021502210E2E1030E00019C6FFD0E9D6F94
:10AA280028C09EF09F6BF0EC67F0020E28183CE1FE
:10AA38005350130DAE0EF324D96E030EF420DA6EC4
:10AA4800020EDF6E5350130DBA0EF324D96E030EA7
:10AA5800F420DA6E080EDF6E53500D0D9A0EF324B3
:10AA6800D96E020EF420DA6E4C0EDF6E53500D0DC7
:10AA78009D0EF324D96E020EF420DA6E080EDF6EF6
:10AA880053500D0DA20EF324D96E020EF420DA6E87
:10AA9800050EDF6E53500D0DA30EF324D96E020E72
:10AAA800F420DA6E690EDF6E516A839012002F6E01
:10AAB8006A0E00019C6FFC0E9D6F2FC09EF09F6B6D
:10AAC8002BC0A0F02CC0A1F0F0EC67F05DD07EECBC
:10AAD8005AF021C030F022C031F023C032F024C037
:10AAE80033F02BC0D9FF2CC0DAFFDF6A20EE01F06B
:10AAF8002B50D9262C50DA2233C0DFFF20EE02F08B
:10AB08002B50D9262C50DA22DF6A20EE03F02B5086
:10AB1800D9262C50DA2232C0DFFF20EE04F02B5069
:10AB2800D9262C50DA22DF6A20EE05F02B50D926E0
:10AB38002C50DA2231C0DFFF20EE06F02B50D92648
:10AB48002C50DA22DF6A20EE07F02B50D9262C5041
:10AB5800DA2230C0DFFF12007EEC5AF021C030F05C
:10AB680022C031F023C032F024C033F02BC01BF0D8
:10AB78002CC01CF030C01DF031C01EF032C01FF0D8
:10AB880033C020F00AEF4EF02F502D6E2E6A2E5053
:10AB9800D8A412002D50010A9AE0030ADDE0120041
:10ABA8000001FC6B8380838E6AD0C4EC5EF025C004
:10ABB800FAF026C0FBF0040E0001FB5D03E3010E72
:10ABC800FC6F03D0FFC0FDF0FE6B8FB414D0535060
:10ABD800220D000EF3249E6F030EF4209F6F000ECB
:10ABE800A06F040EA16F010EA36FA26BFD0EA46FE0
:10ABF80033EC0CF0FF6FFF5109E0130E9C6FFD0E54
:10AC08009D6FFFC09EF09F6BF0EC67F001016251F1
:10AC180033E0385139113A113B112EE053500C0DE5
:10AC2800040EF324D96E010EF420DA6E38C172F1E5
:10AC380039C173F13AC174F1716B000E7125756FEA
:10AC4800010E7221766F000E7321776F000E74214A
:10AC5800786FDE50751910E1DE5076190DE1DE507F
:10AC680077190AE1DE50781907E1000E256E040E07
:10AC7800266E62516EEC5DF09DEC2EF05B6B000170
:10AC8800FC5193E0839E839012000F015969116B68
:10AC9800196B216B8C948C928C90889A110E136E80
:10ACA8003C0E126ECB0EE82EFED7122EFCD7132EBA
:10ACB800FAD700F0110E136E3C0E126ECB0EE82E72
:10ACC800FED7122EFCD7132EFAD700F0020E136E01
:10ACD800A00E126E920EE82EFED7122EFCD7132E5F
:10ACE800FAD700D0000E0E6E300E1FEC63F02A0E5D
:10ACF800126E8E0EE82EFED7122EFCD7000E0E6EA8
:10AD0800300E1FEC63F0000E0E6E300E1FEC63F079
:10AD1800000E0E6E390E1FEC63F0000E0E6E140E50
:10AD28001FEC63F0000E0E6E560E1FEC63F0000E63
:10AD38000E6E6D0E1FEC63F0000E0E6E700E1FECA3
:10AD480063F0000E0E6E0C0E1FEC63F0000E0E6E1C
:10AD5800060E1FEC63F0000E0E6E010E1FEC63F082
:10AD6800D00E126ECA0EE82EFED7122EFCD7120095
:10AD7800266E2650D8A4040C2350241001E1040C9C
:10AD880055B0030C55B4020C54B608D0090ED8902F
:10AD98001F36203621362236E82EF9D72304241010
:10ADA8001AE11FC017F020C018F021C019F022C006
:10ADB8001AF0180E87EC65F0000945E11DC010F087
:10ADC8001EC011F0FE0E126E28EC62F000093BE086
:10ADD800236A246A38D054C025F0060E251609E0E7
:10ADE80023C017F024C018F0196A1A6A970E87EC66
:10ADF80065F01FC017F020C018F021C019F022C05C
:10AE08001AF0190E87EC65F000091DE11DC010F05D
:10AE18001EC011F0FC0E126E28EC62F0000908E06A
:10AE2800020E1E262306D8A0240623502410EEE185
:10AE3800106A116AFD0E126E28EC62F0000903E137
:10AE4800246A010E236E19EC68F023502410D8A44C
:10AE5800010C000CB8C0D9FFB9C0DAFFDECFBFF0D3
:10AE6800DDCFC0F0B8C074F0B9C075F0000E766FD1
:10AE7800776F786F796F35EC37F0C36FC35153E153
:10AE8800C16BC26BBFC03AF0C0C03BF020EE16F0F9
:10AE9800B851D926B951DA22DECF3CF0DECF3DF0E9
:10AEA800DECF3EF0DECF3FF01BEC5BF00001C36F5E
:10AEB800C35139E120EE1AF0B851D926B951DA2236
:10AEC800DECFBCF0DDCFBDF0BCC0D9FFBDC0DAFF1E
:10AED800E50EDE1810E020EE1AF0B851D926B95167
:10AEE800DA22DECFBCF0DDCFBDF0BCC0D9FFBDC0DB
:10AEF800DAFFDF5009E1C14BC22BBA51C11906E193
:10AF0800BB51C21910E002D0C16BC26BB8C09EF031
:10AF1800B9C09FF0A16B010EA06F12EC34F00001D4
:10AF2800C36FC351AFE0040EC31902E1070EC36F2C
:10AF3800C3511200838E83800001D16BD26BD36B17
:10AF4800D46B5350220D000EF324746F030EF420BB
:10AF5800756F350E766F0B0E776F010E796F786B04
:10AF6800D50E7A6F7B6B66EC1DF0D06F01016251D4
:10AF780035E0385139113A113B1130E053500C0D7E
:10AF8800040EF324D96E010EF420DA6E38C1C7F02E
:10AF980039C1C8F03AC1C9F00001C66B000EC62518
:10AFA800CA6F010EC721CB6F000EC821CC6F000EEF
:10AFB800C921CD6FDE50CA1911E1DE50CB190EE15F
:10AFC800DE50CC190BE1DE50CD1908E1350E2B6EA1
:10AFD8000B0E2C6E010162515BEC55F002920001E0
:10AFE800D551FBEC5DF00001CE6FCF6BCE51D12770
:10AFF800CF51D223000ED323D42301015B6B839E50
:10B00800839012001E6A1F6A206A216A226A236AD4
:10B01800246A256A16501710181019101A101B10D8
:10B028001C101D1045E0010E266E0AD0D890163669
:10B038001736183619361A361B361C361D36262A88
:10B048001DAEF4D7D8901E361F362036213622364C
:10B0580023362436253616500E5C17500F581850D4
:10B068001058195011581A5012581B5013581C5088
:10B0780014581D50155811E316500E5E17500F5AEC
:10B088001850105A1950115A1A50125A1B50135A64
:10B098001C50145A1D50155A1E80D8901D321C324F
:10B0A8001B321A321932183217321632262ECAD7E4
:10B0B8001EC00EF01FC00FF020C010F021C011F00C
:10B0C80022C012F023C013F024C014F025C015F0DC
:10B0D8001200C4C0D9FFC5C0DAFFDECFC6F0DDCF8D
:10B0E800C7F0C4C0B8F0C5C0B9F0000EBB6F010E00
:10B0F800BA6F2EEC57F0C86FC85147E1C6C03AF096
:10B10800C7C03BF020EE16F0C451D926C551DA224B
:10B11800DECF3CF0DECF3DF0DECF3EF0DECF3FF0BD
:10B128001BEC5BF00001C86FC8512FE120EE1AF04C
:10B13800C451D926C551DA22DECF0EF0DDCF0FF08B
:10B14800116A106A136A200E126E5AEC67F0000139
:10B1580020EE1AF0C451D926C551DA22DECF0EF0FE
:10B16800DDCF0FF01C0EC425106E000EC521116E28
:10B17800136A0B0E126E1AEC64F020EE03F0C6513F
:10B18800D926C751DA22010EDF6EC851120001011B
:10B198005C6B506A486B496B020E5B6F83905A6B0D
:10B1A800596B536A030E536401D049D053500C0DA8
:10B1B800030EF324D96E010EF420DA6EDF6A5350C1
:10B1C8000C0D020EF324D96E010EF420DA6EDF6A3C
:10B1D80053500C0D000EF324D96E010EF420DA6ED4
:10B1E800DE6ADD6A53500C0D040EF324D96E010E8D
:10B1F800F420DA6EDE6ADE6ADE6ADD6A53500C0D10
:10B208000B0EF324D96E010EF420DA6E100EDF6EE9
:10B2180053500C0D0A0EF324D96E010EF420DA6E89
:10B22800020EDF6E53500C0D080EF324D96E010E7A
:10B23800F420DA6E240EDE6EDD6A532AB3D7536A21
:10B248000101586B12008380838E000E0E6E040E6F
:10B258000F6E116A1068010E136E126AE5EC4CF05D
:10B26800FA0E00019C6FFD0E9D6FF0EC67F0CB6B42
:10B27800CC6BCBC04BF0010E4B164B324B3283508C
:10B288004B187F0B4B18836E2E0EE5EC67F08FB4CE
:10B2980015D05350220D000EF32400019E6F030EAB
:10B2A800F4209F6F000EA06F040EA16F010EA36F14
:10B2B800A26BC80EA46F33EC0CF0CA6F0001CA5120
:10B2C80009E0690E9C6FFF0E9D6FCAC09EF09F6BD0
:10B2D800F0EF67F0CB4BCC2BCCBFCBD7CC5103E1F5
:10B2E8000A0ECB5DC6E3070E9C6FFF0E9D6FF0EC58
:10B2F80067F0839E83908390516A1200090E186E3E
:10B308000F5010103BE00FC0D9FF10C0DAFFDE501D
:10B31800DE1034E00FC0D9FF10C0DAFFDECF12F024
:10B32800DDCF13F012C0D9FF13C0DAFFDF5026E0DB
:10B338000FC0D9FF10C0DAFF10EE05F0DE50E1268D
:10B34800DD50E22220EE02F00F50D9261050DA220A
:10B35800E650DE1813E1E650DE1810E10FC0D9FF01
:10B3680010C0DAFF10EE01F0DE50E126DD50E222D7
:10B37800E75013EC68F0126E12A0186A185003E038
:10B38800166A176A08D00FC0D9FF10C0DAFFDECFDF
:10B3980016F0DDCF17F01150D96EDA6A16C0DEFF4D
:10B3A80017C0DDFF1850120020EE03F00E50D9260A
:10B3B8000F50DA22DF50166E176A186A196A20EEE3
:10B3C80002F00E50D9260F50DA22DF5016C013F0C3
:10B3D80017C014F018C015F0126A1210166E135028
:10B3E800176E1450186E1550196E20EE01F00E509D
:10B3F800D9260F50DA22DF5016C013F017C014F008
:10B4080018C015F0126A1210166E1350176E1450E9
:10B41800186E1550196E0EC0D9FF0FC0DAFFDF5035
:10B4280016C013F017C014F018C015F0126A1210E5
:10B43800166E1350176E1450186E1550196E16C0EC
:10B448000EF017C00FF018C010F019C011F012005C
:10B45800256E2550D8A4040C2350241001E1040CB7
:10B4680055B0030C54B608D0090ED8901F362036B4
:10B4780021362236E82EF9D7245006E1020E235C45
:10B4880003E2276A110E02D0276A120E266E26C022
:10B4980028F01FC017F020C018F021C019F022C0F2
:10B4A8001AF0285087EC65F000091DE11DC00EF068
:10B4B8001EC00FF0020E116E106ACEEC61F000098A
:10B4C80008E0020E1E262306D8A0240623502410C6
:10B4D800EDE1120E281807E1176A186A196A1A6A44
:10B4E8000C0E87EC65F019EC68F023502410D8A4F2
:10B4F800010C000CA3EC65F0CC0E9DEC67F0660E19
:10B508009DEC67F080EC67F0276E275005E1216A13
:10B51800226A236A246A1200256A266A2550270FA0
:10B52800D96EDA6A80EC67F0DF6E254A262A26BED5
:10B53800F5D7265003E1040E255CF0E3F20E000176
:10B548009C6FFB0E9D6F27C09EF09F6B28C0A0F0DC
:10B55800A16B29C0A2F0A36B2AC0A4F0A56B27C0D9
:10B56800A6F028C0A7F029C0A8F02AC0A9F0F0ECDE
:10B5780067F02A502910281003E1060E275CC7E35C
:10B5880027C021F028C022F029C023F02AC024F0C7
:10B598001200196A0F0E186E070E1826176A18502F
:10B5A800D96EDA6ADF501A6E1A3A0F0E1A161A1680
:10B5B8001A500CE0BD0E1A24D96EDA6A010EDA228E
:10B5C800DF50E5EC67F0010E196E0BD0190409E1A4
:10B5D800BD0E1A24D96EDA6A010EDA22DF50E5ECC4
:10B5E80067F01850D96EDA6ADF501A6E0F0E1A1605
:10B5F8001A500CE0BD0E1A24D96EDA6A010EDA224E
:10B60800DF50E5EC67F0010E196E0BD0190409E163
:10B61800BD0E1A24D96EDA6A010EDA22DF50E5EC83
:10B6280067F01806172A070E1764B9D7070C446A7B
:10B6380020EE2BF03A50D9263B50DA223C50DE1847
:10B6480009E13D50DE1806E13E50DE1803E13F50A7
:10B65800DE1839E03AC027F03BC028F07AEC48F011
:10B66800446E445030E12F0E3A241D6E000E3B20EC
:10B678001E6E3CC01FF03DC020F03EC021F03FC010
:10B6880022F0246A010E236E20EE01F03A50D926EA
:10B698003B50DA22DF502CEC5AF0000906E03C68F7
:10B6A8003D683E683F68010E446E20EE2BF03A502C
:10B6B800D9263B50DA223CC0DEFF3DC0DEFF3EC04B
:10B6C800DEFF3FC0DEFF445012001150121003E0AD
:10B6D8001150121003E10F50DAEF67F020EE04F07A
:10B6E8001150D9261250DA22DE50DE1016E020EE74
:10B6F80004F01150D9261250DA2210EE02F011503F
:10B70800E1261250E222DE50E65CE650800A176E0F
:10B71800DE50800A1758D8B0120020EE02F01150FF
:10B72800D9261250DA22DECF13F0DDCF14F011C083
:10B73800D9FF12C0DAFFDECF15F0DDCF16F01350B7
:10B748001524D96E14501620DA6E0FC0DFFF20EED4
:10B7580002F01150D9261250DA22DE2A000EDD221C
:10B76800000C02500209026E040E536033D0350EED
:10B778000E6E0B0E0F6E5350050DD10EF324106E86
:10B78800010EF420116E136A050E126ED8EC63F0E8
:10B798003A0E0E6E0B0E0F6E5350130DAA0EF324B5
:10B7A800106E030EF420116E136A130E126ED8EC8D
:10B7B80063F04D0E0E6E0B0E0F6E53500D0D980E5E
:10B7C800F324106E020EF420116E136A0D0E126E21
:10B7D800D8EC63F0030E536409D0010E516E0201D8
:10B7E8001B5110091B6F000EE8CF36FB250EFBEC32
:10B7F8005DF002928390120003D00E4A0F2A102A9D
:10B808001050D96EDA6ADF50116E0EC0F6FF0FC005
:10B81800F7FF000EF86E0E0EF76403D00800F5501F
:10B8280005D0F6CFE9FFF7CFEAFFEF50111813E183
:10B838000EC0F6FF0FC0F7FF000EF86E0E0EF7648D
:10B8480003D00800F55005D0F6CFE9FFF7CFEAFF9F
:10B85800EF500009D2E10EC0F6FF0FC0F7FF000E4F
:10B86800F86E0E0EF76403D00800F55005D0F6CF39
:10B87800E9FFF7CFEAFFEF50116E1050D96EDA6A80
:10B88800DF50115C0E6E0F6AD8A00F061200175019
:10B8980018100AE140C117F041C118F017501810EC
:10B8A80003E1176A186A120017C012F018C013F0E3
:10B8B80019C014F03BEC64F01250172613501822EC
:10B8C80017C0D9FF18C0DAFFDF5006E10101406B4D
:10B8D800416B176A186A120017C012F018C013F0EB
:10B8E80019C014F05BEC64F0125017240101406F8A
:10B8F80013501820416F40C1D9FF41C1DAFFDF5012
:10B9080009E040C1D9FF41C1DAFF000EDF6A404BB0
:10B91800412B02D0406B416B17C017F018C018F0CC
:10B928001200A96BAA6B9FC0ABF0A0C0ACF0A10736
:10B93800D8A0A20727D0A3C074F0A4C075F0A50EA4
:10B94800766F776B796B010E786FB10E7A6F7B6BC0
:10B9580066EC1DF0B105B2111EE1A551AD6FAE6BDD
:10B96800AF6BB06BABC0D9FFACC0DAFFADC0DFFFC7
:10B97800AB4BAC2BA94BAA2B0A0EAD19AE11AF11CC
:10B98800B01109E0A151A95DAA51800A4B6EA251DC
:10B99800800A4B58D0E3ABC0D9FFACC0DAFFDF6AEE
:10B9A800A951AA1103E19F6BA06B12009FC09FF0E1
:10B9B800A0C0A0F01200B3C0B7F0B4C0B8F0B70E82
:10B9C8000E6E1BEC4BF00EC0BBF00FC0BCF00001BC
:10B9D800BCBF0B0CD890BB35D96EBC35DA6E4E0E99
:10B9E800D926010EDA22DECFB9F0DDCFBAF0B9518F
:10B9F800BA1105E0B9C0D9FFBAC0DAFFDF6AB151A0
:10BA0800B21105E0B1C0D9FFB2C0DAFFDF6AD89041
:10BA1800BB35D96EBC35DA6E4E0ED926010EDA2248
:10BA2800B1C0DEFFB2C0DDFFB55101E1000CB30EBD
:10BA38007C6FB10E7D6F7E6B7F6BADEC00F000010B
:10BA4800B66FB65112000EC015F00FC016F010C038
:10BA580017F011C018F01206D8A0130612280CE12E
:10BA680013280AE10E6A0F6A1200154A162A174AA5
:10BA7800182A1206D8A0130615C0F6FF16C0F7FF3D
:10BA88000800F55015E017C0D9FF18C0DAFFDF50DD
:10BA98000FE0125013100CE017C0D9FF18C0DAFFDE
:10BAA80015C0F6FF16C0F7FFDE500900F518DDE0F7
:10BAB80015C0F6FF16C0F7FF0800F5CF14F017C041
:10BAC800D9FF18C0DAFFDF50145C0E6E0F6AD8A0D9
:10BAD8000F061200296E39D020EE01F02550D92624
:10BAE8002650DA22DF502D6E20EE03F02550D9269D
:10BAF8002650DA22DF502C6E20EE05F02550D9268C
:10BB08002650DA22DF502B6E20EE07F02550D9267A
:10BB18002650DA22DF502A6E2AC011F02BC012F00C
:10BB28002CC013F02DC014F07CEF62F025C00EF08D
:10BB380026C00FF080EC43F00EC02AF00FC02BF0A7
:10BB480010C02CF011C02DF0E7D72950276E286AB5
:10BB58002850D8A412002750010ABEE0030AE6E0E4
:10BB680012001E6A1F6A206A216A226A236A246AEE
:10BB7800256A0EA010D016501E2617501F221850E6
:10BB88002022195021221A5022221B5023221C50F5
:10BB980024221D502522D890163617361836193605
:10BBA8001A361B361C361D36D8901532143213320D
:10BBB8001232113210320F320E320E500F10101096
:10BBC80011101210131014101510D3E11EC00EF02E
:10BBD8001FC00FF020C010F021C011F022C012F0D9
:10BBE80023C013F024C014F025C015F01200016E14
:10BBF8000BEE35F08490849A1390F29E83A4FED7BE
:10BC080089688EA8FED78EA81DD0010424E0EE50C6
:10BC1800866E861E8B6A8EA815D08EA2FCD78EA241
:10BC2800FAD789908EA80ED08EB2FCD78EA4FED7F4
:10BC38008980898A8EA806D08EB4FCD78EA802D0B7
:10BC4800012EE1D78B68F90E896E12901298138035
:10BC5800F28E015012008EA2FED702B2899AEE50DF
:10BC6800866E861E8B6ADDD70000ECD70000032E97
:10BC7800FDD7000C25EE04F0DE50DE10FBE000C519
:10BC880016F001C517F0060E1624D96E050E1720FA
:10BC9800DA6EDF50146E060E1624D96E070E1720C2
:10BCA800DA6EDF50156E164A172A1068010E116EEB
:10BCB80016C012F017C013F01050121611501316B8
:10BCC80012C000F513C001F5F29E25EE04F0DE0661
:10BCD800000EDD5AF28E0EC0D9FF0FC0DAFF15C074
:10BCE800DFFF25EE04F0010EDBBE04D0DB5003E1DC
:10BCF800DE0401E28982145012000E501202F3CFC2
:10BD080016F0F4CF17F0186A196A0E501302F350A0
:10BD18001726F4501822000E19220F501202F35061
:10BD28001726F4501822000E19220E501402F35050
:10BD38001826F45019220F501302F3501826F45005
:10BD4800192210501202F3501826F45019221550D7
:10BD58000E02F35019260F501402F35019261050F2
:10BD68001302F350192611501202F350192616C067
:10BD78000EF017C00FF018C010F019C011F0120023
:10BD8800286A296A01016C6B2A6A30D092EC63F048
:10BD98002150221020E02A0E0E6E0F6A3EEC5EF053
:10BDA800276E2AA80CD0BB0E00019C6FFE0E9D6F5B
:10BDB80027C09EF09F6BF0EC67F083900CD0000ECC
:10BDC80001016C25D96EDA6A040EDA2227C0DFFF7A
:10BDD8006C2B284A292A2AAA07D0000E2824256E67
:10BDE800040E2920266E12008EAC02D02904CEE360
:10BDF80028C025F029C026F01200150E146EC60EB4
:10BE0800E82EFED7142EFCD700D020D0150E146EC5
:10BE1800C60EE82EFED7142EFCD700D0010E0E6EEB
:10BE280012C0F6FF13C0F7FF000EF86E0E0EF7648F
:10BE380003D00800F55005D0F6CFE9FFF7CFEAFFA9
:10BE4800EF501FEC63F0124A132AD7D712C0F6FF3F
:10BE580013C0F7FF000EF86E0E0EF76403D008004B
:10BE6800F55005D0F6CFE9FFF7CFEAFFEF5000090C
:10BE7800CDE11200166A176A186A196A125013106F
:10BE88001410151029E0010E1A6E06D0D89012363B
:10BE98001336143615361A2A15AEF8D7D890163632
:10BEA80017361836193612500E5C13500F581450A6
:10BEB80010581550115809E312500E5E13500F5ABE
:10BEC8001450105A1550115A1680D8901532143241
:10BED800133212321A2EE2D716C00EF017C00FF026
:10BEE80018C010F019C011F01200866A846A8B68B5
:10BEF800896801016C6B83928394566B576B0AD0E7
:10BF0800000E5625D96E040E5721DA6E000EDF6E2C
:10BF1800564B572B57BFF4D7575102E15605F0E35C
:10BF2800566B576B09D0350E5625D96E0B0E572117
:10BF3800DA6EDF6A564B572B57BFF5D75705F3E331
:10BF48000F011769D6501F0B4009D66ED6980F0EF1
:10BF5800D612D588D5120E01C29BD58E0F0C1A0E9B
:10BF680017240E6E000E18200F6E0EEC66F00EC031
:10BF78001DF00FC01EF01F6A206A15C0D9FF16C039
:10BF8800DAFF030EDE181CE1140E17240E6E000EE5
:10BF980018200F6E0EEC66F00E50196E0F501A6EC8
:10BFA8001B6A1C6A1AC01CF019C01BF01A6A196AAD
:10BFB80019501D121A501E121B501F121C5020120D
:10BFC8001DC015F01EC016F01FC017F020C018F0D5
:10BFD8001200166E0C0E161807E019EC68F0C2EC89
:10BFE80067F0000901E1FF0C1650400903EC68F006
:10BFF800135003EC68F0125003EC68F0115003EC96
:10C0080068F0105003EC68F0010E156E165002E14E
:10C01800950E156E080E161802E1870E156E15504E
:10C0280003EC68F00C0E161802E10CEC68F00A0E2E
:10C03800156E0CEC68F0146E14AE02D0152EF9D7FC
:10C0480014501200838002500209026E58050DE157
:10C05800000EE8CF35FB500EE8CF36FB000EE8CFD8
:10C0680037FBE8CF38FB586B1DD02BEE35F059C1A4
:10C07800DFFF000EE8CF36FB0D0EE8CF37FB000ED2
:10C08800E8CF38FB8FA403D0600EE8CF38FB8FA42D
:10C0980006D037CB0EF0200E0E120EC037FB010E65
:10C0A800E8CF39FB050EFBEC5DF002920101596BFC
:10C0B8008390120012501310D8B4000C12C0D9FF8C
:10C0C80013C0DAFFDF5001E1000C12C00EF013C0FC
:10C0D8000FF0F9EC63F00EC014F00FC015F0020E6B
:10C0E8001418151001E0000C160E0E6E12C0D9FFC0
:10C0F80013C0DAFFDF50A5EC62F00009D8B4000CD9
:10C10800170E0E6E20EE01F01250D9261350DA22C7
:10C11800DF50A5EC62F0000901E1000C1638F00BC5
:10C1280017101200106E6D0EF66EF80EF76E0900FD
:10C13800F550105C2CE36E0EF66EF80EF76E10508C
:10C148000900F55C04E30F6A010E0E6E010C6F0E18
:10C15800F66EF80EF76E0900F550105C08E3700EE5
:10C16800F66EF80EF76E10500900F55CECE2710EF1
:10C17800F66EF80EF76E0900F550105C08E3720EC3
:10C18800F66EF80EF76E10500900F55CDCE20E6AE8
:10C198000F6A12000EC015F00FC016F010C017F08D
:10C1A80011C018F015C0D9FF16C0DAFFDF50146EA1
:10C1B80017C0F6FF18C0F7FF000EF86E0E0EF764F2
:10C1C80003D00800F55005D0F6CFE9FFF7CFEAFF16
:10C1D800EF50145C196E1A6AD8A01A06174A182A62
:10C1E800154A162A1206D8A013061250131003E097
:10C1F80019501A10D7E019C00EF01AC00FF012002B
:10C208000EC0D9FF0FC0DAFF10C0DFFF0E4A0F2A99
:10C218001150106E1250116E1350126E136A0EC028
:10C22800D9FF0FC0DAFF10C0DFFF0E4A0F2A1150E6
:10C23800106E1250116E1350126E136A0EC0D9FF91
:10C248000FC0DAFF10C0DFFF0E4A0F2A1150106E20
:10C258001250116E1350126E136A0EC0D9FF0FC020
:10C26800DAFF10C0DFFF0E4A0F2A1200536A030ECE
:10C27800536401D02AD053500C0D030EF324D96E09
:10C28800010EF420DA6EDF6A53500C0D020EF3240F
:10C29800D96E010EF420DA6EDF6A53500C0D000ED1
:10C2A800F324D96E010EF420DA6EDE6ADD6A53508B
:10C2B8000C0D040EF324D96E010EF420DA6EDE6A3A
:10C2C800DE6ADE6ADD6A532AD2D7536A83905B6BD3
:10C2D8001200125013101410151023E0010E166EE0
:10C2E80006D0D8901236133614361536162A15AEDF
:10C2F800F8D712500E5C13500F58145010581550A0
:10C30800115808E312500E5E13500F5A1450105A69
:10C318001550115AD8901532143213321232162E83
:10C32800E8D70EC00EF00FC00FF010C010F011C00B
:10C3380011F01200536A0E6A0F6A53501E0D070E51
:10C34800F324D96E020EF420DA6E070EDE6AE806D0
:10C35800FDE253501E0D1B0EF324D96E020EF4207D
:10C36800DA6EDF6A53501E0D170EF324D96E020ED3
:10C37800F420DA6EDE6ADE6ADE6ADD6A0E4A0F2AA9
:10C388000FBEDBD70F5003E1040E0E5CD6E383909B
:10C39800516A1200070E136ED00E126E0FD00CECFD
:10C3A80068F0146E14280DE1E40E00D000D0E82ED9
:10C3B800FCD700D000D01206D8A0130612501310D4
:10C3C800EEE1FE0E141801E0000C0CEC68F00EC053
:10C3D800D9FF0FC0DAFFDF6E0E4A0F2A1006D8A069
:10C3E800110610501110F1E10CEC68F00CEC68F03B
:10C3F800010C0EC014F00FC015F013D01206D8A00F
:10C40800130610C0D9FF11C0DAFF104A112A14C050
:10C41800E1FF15C0E2FF144A152ADFCFE7FFE75016
:10C428000BE01250131008E0E9D714C0D9FF15C06B
:10C43800DAFFDF6A144A152A1206D8A01306122852
:10C44800F4E11328F2E11200BEEC65F0000901E105
:10C45800000C125003EC68F0FD0E12181EE0020EDC
:10C46800146E136A10C0D9FF11C0DAFFDF5003EC55
:10C4780068F0104A112A1306D8A014061350141095
:10C48800F1E10CEC68F00CEC68F00CEC68F0156E5F
:10C4980015501F0B050A01E0000C010C15D00FC048
:10C4A800F6FF10C0F7FF000EF86E0E0EF76403D00B
:10C4B8000800F55005D0F6CFE9FFF7CFEAFFEF50B7
:10C4C800E5EC67F00F4A102A0FC0F6FF10C0F7FF1F
:10C4D800000EF86E0E0EF76403D00800F55005D074
:10C4E800F6CFE9FFF7CFEAFFEF500009D8E11200D5
:10C4F80011C015F012C016F013C017F014C018F0D0
:10C50800A3EC65F0CC0E9DEC67F0990E9DEC67F0FE
:10C518000C0E9DEC67F0196A1A6A1950150FD96E3E
:10C52800DA6ADF509DEC67F0194A1A2A1ABEF5D765
:10C538001A5002E0A3EF65F0040E195CEEE3A3EFD6
:10C5480065F00F6E0E5001E1000C2F0E0F6409D03C
:10C558003A0E0F6006D00E50D96EDA6A0F50D00F1F
:10C5680017D0400E0F6409D0470E0F6006D00E504A
:10C57800D96EDA6A0F50C90F0BD0600E0F64000C29
:10C58800670E0F60000C0E50D96EDA6A0F50A90FB3
:10C59800DF6E010C226E750E236EF80E246E216A72
:10C5A8000AD023C0F6FF24C0F7FF234A242A080034
:10C5B800F550F7E1212A2250211807E023C0F6FFA1
:10C5C80024C0F7FF0800F550ECE1080E00019C6F4D
:10C5D800FE0E9D6F22C09EF09F6B23C0A0F024C06A
:10C5E800A1F0F0EF67F0106E690EF66EF80EF76EB8
:10C5F8000900F550105C1CE36A0EF66EF80EF76E33
:10C6080010500900F55C04E30F6A010E0E6E010C70
:10C618006B0EF66EF80EF76E0900F550105C08E325
:10C628006C0EF66EF80EF76E10500900F55CECE231
:10C638000E6A0F6A12000F6E87920A0EE82EFED756
:10C6480000D00EB002D0879401D08784000E116EFE
:10C65800010E106E0FAE02D0838A01D0839AD89053
:10C668000F36879000F000F0878000F000F0879088
:10C67800104A112A11BEEED7115003E1090E105CC1
:10C68800E9E3878212000109122001000100170066
:10C69800002D119420D00F00010109122001000182
:10C6A800001700002D119420D00F0001010912205D
:10C6B800010001001700002D119420D00F00010186
:10C6C800091220010001001700002D119420D00F3D
:10C6D8000001010E0E6E0F6A88868782878400F03B
:10C6E80000F0879400F000F0106A116A8DA602D05D
:10C6F8000E500F12D8900E36879000F000F0878009
:10C7080000F000F08790104A112A11BEEFD711509F
:10C7180003E1030E105CEAE30F50120025EE04F06B
:10C72800010EDBBE05D0DB5004E10A0EDE5C01E23F
:10C73800898225EE04F0010EDBBE0FD0DE28010E43
:10C74800DE580BE3610E00019C6FFF0E9D6F04C560
:10C758009EF005C59FF0F0EC67F004C521F005C513
:10C7680022F012009F0E166E176814C018F015C03C
:10C7780019F01650182617501922195005E11A0EEB
:10C78800185C02E2010E01D0000E1A6E1B6A1A50E4
:10C798001B1005E05F0E1414146E156A120014C005
:10C7A80014F015C015F0120010C016F011C017F0E3
:10C7B8000EC014F00FC015F010D016C0D9FF17C066
:10C7C800DAFFDF50186E164A172A14C0D9FF15C0B1
:10C7D800DAFF18C0DFFF144A152A1206D8A013067C
:10C7E8001228EBE11328E9E112000EC010F00FC087
:10C7F80011F002D00E4A0F2A0EC0F6FF0FC0F7FF45
:10C80800000EF86E0E0EF76403D00800F55005D040
:10C81800F6CFE9FFF7CFEAFFEF500009EBE1105040
:10C828000E5C0E6E11500F580F6E12000EC014F0F1
:10C838000FC015F010C016F011C017F012501310E9
:10C84800D8B4120016C0D9FF17C0DAFF14C0E1FF30
:10C8580015C0E2FFDFCFE7FF164A172A144A152A48
:10C868001206D8A0130612501310ECE11200156A34
:10C87800166A04D0124A132A154A162A12C0D9FF7A
:10C8880013C0DAFFDF500EE014C00EF012C0D9FF5B
:10C8980013C0DAFFDF500F6E106A47EC67F00E50D6
:10C8A8000F10E8E115C012F016C013F01200156A57
:10C8B800166A04D0124A132A154A162A12C0D9FF3A
:10C8C80013C0DAFFDF500EE014C00EF012C0D9FF1B
:10C8D80013C0DAFFDF500F6E106A47EC67F00E5096
:10C8E8000F10E8E015C012F016C013F012001A0E6F
:10C8F80014240E6E000E15200F6E16C010F017C00F
:10C9080011F020EC67F012C0D9FF13C0DAFF030E54
:10C91800DE18D8A41200140E14240E6E000E152072
:10C928000F6E18C010F019C011F020EF67F05B6BA4
:10C938008380838E000E0E6E040E0F6E116AF60E43
:10C94800106E010E136E126AE5EC4CF0FA0E00013F
:10C958009C6FFD0E9D6FF0EC67F0070E9C6FFF0E4D
:10C968009D6FF0EC67F0839E839012003031323374
:10C97800343536373839414243444546350B1FE78D
:10C98800800102E805800102E805800102E80580CF
:10C998000102E80568706469736B2E636667004876
:09C9A80050393132314400000025
:10C9B2000E6E0E500EE020EC68F0200EE82EFED730
:10C9C20023EC68F0CC0E00D0E82EFDD700D000D0CA
:10C9D200120020EC68F0C00E00D0E82EFDD723EC48
:10C9E20068F0350EE82EFED700F012008E0E446E6F
:10C9F2008AC045F08BC046F0476A486A496A4A6A6B
:10CA0200450E856F866B8CC087F08DC088F0440E12
:10CA1200896F21EC05F0475000018A25D96E4850F4
:10CA22008B21DA6EDF6A000C6DC049F06EC04AF0ED
:10CA32002DEC49F0716F715112E16DC00FF06EC0B3
:10CA420010F06F0E116E82EC59F00001716F71518E
:10CA520006E16DC0D9FF6EC0DAFFDE6ADD6A715190
:10CA62001200000EF2BE010E116E0F50030B7F6E0C
:10CA72000EC07EFF10C080FF3F0E81168184F29EA1
:10CA8200550E826EAA0E826E818281B2FED7819489
:10CA920011B002D0F29E01D0F28E1200350E0E6E4F
:10CAA2000B0E0F6E116A106A010E136E126AE5EC1C
:10CAB2004CF002500209026E2BEE35F05BC1DFFF33
:10CAC200226A010E216E8BEC3DF0029283800101FD
:10CAD2005B6B120002D00E4A0F2A0EC0F6FF0FC087
:10CAE200F7FF0800F55009E00EC0F6FF0FC0F7FF90
:10CAF2000800F55010181110EEE10EC0F6FF0FC03D
:10CB0200F7FF0800F5500E6E0F6A12001B6E1BAE87
:10CB12000ED01B9E106A116A126A136A370EEDEC70
:10CB22005FF01C6E010E1C6402D01C50120017C074
:10CB320010F018C011F019C012F01AC013F01B50F7
:10CB4200EDEF5FF020EC68F00A0E0F6EF80EE82EA3
:10CB5200FED70F2EFCD700D023EC68F0E00E00D0F9
:10CB6200E82EFDD7FAEC67F0090E0F6E840EE82E60
:10CB7200FED70F2EFCD723EF68F0130E0F6E880E30
:10CB82000E6E0ED00CEC68F0FF0A0DE0E40E00D041
:10CB920000D0E82EFCD700D000D00E06D8A00F0699
:10CBA2000E500F10EFE10E500F10D8A4010C000C24
:10CBB200010E146E200E0E180F1011E0F70E106EFB
:10CBC20011680EC012F00FC013F01050122611504F
:10CBD2001322135003E1050E125C01E3146A14C020
:10CBE2000EF00F6A120000004F01000F000000005B
:10CBF20009FF0000004F01000F0000000009FF00C4
:10CC020000004F01000F0000000009FF0000004F6C
:10CC120001000F0000000009FF0020EE01F00E509D
:10CC2200D9260F50DA22DF50136E146A0EC0D9FFD4
:10CC32000FC0DAFFDF50106E1350116E1050136EDA
:10CC420011C014F013C00EF014C00FF012001D6AD0
:10CC52001E6A0BD01CC00FF0106A1AC011F01BC064
:10CC620012F069EC5BF01D4A1E2A1D501824D96E81
:10CC72001E501920DA6EDF501C6E1C50EBE11200C0
:10CC820060900F0E0F01596F070E396F356F4F0EFF
:10CC9200936E8A6A8A888A828A82010E8F6E130E46
:10CCA2000E01B76F0F0EFA6F100EFC6F140EB86FF5
:10CCB200140C9F0E106E1168200E0E10126E000ED4
:10CCC2000F10136E1050122611501322135005E14B
:10CCD2001A0E125C02E2010E01D0000E0E6E0F6AF5
:10CCE200120021BE04D021500FE120040DE220C029
:10CCF20022F021C023F0221E231E224A232A22C010
:10CD020020F023C021F0120020C020F021C021F029
:10CD12001200350E0E6E0B0E0F6E116A106A010EA6
:10CD2200136E126AE5EC4CF0010EE8CF35FB0250AF
:10CD32000209026E010EFBEC5DF0029212009F0EE0
:10CD4200106E11680EC012F00FC013F010501226B0
:10CD520011501322135005E11A0E125C02E2010E69
:10CD620001D0000E0E6E0F6A1200BF0E106E116817
:10CD72000EC012F00FC013F01050122611501322E1
:10CD8200135005E11A0E125C02E2010E01D0000EF0
:10CD92000E6E0F6A1200D00E106E11680EC012F0E5
:10CDA2000FC013F01050122611501322135005E138
:10CDB2000A0E125C02E2010E01D0000E0E6E0F6A24
:10CDC20012009F869E84090E0E01FD6F9F98890EA8
:10CDD2009B6E9C6A9E989D8E9D889D9AC599F28AAB
:10CDE200F28E9E909D9C9E9A9E8A1200136A110E4C
:10CDF200126E09D00A0EE82EFED700D0010E0E6E7A
:10CE0200200E1FEC63F01206D8A013061228F2E1DE
:10CE12001328F0E112000E6E0E5009E0966A4F0ED2
:10CE2200936E220E966E400E956E968A400C966A0E
:10CE3200100E966E2A0E966E900E936EF4D70EC05A
:10CE4200D9FF0FC0DAFF10C0DFFF0E4A0F2A11C050
:10CE520010F0116A0EC0D9FF0FC0DAFF10C0DFFF59
:10CE62000E4A0F2A120020EC68F0200EE82EFED7A0
:10CE720023EC68F0300EE82EFED7FAEC67F00F6E66
:10CE8200B00E00D0E82EFDD70F5012000E50D96E12
:10CE9200DA6A0F50DE1804E10EC00EF00F6A1200BB
:10CEA2000E2A0E04D96EDA6ADF50F0E10E6A0F6ABA
:10CEB20012000EC014F00FC015F014C0D9FF15C037
:10CEC200DAFF10C0DFFF144A152A1206D8A0130693
:10CED20012501310F2E11200070E8C6E9150070BE4
:10CEE2000E6E888A8DAA02D0080E0E26020E01014D
:10CEF200641903E10E1C0F0B0E6E0E501200106A25
:10CF0200116AD890103234EC67F0000901E0108EFB
:10CF1200112A070E1164F5D710501200000EE8CF47
:10CF220000F5E8CF01F5E8CF02F5E8CF03F5E8CF49
:10CF320004F5E8CF05F5000C0F6E106A0F50010BD7
:10CF4200D9EC64F0D8900F32102A070E1064F6D78D
:10CF5200070C020E516E400E02011B6F6A0E000199
:10CF62008A6FFA0E8B6FB6EF67F08C0E446E856B8C
:10CF7200866B8AC087F08BC088F0440E896F21EFE0
:10CF820005F028EC68F00CEC68F0BEEC65F00009E6
:10CF920001E0010C19EC68F0000C0F50030B7F6EDE
:10CFA2000EC07EFF3F0E8116818000F000F080509F
:10CFB20012000E6E03D02AEC68F004000E01CDA917
:10CFC200FAD70EC09AFF12000E6E03D02AEC68F058
:10CFD20004000E01CDA9FAD70EC09AFF12009E0ED0
:10CFE200206E9CC01BF09DC01CF0200E1D6E7EEFBB
:10CFF20028F088888DA803D0010E0E6E01D00E6A2B
:10D002000E5012000E6E0EC092FF0E01CDA1FDD782
:10D01200CD919250120092680E01CDA1FDD7CD9113
:10D02200925012000E6E0E5001E0010C555012008B
:10D0320026EC68F00CEF68F083905B6B120083982B
:10D042008898120083988888120085801200859043
:05D052001200120001B4
:10F8680000819FE0FC407E80FC000020004F4B00A0
:10F878004449534B5F455252004E4F545F524541E5
:10F888004459004E4F5F46494C45004E4F545F4F18
:10F8980050454E4544004E4F545F454E41424C45FD
:10F8A80044004E4F5F46494C455F53595354454DAC
:10F8B80000000D0A202532582025325820253273A1
:10F8C8002025327320253273202532732025327388
:10F8D8002025327320253273202532732025347376
:10F8E8002025347320253473202534732025347360
:10F8F80020253473202534732025347320000D0A05
:10F9080048504469736B204D6B2049492028313891
:10F918004634364B3430292025732025732025732F
:10F92800205374617274696E672E2E2E0D0A000DB5
:10F938000A4461746120706F7274206973202558BD
:10F94800202D2053686F756C64206265203C3E2032
:10F9580030784646000D0A5365656B206572722043
:10F968002564203E2025642C202564203E20256423
:10F978002C202564203E202564000D0A53746174F0
:10F98800757320706F7274206973202558202D209C
:10F9980053686F756C642062652030784646000DA8
:10F9A8000A4461746120706F72742069732025584D
:10F9B800202D2053686F756C64206265203078466E
:10F9C80046000D0A526420752025642072746E204A
:10F9D80025642C2025642062797465732072656122
:10F9E800640D0A000D0A25303458205353383078F6
:10F9F8003A5374617475732C20756E69742025648C
:10FA08003A20256420000D0A4D61782056656374FC
:10FA18006F72206469736B20256420256C6420282C
:10FA2800256C582920000D0A44736B73656C206996
:10FA3800732025642C206E756D62657220697320B1
:10FA4800256420000D0A426C6F636B73697A652028
:10FA5800666F72206469736B2025642069732025A2
:10FA680064000D0A5374617475732073657420748F
:10FA78006F20706F776572206661696C000D0A25CA
:10FA8800303258253032582053533830783A466D42
:10FA980074206F70747300466F756E6420616E20F9
:10FAA8005254432066696C652061742025580D0AFC
:10FAB800004C6F6F6B696E6720666F7220616E20F5
:10FAC8005254432066696C650D0A000D0A55736926
:10FAD8006E67206469736B2067656F6D65747279F2
:10FAE800202573200046696E6446696C652066614E
:10FAF800696C6564207365617263680D0A000D0A9C
:10FB080053746174757320706F7274206973202543
:10FB180058202D204F4B000D0A5365656B20746FDC
:10FB280020256C64206661696C6564202564000D7D
:10FB38000A57726974655F736563746F72732066C0
:10FB480061696C202564000D0A454550524F4D20CF
:10FB58006469736B206E756D626572202564000D93
:10FB68000A4469736B2073656C656374206E756DE8
:10FB7800626572202564005365656B696E67207441
:10FB88006F20736563746F722025580D0A004669EB
:10FB98006E6446696C65206661696C65642072658F
:10FBA80061640D0A000D0A4F70656E696E67206505
:10FBB80078697374696E6720257320000D0A4461A3
:10FBC800746120706F7274206973202558202D206D
:10FBD8004F4B000D0A476F7420256C7520202D208F
:10FBE800726573657474696E6700202558202558FE
:10FBF80020255820255820256C752020200A000D26
:10FC08000A4469736B206368616E67656420746F6A
:10FC1800202564000D0A57726F7465206469736B40
:10FC28006E6F3A20256420000D0A57616974696E69
:10FC38006720666F72206361726420000D0A547237
:10FC48006967706F696E7420697320256420000DE0
:10FC58000A46696C65202573206973206F70656E8C
:10FC680020000D0A7274635F726561642825642C34
:10FC7800255829000D0A253032582530325820459C
:10FC8800786974200020436F6C642025582C202547
:10FC9800582C202558004E6F742061204C4946206E
:10FCA8006469736B0D0A000D0A526561642064650E
:10FCB80073637269626520000D0A46696C652025C8
:10FCC8005820697320257320000D0A4469736B203E
:10FCD800255820697320257320002041544E206147
:10FCE80073736572746564202564000D0A48737423
:10FCF80020627974657332202564000D0A204F70E4
:10FD080074696F6E732025640D0A000D0A577269B5
:10FD18007465206661696C202564000D0A5265616E
:10FD280064696E67205254430D0A000D0A416D69DB
:10FD3800676F2039313231440D0A000D0A53532FB1
:10FD480038302039313232440D0A000D0A44736BC1
:10FD580073656C20697320256420000D0A52656163
:10FD68006420256420627974657300566563746F36
:10FD7800722069732025580D0A000D0A5353383034
:10FD8800782025642025642000222A2B2C3A3B3C2D
:10FD98003D3E3F5B5D7C7F000D0A4F70656E696E6E
:10FDA800672025732020000D0A4465627567206965
:10FDB8007320256420000D0A436C6F636B20697300
:10FDC80020256420000D0A50726F746F206973201B
:10FDD800256420000D0A5265616420636F6E6669B0
:10FDE8006720000D0A46696C656E616D6520257394
:10FDF80020000D0A466F726D617474696E67200089
:10FE080072633D25752046525F25730D0A002A2A24
:10FE1800204E4F204449534B202A2A002A2A205694
:10FE28006572696679202A2A000D0A7362797465F9
:10FE38007331202564000D0A41737365727420457F
:10FE48004F49000D0A4173736572742041544E0086
:10FE58000D0A4E6F20636172642025640064657327
:10FE680063726962652E636667002F6C69666461F8
:10FE780074612E62696E000D0A456E61626C6520C0
:10FE8800505000EB76904558464154202020000DF4
:10FE98000A4D6F756E74696E6720004E6F7620325A
:10FEA800312032303233000D0A4173736572742089
:10FEB80050500020255820772041544E20000D0A2C
:10FEC800476F742041544E31000D0A476F7420412A
:10FED800544E32000D0A476F742041544E33004C83
:10FEE8006F6164696E672E2E2E00204944202558C4
:10FEF80025303258002A2A20525141202A2A004609
:10FF08006D74206578697420000D0A476F74204964
:10FF18004643002025643A20253032580020476F98
:10FF2800742041544E0031383A30323A3434005B50
:10FF38002532582025645D004572726F7220256451
:10FF48000048504469736B20003C6964656E743ED8
:10FF5800004E6F2063617264004669466F20255821
:10FF68000072633D2564200044534B53454C004EBA
:10FF7800414D452558004449534B255800464154A6
:10FF880033320044454255470050524F544F0052B7
:10FF980065616479000D0A257320007B4552527D06
:10FFA80000302E3236004946432000454F49200094
:10FFB80052454E2000535251200044415620004ED5
:10FFC800444143004E524644004641540052544373
:10FFD8000054524700434C4B00253258004430002F
:10FFE8004431004432004433004434004435004472
:08FFF80036004437002B000025
:020000040020DA
:10000000FF0FFF0FFF0FFF0FFF0FFF0FFF0FFF0F80
:020000040030CA
:0C0000008CFFFFFC8EFFFFFFFFFFFFFFE7
:00000001FF
